:020000040800F2
:1000000000060020E1010008E3010008E301000808
:10001000E3010008E3010008E3010008E301000830
:10002000E3010008E3010008E3010008692F00086C
:10003000E3010008E3010008E3010008E301000810
:10004000E3010008E3010008E3010008E301000800
:10005000E3010008E301000811320008393200080A
:100060006132000889320008B1320008E30100085B
:10007000E3010008E3010008E3010008E3010008D0
:10008000E3010008E3010008E3010008E3010008C0
:10009000E3010008E3010008E3010008D932000889
:1000A000E3010008E3010008E3010008E3010008A0
:1000B000AD330008E3010008E3010008E301000894
:1000C000E3010008E3010008E3010008E301000880
:1000D000E3010008E3010008E3010008E301000870
:1000E0003D330008E3010008E3010008E3010008D4
:1000F000E3010008E3010008E3010008E301000850
:10010000E3010008E3010008E3010008E30100083F
:10011000E3010008E3010008E3010008E30100082F
:10012000E3010008E3010008E3010008E30100081F
:10013000E3010008E3010008E3010008E30100080F
:10014000E3010008E3010008E30100081D2700089F
:10015000E3010008E3010008E3010008E3010008EF
:10016000E3010008E3010008E3010008E3010008DF
:10017000E3010008E3010008E3010008E3010008CF
:10018000E3010008E3010008E3010008E3010008BF
:10019000E3010008E3010008E3010008E3010008AF
:1001A000E3010008E3010008E3010008E30100089F
:1001B000E3010008E3010008E3010008E30100088F
:1001C000E3010008E3010008E3010008E30100087F
:1001D000E3010008E3010008E3010008E30100086F
:1001E00002E000F000F8FEE772B6374880F30888B6
:1001F000364880F3098836483649086040F20000E6
:10020000CCF200004EF63471CEF200010860BFF36C
:100210004F8FBFF36F8F40F20000C0F2F0004EF638
:100220008851CEF200010860BFF34F8FBFF36F8F8C
:100230004FF00000E1EE100A4EF63C71CEF20001E4
:100240000860062080F31488BFF36F8F01F02EFF43
:1002500002F028FE4FF055301F491B4A91423CBF27
:1002600041F8040BFAE71D49184A91423CBF41F896
:10027000040BFAE71A491B4A1B4B9A423EBF51F83E
:10028000040B42F8040BF8E700201849184A914281
:100290003CBF41F8040BFAE701F00CFF02F056FEF8
:1002A000144C154DAC4203DA54F8041B8847F9E7A7
:1002B00000F042F8114C124DAC4203DA54F8041B22
:1002C0008847F9E701F0F4BE000600200022002074
:1002D0000000000808ED00E00000002000060020FB
:1002E0007837000800220020402200204022002011
:1002F000602E0020E0010008E0010008E001000895
:10030000E00100082DE9F04F2DED108AC1F80CD066
:10031000C3689D46BDEC108ABDE8F08F002383F3CF
:1003200011882846A047002001F072FAFEE701F08C
:1003300001FA00DFFEE7000038B500F0BBFB01F07A
:1003400085FE054601F0A8FE0446C8B90E4B9D4245
:1003500018D001339D4218BF044641F2883504BFCE
:1003600001240025002001F07BFE0CB100F074F8A0
:1003700000F000FD284600F0BFF800F06DF8F9E746
:100380000025EFE70546EDE7010007B008B500F0EE
:1003900063FBA0F120035842584108BD07B541F264
:1003A0001203022101A8ADF8043000F073FB03B082
:1003B0005DF804FB38B5302383F3118817480368D0
:1003C0000BB101F0F1FA164A144800234FF47A7188
:1003D00001F0E0FA002383F31188124C236813B173
:1003E0002368013B2360636813B16368013B63606A
:1003F0000D4D2B7833B963687BB9022000F024FCE3
:10040000322363602B78032B07D163682BB902205A
:1004100000F01AFC4FF47A73636038BD402200206C
:10042000B50300086023002058220020084B1870F4
:1004300003280CD8DFE800F008050208022000F0CD
:10044000F9BB022000F0ECBB024B00225A6070475F
:100450005822002060230020234B244A10B51C465C
:10046000196801313FD004339342F9D16268A24246
:1004700039D31F4B9B6803F1006303F540439A4255
:1004800031D2002000F030FB0220FFF7CFFF194BE4
:100490001A6C00221A64196E1A66196E596C5A6425
:1004A000596E5A665A6E5A6942F080025A615A6908
:1004B00022F080025A615A691A6942F000521A61A8
:1004C0001A6922F000521A611B6972B64FF0E023DC
:1004D0003021C3F8084DD4E9003281F311889D46DC
:1004E00083F30888104710BD00C0000820C0000832
:1004F00000220020003802402DE9F04F93B0AA4BB3
:1005000000902022FF210AA89D6800F0DDFBA74A89
:100510001378A3B9A648012103601170302383F337
:10052000118803680BB101F03FFAA24AA0480023EA
:100530004FF47A7101F02EFA002383F31188009BA7
:1005400013B19D4B009A1A609C4A009C1378032BB0
:100550001EBF00231370984A4FF0000A18BF536063
:10056000D3465646D146012000F064FB24B1924B9D
:100570001B68002B00F01182002000F06DFA039040
:10058000039B002BF2DB012000F04AFB039B213B85
:10059000162BE8D801A252F823F000BFF905000895
:1005A00021060008B5060008670500086705000871
:1005B000670500083F0700080F0900082908000820
:1005C0008B080008B3080008D90800086705000870
:1005D000EB080008670500085D0900089906000897
:1005E00067050008A109000805060008990600082B
:1005F000670500088B0800080220FFF7C7FE0028E7
:1006000040F0F581009B0221BAF1000F08BF1C46A3
:1006100005A841F21233ADF8143000F03BFAA2E71E
:100620004FF47A7000F018FA071EEBDB0220FFF798
:10063000ADFE0028E6D0013F052F00F2DA81DFE8A9
:1006400007F0030A0D10133605230593042105A8AE
:1006500000F020FA17E054480421F9E75848042133
:10066000F6E758480421F3E74FF01C08404600F035
:100670003DFA08F104080590042105A800F00AFAE3
:10068000B8F12C0FF2D1012000FA07F747EA0B0B63
:100690005FFA8BFB4FF0000900F062FB26B10BF014
:1006A0000B030B2B08BF0024FFF778FE5BE74648DF
:1006B0000421CDE7002EA5D00BF00B030B2BA1D10D
:1006C0000220FFF763FE074600289BD0012000F0C0
:1006D0000BFA0220FFF7AAFE00261FFA86F8404612
:1006E00000F012FA044690B10021404600F01CFAD6
:1006F00001360028F1D1BA46044641F21213022114
:1007000005A8ADF814303E4600F0C4F92BE70120EF
:10071000FFF78CFE2546244B9B68AB4207D9284641
:1007200000F0E4F9013040F067810435F3E7234B32
:1007300000251D70204BBA465D603E46ACE7002E9A
:100740003FF460AF0BF00B030B2B7FF45BAF022089
:10075000FFF76CFE322000F07FF9B0F10008FFF6E1
:1007600051AF18F003077FF44DAF0F4A926808EBC2
:10077000050393423FF646AFB8F5807F3FF742AF9F
:10078000124B0193B84523DD4FF47A7000F064F901
:100790000390039A002AFFF635AF019B039A03F8F2
:1007A000012B0137EDE700BF002200205C23002071
:1007B00040220020B50300086023002058220020BA
:1007C00004220020082200200C2200205C220020AD
:1007D000C820FFF7DBFD074600283FF413AF1F2DAD
:1007E00011D8C5F1200242450AAB25F0030028BF0D
:1007F000424683490192184400F040FA019A804829
:10080000FF2100F061FA4FEAA8037D490193C8F384
:100810008702284600F060FA064600283FF46DAFD4
:10082000019B05EB830537E70220FFF7AFFD0028AA
:100830003FF4E8AE00F0A4F900283FF4E3AE00274F
:10084000B846704B9B68BB4218D91F2F11D80A9B22
:1008500001330ED027F0030312AA134453F8203CAF
:1008600005934046042205A900F0AEFA04378046FD
:10087000E7E7384600F03AF90590F2E7CDF8148042
:10088000042105A800F006F906E70023642104A866
:10089000049300F0F5F800287FF4B4AE0220FFF7CF
:1008A00075FD00283FF4AEAE049800F051F90590B4
:1008B000E6E70023642104A8049300F0E1F800288F
:1008C0007FF4A0AE0220FFF761FD00283FF49AAE4E
:1008D000049800F04DF9EAE70220FFF757FD0028E1
:1008E0003FF490AE00F05CF9E1E70220FFF74EFD27
:1008F00000283FF487AE05A9142000F057F9042121
:100900000746049004A800F0C5F83946B9E732203C
:1009100000F0A2F8071EFFF675AEBB077FF472AEBB
:10092000384A926807EB090393423FF66BAE022008
:10093000FFF72CFD00283FF465AE27F003074F4476
:10094000B9453FF4A9AE484600F0D0F8042105901F
:1009500005A800F09FF809F10409F1E74FF47A7057
:10096000FFF714FD00283FF44DAE00F009F9002810
:1009700044D00A9B01330BD008220AA9002000F0C2
:10098000ABF900283AD02022FF210AA800F09CF9F8
:10099000FFF704FD1C4800F041FF13B0BDE8F08FE5
:1009A000002E3FF42FAE0BF00B030B2B7FF42AAE7F
:1009B0000023642105A8059300F062F8074600288B
:1009C0007FF420AE0220FFF7E1FC804600283FF4D0
:1009D00019AEFFF7E3FC41F2883000F01FFF0598E5
:1009E00000F0F0F9464600F0BBF93C46BBE5064690
:1009F00052E64FF0000905E6BA467EE637467CE649
:100A00005C22002000220020A086010070B50F4B60
:100A10001B780133DBB2012B0C4611D80C4D296831
:100A20004FF47A730E6AA2FB03320146224628462F
:100A3000B047844204D1074B00221A70012070BDD8
:100A40004FF4FA7000F0EAFE0020F8E710220020D0
:100A5000082600209423002007B500230246012128
:100A60000DF107008DF80730FFF7D0FF20B19DF89A
:100A7000070003B05DF804FB4FF0FF30F9E700001A
:100A80000A4608B50421FFF7C1FF80F00100C0B29B
:100A9000404208BD30B4054C2368DD69044B0A466A
:100AA000AC460146204630BC604700BF0826002007
:100AB000A086010070B501F0CFF9094E094D3080D4
:100AC000002428683388834208D901F0BFF92B68D5
:100AD00004440133B4F5404F2B60F2D370BD00BF26
:100AE000962300206823002001F064BA00F1006022
:100AF00000F540400068704700F10060920000F58A
:100B0000404001F0EFB90000054B1A68054B1B8807
:100B10009B1A834202D9104401F098B90020704713
:100B2000682300209623002038B5084D044629B1DB
:100B300028682044BDE8384001F0A8B9286820445E
:100B400001F08CF90028F3D038BD00BF68230020E5
:100B500010F003030AD1B0F5047F05D200F1005074
:100B6000A0F51040D0F80038184670470023FBE786
:100B700000F10050A0F51040D0F8100A70470000B6
:100B8000064991F8243033B10023086A81F82430F3
:100B90000822FFF7B1BF0120704700BF6C2300207F
:100BA000014B1868704700BF002004E070B5194B76
:100BB0001D68194B0138C5F30B0408442D0C0422A1
:100BC0001E88A6420BD15C680A46013C824213464D
:100BD0000FD214F9016F4EB102F8016BF6E7013A3A
:100BE00003F10803ECD181420B4602D22C2203F818
:100BF000012B0A4A05241688AE4204D1984284BFCC
:100C0000967803F8016B013C02F10402F3D1581A03
:100C100070BD00BF002004E0903400087C34000860
:100C2000022802BF024B4FF080729A61704700BFEA
:100C300000000240022802BF024B4FF480729A610A
:100C4000704700BF00000240022801BF024A5369FA
:100C500083F48073536170470000024070B504460E
:100C60004FF47A764CB1412C254628BF412506FB2E
:100C700005F000F0D3FD641BF4E770BD10B5002350
:100C8000934203D0CC5CC4540133F9E710BD00009B
:100C900010B5013810F9013F3BB191F900409C4279
:100CA00003D11AB10131013AF4E71AB191F90020E8
:100CB000981A10BD1046FCE703460246D01A12F9F6
:100CC000011B0029FAD1704702440346934202D027
:100CD00003F8011BFAE770472DE9F8431F4D14464E
:100CE00095F824200746884652BBDFF870909CB3E5
:100CF00095F824302BB92022FF2148462F62FFF7B8
:100D0000E3FF95F82400C0F10802A24228BF224662
:100D1000D6B24146920005EB8000FFF7AFFF95F891
:100D20002430A41B1E44F6B2082E17449044E4B2AB
:100D300085F82460DBD1FFF723FF0028D7D108E036
:100D40002B6A03EB82038342CFD0FFF719FF002801
:100D5000CBD10020BDE8F8830120FBE76C23002005
:100D6000024B1A78024B1A70704700BF9423002080
:100D70001022002010B5104C104800F0B5F82146A4
:100D80000E4800F0DDF82468626DD2F8043843F0B4
:100D90000203C2F804384FF47A70FFF75FFF084986
:100DA000204600F0D3F9626DD2F8043823F0020334
:100DB000C2F8043810BD00BF5C35000808260020CA
:100DC000643500087047000030B5094D0A4491426F
:100DD0000DD011F8013B5840082340F30004013BBB
:100DE0002C4013F0FF0384EA5000F6D1EFE730BD4A
:100DF0002083B8ED026843681143016003B11847CE
:100E00007047000013B5446BD4F894341A68117815
:100E1000042915D1217C022912D1197912890123C3
:100E20008B4013420CD101A904F14C0001F0F6FEF5
:100E3000D4F89444019B21790246206800F0D0F94F
:100E400002B010BD143001F079BE00004FF0FF3346
:100E5000143001F073BE00004C3001F04BBF0000B5
:100E60004FF0FF334C3001F045BF0000143001F06B
:100E700047BE00004FF0FF31143001F041BE0000CA
:100E80004C3001F017BF00004FF0FF324C3001F042
:100E900011BF00000020704710B5D0F894341A68D4
:100EA00011780429044617D1017C022914D15979FB
:100EB000528901238B4013420ED1143001F0DAFD28
:100EC000024648B1D4F894444FF4807361792068A5
:100ED000BDE8104000F072B910BD0000406BFFF794
:100EE000DBBF0000704700007FB5124B036000239A
:100EF0004360C0E90233012502260F4B0574044606
:100F00000290019300F18402294600964FF4807309
:100F1000143001F08BFD094B0294CDE9006304F518
:100F200023724FF48073294604F14C0001F052FE05
:100F300004B070BDB0340008DD0E0008050E0008D6
:100F40000B68302282F311880A7903EB82029061E8
:100F50004A79093243F822008A7912B103EB8203FD
:100F600098610223C0F894140374002080F3118860
:100F70007047000038B5037F044613B190F8543031
:100F8000ABB9201D01250221FFF734FF04F1140045
:100F900025776FF0010100F069FC84F8545004F1EA
:100FA0004C006FF00101BDE8384000F05FBC38BD77
:100FB00010B5012104460430FFF71CFF00232377FE
:100FC00084F8543010BD000038B5044600251430B4
:100FD00001F044FD04F14C00257701F013FE201DC3
:100FE00084F854500121FFF705FF2046BDE8384042
:100FF000FFF752BF90F8443003F06003202B07D175
:1010000090F84520212A4FF0000303D81F2A06D864
:1010100000207047222AFBD1C0E90E3303E0034AC7
:1010200082630722C26303640120704711220020FB
:1010300037B5D0F894341A681178042904461AD1C7
:10104000017C022917D11979128901238B4013429F
:1010500011D100F14C05284601F094FE58B101A9C8
:10106000284601F0DBFDD4F89444019B2179024627
:10107000206800F0B5F803B030BD0000F0B500EB1B
:10108000810385B09E6904460D46FEB1302383F38B
:10109000118804EB8507301D0821FFF7ABFEFB68C4
:1010A0005B691B6806F14C001BB1019001F0C4FDA7
:1010B000019803A901F0B2FD024648B1039B2946FD
:1010C000204600F08DF8002383F3118805B0F0BDB1
:1010D000FB685A691268002AF5D01B8A013B13404D
:1010E000F1D104F14402EAE7093138B550F8214062
:1010F000DCB1302383F31188D4F894241368527937
:1011000003EB8203DB689B695D6845B104216018CD
:10111000FFF770FE294604F1140001F0B5FC2046EB
:10112000FFF7BAFE002383F3118838BD7047000033
:1011300001F014B8012303700023C0E90133C36137
:1011400083620362C36243620363704738B5044637
:10115000302383F311880025C0E90355C0E9055504
:10116000416001F00BF80223237085F311882846B3
:1011700038BD000070B500EB810305465069DA60A8
:101180000E46144618B110220021FFF79DFDA069FC
:1011900018B110220021FFF797FD31462846BDE81F
:1011A000704001F0B5B80000826802F00112826060
:1011B0000022C0E90422826101F036B9F0B400EBEC
:1011C00081044789E4680125A4698D403D43458138
:1011D00023600023A2606360F0BC01F051B90000FD
:1011E000F0B400EB81040789E468012564698D404F
:1011F0003D43058123600023A2606360F0BC01F0E1
:10120000CBB9000070B50223002504460370C0E985
:101210000255C0E90455C564856180F8345001F079
:1012200013F863681B6823B129462046BDE8704067
:10123000184770BD0378052B10B504460AD080F816
:1012400050300523037043681B680BB10421984795
:101250000023A36010BD00000178052906D190F895
:101260005020436802701B6803B1184770470000A4
:1012700070B590F83430044613B1002380F8343050
:1012800004F14402204601F0F1F863689B68B3B9A9
:1012900094F8443013F0600535D00021204601F069
:1012A00091FB0021204601F083FB63681B6813B1AA
:1012B000062120469847062384F8343070BD204626
:1012C00098470028E4D0B4F84A30E26B9A4288BFCD
:1012D000E36394F94430E56B002B4FF0300380F268
:1012E0000381002D00F0F280092284F8342083F37A
:1012F00011880021D4E90E232046FFF771FF002357
:1013000083F31188DAE794F8452003F07F0343EA7A
:10131000022340F20232934200F0C58021D8B3F597
:10132000807F48D00DD8012B3FD0022B00F0938056
:10133000002BB2D104F14C02A2630222E2632364C7
:10134000C1E7B3F5817F00F09B80B3F5407FA4D166
:1013500094F84630012BA0D1B4F84C3043F002038E
:1013600032E0B3F5006F4DD017D8B3F5A06F31D090
:10137000A3F5C063012B90D8636894F846205E689B
:1013800094F84710B4F848302046B047002884D07D
:101390004368A3630368E3631AE0B3F5106F36D0C4
:1013A00040F6024293427FF478AF5C4BA363022382
:1013B000E3630023C3E794F84630012B7FF46DAF5D
:1013C000B4F84C3023F00203C4E90E55A4F84C30B5
:1013D000256478E7B4F84430B3F5A06F0ED194F8E3
:1013E000463084F84E30204600F086FF63681B6864
:1013F00013B1012120469847032323700023C4E939
:101400000E339CE704F14F03A3630123C3E7237862
:10141000042B10D1302383F311882046FFF7C4FE3C
:1014200085F311880321636884F84F5021701B688D
:101430000BB12046984794F84630002BDED084F854
:101440004F300423237063681B68002BD6D0022121
:1014500020469847D2E794F848301D0603F00F0164
:1014600020460AD500F0F4FF012804D002287FF4BA
:1014700014AF2B4B9AE72B4B98E700F0DBFFF3E719
:1014800094F84630002B7FF408AF94F8483013F0FE
:101490000F01B3D01A06204602D501F0A7FAADE736
:1014A00001F09AFAAAE794F84630002B7FF4F5AEE3
:1014B00094F8483013F00F01A0D01B06204602D547
:1014C00001F080FA9AE701F073FA97E7142284F8A2
:1014D000342083F311882B462A4629462046FFF7FD
:1014E0006DFE85F31188E9E65DB1152284F834209C
:1014F00083F311880021D4E90E232046FFF75EFE16
:10150000FDE60B2284F8342083F311882B462A460B
:1015100029462046FFF764FEE3E700BFE0340008F9
:10152000D8340008DC34000838B590F8343004466C
:10153000002B3ED0063BDAB20F2A34D80F2B32D81C
:10154000DFE803F0373131082232313131313131C6
:1015500031313737C56BB0F84A309D4214D2C36879
:101560001B8AB5FBF3F203FB12556DB9302383F3ED
:1015700011882B462A462946FFF732FE85F311884B
:101580000A2384F834300EE0142384F834303023F6
:1015900083F3118800231A4619462046FFF70EFEF2
:1015A000002383F3118838BD036C03B198470023EF
:1015B000E7E70021204601F005FA0021204601F06E
:1015C000F7F963681B6813B1062120469847062384
:1015D000D7E7000010B590F83430142B044629D01A
:1015E00017D8062B05D001D81BB110BD093B022B23
:1015F000FBD80021204601F0E5F90021204601F04A
:10160000D7F963681B6813B1062120469847062363
:1016100019E0152BE9D10B2380F83430302383F304
:10162000118800231A461946FFF7DAFD002383F3D9
:101630001188DAE7C3689B695B68002BD5D1036C1E
:1016400003B19847002384F83430CEE700230375B4
:10165000826803691B6899689142FBD25A680360EB
:101660004260106058607047002303758268036908
:101670001B6899689142FBD85A6803604260106009
:101680005860704708B50846302383F311880B7DF6
:10169000032B05D0042B0DD02BB983F3118808BD83
:1016A0008B6900221A604FF0FF338361FFF7CEFF92
:1016B0000023F2E7D1E9003213605A60F3E700003B
:1016C000FFF7C4BF054BD9680875186802681A602F
:1016D000536001220275D860FEF714BE98230020E3
:1016E00030B50C4BDD684B1C87B004460FD02B4641
:1016F000094A684600F04EF92046FFF7E3FF009BD9
:1017000013B1684600F050F9A86907B030BDFFF783
:10171000D9FFF9E79823002085160008044B1A68C2
:10172000DB6890689B68984294BF00200120704756
:1017300098230020084B10B51C68D86822681A60EE
:10174000536001222275DC60FFF78EFF01462046C0
:10175000BDE81040FEF7D6BD9823002038B5074CF1
:1017600007490848012300252370656001F042FB0A
:101770000223237085F3118838BD00BF00260020A6
:10178000E83400089823002000F044B9034A516867
:1017900053685B1A9842FBD8704700BF001000E006
:1017A0008B60022308618B82084670478368A3F12F
:1017B000840243F8142C026943F8442C426943F82C
:1017C000402C094A43F8242CC26843F8182C022202
:1017D00003F80C2C002203F80B2C044A43F8102CBD
:1017E000A3F12000704700BF1D03000898230020CC
:1017F00008B5FFF7DBFFBDE80840FFF761BF000059
:10180000024BDB6898610F20FFF75CBF9823002034
:10181000302383F31188FFF7F3BF000008B50146BA
:10182000302383F311880820FFF75AFF002383F346
:10183000118808BD064BDB6839B1426818605A60F0
:10184000136043600420FFF74BBF4FF0FF30704739
:10185000982300200368984206D01A6802605060FE
:1018600099611846FFF72CBF7047000038B5044651
:101870000D462068844200D138BD036823605C6057
:101880008561FFF71DFFF4E710B503689C68A2426D
:101890000CD85C688A600B604C6021605960996864
:1018A0008A1A9A604FF0FF33836010BD1B68121BC9
:1018B000ECE700000A2938BF0A2170B504460D463E
:1018C0000A26601901F090FA01F07CFA041BA54287
:1018D00003D8751C2E460446F3E70A2E04D9BDE84A
:1018E0007040012001F0C6BA70BD0000F8B5144B7D
:1018F0000D46D96103F1100141600A2A196982601D
:1019000038BF0A22016048601861A818144601F027
:101910005DFA0A2701F056FA431BA342064606D396
:101920007C1C281901F060FA27463546F2E70A2F99
:1019300004D9BDE8F840012001F09CBAF8BD00BF11
:1019400098230020F8B506460D4601F03BFA0F4AF1
:10195000134653F8107F9F4206D12A46014630466F
:10196000BDE8F840FFF7C2BFD169BB68441A2C1923
:1019700028BF2C46A34202D92946FFF79BFF2246E7
:1019800031460348BDE8F840FFF77EBF98230020AA
:10199000A823002010B4C0E9032300235DF8044B02
:1019A0004361FFF7CFBF000010B5194C236998427F
:1019B0000DD0D0E90032816813605A609A680A44F9
:1019C0009A60002303604FF0FF33A36110BD2346EC
:1019D000026843F8102F53600022026022699A4285
:1019E00003D1BDE8104001F0F9B9936881680B4458
:1019F000936001F0E7F92269E1699268441AA24212
:101A0000E4D91144BDE81040091AFFF753BF00BFE5
:101A1000982300202DE9F047DFF8BC8008F110077B
:101A20002C4ED8F8105001F0CDF9D8F81C40AA6817
:101A3000031B9A423ED81444D5E900324FF0000906
:101A4000C8F81C4013605A60C5F80090D8F81030F0
:101A5000B34201D101F0C2F989F31188D5E903310C
:101A600028469847302383F311886B69002BD8D020
:101A700001F0A8F96A69A0EB04094A4582460DD233
:101A8000022001F0F7F90022D8F81030B34208D153
:101A900051462846BDE8F047FFF728BF121A2244F6
:101AA000F2E712EB090938BF4A4629463846FFF7E4
:101AB000EBFEB5E7D8F81030B34208D01444211A31
:101AC000C8F81C00A960BDE8F047FFF7F3BEBDE809
:101AD000F08700BFA8230020982300200020704733
:101AE000FEE70000704700004FF0FF307047000035
:101AF00002290CD0032904D00129074818BF00206F
:101B00007047032A05D8054800EBC2007047044817
:101B100070470020704700BFC03500082022002019
:101B20007435000870B59AB00546084601A91446F8
:101B300000F0C2F801A8FFF7BFF8431C5B00C5E93D
:101B400000340022237003236370C6B201AB023459
:101B50001046D1B28E4204F1020401D81AB070BD11
:101B600013F8011B04F8021C04F8010C0132F0E721
:101B700008B5302383F311880348FFF759FA00238F
:101B800083F3118808BD00BF0826002090F8443078
:101B900003F01F02012A07D190F845200B2A03D138
:101BA0000023C0E90E3315E003F06003202B08D1B9
:101BB000B0F848302BB990F84520212A03D81F2AC5
:101BC00004D8FFF717BA222AEBD0FAE7034A826358
:101BD0000722C26303640120704700BF182200205F
:101BE00007B5052917D8DFE801F0191603191920E0
:101BF000302383F31188104A01900121FFF7BAFACC
:101C000001980E4A0221FFF7B5FA0D48FFF7DCF9FB
:101C1000002383F3118803B05DF804FB302383F3C2
:101C200011880748FFF7A6F9F2E7302383F31188FC
:101C30000348FFF7BDF9EBE7143500083835000815
:101C40000826002038B50C4D0C4C0D492A4604F1ED
:101C50000800FFF767FF05F1CA0204F11000094907
:101C6000FFF760FF05F5CA7204F118000649BDE8E8
:101C70003840FFF757BF00BFD02A002020220020A5
:101C8000F4340008FE3400080935000870B5044635
:101C900008460D46FFF710F8C6B220460134037817
:101CA0000BB9184670BD32462946FEF7F1FF0028F1
:101CB000F3D10120F6E700002DE9F04705460C4678
:101CC000FEF7FAFF2A49C6B22846FFF7DFFF08B140
:101CD0000936F6B227492846FFF7D8FF08B1103673
:101CE000F6B2632E0BD8DFF88880DFF88890224F99
:101CF000DFF890A02E7846B92670BDE8F087294617
:101D00002046BDE8F04701F09BBB252E2CD10722D1
:101D100041462846FEF7BCFF60B9184B224603F146
:101D2000100153F8040B42F8040B8B42F9D107352C
:101D30001034DFE7082249462846FEF7A9FF98B984
:101D40000F4BA21C197809090232C95D02F8041C64
:101D500013F8011B01F00F015345C95D02F8031C84
:101D6000F0D118340835C5E704F8016B0135C1E737
:101D7000E035000809350008F9350008E8350008A5
:101D8000107AFF1F1C7AFF1FBFF34F8F024AD368E0
:101D9000DB03FCD4704700BF003C024008B5094B90
:101DA0001B7873B9FFF7F0FF074B1A69002ABFBF12
:101DB000064A5A6002F188325A601A6822F4806238
:101DC0001A6008BD2E2D0020003C0240230167450B
:101DD00008B50B4B1B7893B9FFF7D6FF094B1A696F
:101DE00042F000421A611A6842F480521A601A687E
:101DF00022F480521A601A6842F480621A6008BDA8
:101E00002E2D0020003C02400B28F0B516D80C4CBB
:101E10000C4923787BB90C4D0E460C234FF0006221
:101E200055F8047B46F8042B013B13F0FF033A44BA
:101E3000F6D10123237051F82000F0BD0020FCE70B
:101E4000602D0020302D00200C360008014B53F887
:101E5000200070470C3600080C2070470B2810B586
:101E6000044601D9002010BDFFF7CEFF064B53F802
:101E700024301844C21A0BB90120F4E71268013269
:101E8000F0D1043BF6E700BF0C3600080B2810B574
:101E9000044621D8FFF778FFFFF780FF0F4AF323AE
:101EA000D360C300DBB243F4007343F00203136159
:101EB000136943F480331361FFF766FFFFF7A4FF54
:101EC000074B53F8241000F0D9F8FFF781FF2046A4
:101ED000BDE81040FFF7C2BF002010BD003C02402B
:101EE0000C360008F8B512F00103144642D18218EE
:101EF000B2F1016F57D82D4B1B6813F0010352D07C
:101F00002B4DFFF74BFFF323EB60FFF73DFF40F254
:101F10000127032C15D824F001046618244C401A1C
:101F200040F20117B142236900EB010524D123F0EF
:101F300001032361FFF74CFF0120F8BD043C04308E
:101F4000E7E78307E7D12B6923F440732B612B6903
:101F50003B432B6151F8046B0660BFF34F8FFFF7D3
:101F600013FF03689E42E9D02B6923F001032B6124
:101F7000FFF72EFF0020E0E723F44073236123697D
:101F80003B4323610B882B80BFF34F8FFFF7FCFE91
:101F90002D8831F8023BADB2AB42C3D0236923F0A8
:101FA00001032361E4E71846C7E700BF0038024099
:101FB000003C0240084908B50B7828B11BB9FFF76F
:101FC000EDFE01230B7008BD002BFCD0BDE80840DE
:101FD0000870FFF7FDBE00BF2E2D002010B5024493
:101FE000064BD2B2904200D110BD441C00B253F84F
:101FF000200041F8040BE0B2F4E700BF5028004095
:102000000F4B30B51C6F240407D41C6F44F40074CC
:102010001C671C6F44F400441C670A4C236843F49B
:10202000807323600244084BD2B2904200D130BD8D
:10203000441C00B251F8045B43F82050E0B2F4E7CE
:1020400000380240007000405028004007B50122CF
:1020500001A90020FFF7C2FF019803B05DF804FB5F
:1020600013B50446FFF7F2FFA04205D0012201A9F3
:1020700000200194FFF7C4FF02B010BD70470000BC
:10208000034B1A681AB9034AD2F874281A607047C9
:10209000642D00200030024008B5FFF7F1FF024B2D
:1020A0001868C0F3407008BD642D00207047000020
:1020B000FEE700000A4B0B480B4A90420BD30B4B38
:1020C000DA1C121AC11E22F003028B4238BF002212
:1020D0000021FEF7F9BD53F8041B40F8041BECE7A0
:1020E000B8370008602E0020602E0020602E0020EF
:1020F00070B5D0E915439E6800224FF0FF3504EB20
:1021000042135101D3F800090028BEBFD3F80009DB
:1021100040F08040C3F80009D3F8000B0028BEBF90
:10212000D3F8000B40F08040C3F8000B0132631875
:102130009642C3F80859C3F8085BE0D24FF0011388
:10214000C4F81C3870BD0000890141F02001016114
:1021500003699B06FCD41220FFF718BB10B5054C91
:102160002046FEF7E7FF4FF0A0436365024BA365EF
:1021700010BD00BF682D00206036000870B50378E0
:10218000012B054650D12A4B446D98421BD1294B57
:102190005A6B42F080025A635A6D42F080025A65CF
:1021A0005A6D5A6942F080025A615A6922F08002DF
:1021B0005A610E2143205B6900F022FC1E4BE36054
:1021C0001E4BC4F800380023C4F8003EC02323602F
:1021D0006E6D4FF40413A3633369002BFCDA012303
:1021E00033610C20FFF7D2FA3369DB07FCD41220ED
:1021F000FFF7CCFA3369002BFCDA0026A6602846EC
:10220000FFF776FF6B68C4F81068DB68C4F81468E1
:10221000C4F81C684BB90A4BA3614FF0FF336361EC
:10222000A36843F00103A36070BD064BF4E700BF51
:10223000682D0020003802404014004003002002B6
:10224000003C30C0083C30C0F8B5446D0546002164
:102250002046FFF779FFA96D00234FF001128F6828
:10226000C4F834384FF00066C4F81C284FF0FF3033
:1022700004EB431201339F42C2F80069C2F8006BBD
:10228000C2F80809C2F8080BF2D20B686A6DEB6558
:10229000636210231361166916F01006FBD1122039
:1022A000FFF774FAD4F8003823F4FE63C4F800385A
:1022B000A36943F4402343F01003A3610923C4F846
:1022C0001038C4F814380A4BEB604FF0C043C4F820
:1022D000103B084BC4F8003BC4F81069C4F800393F
:1022E000EB6D03F1100243F48013EA65A362F8BDBD
:1022F0003C36000840800010426D90F84E10D2F835
:10230000003823F4FE6343EA0113C2F80038704733
:102310002DE9F84300EB8103456DDA68166806F095
:102320000306731E022B05EB41130C4680460FFA81
:1023300081F94FEA41104FF00001C3F8101B4FF034
:10234000010104F1100398BFB60401FA03F3916987
:102350008EBF334E06F1805606F5004600293AD06E
:10236000578A04F15801490137436F50D5F81C18BA
:102370000B43C5F81C382B180021C3F810195369FA
:102380000127611EA7409BB3138A928B9B08012AE9
:1023900088BF5343D8F85C20981842EA034301F100
:1023A000400205EB8202C8F85C00214653602846D3
:1023B000FFF7CAFE08EB8900C3681B8A43EA84530F
:1023C000483464011E432E51D5F81C381F43C5F80C
:1023D0001C78BDE8F88305EB4917D7F8001B21F4FA
:1023E0000041C7F8001BD5F81C1821EA0303C0E719
:1023F00004F13F0305EB83030A4A5A60284621464D
:10240000FFF7A2FE05EB4910D0F8003923F4004392
:10241000C0F80039D5F81C3823EA0707D7E700BF12
:102420000080001000040002826D1268C265FFF790
:102430005FBE00005831436D49015B5813F4004002
:1024400004D013F4001F0CBF0220012070470000CD
:102450004831436D49015B5813F4004004D013F434
:10246000001F0CBF022001207047000000EB81011B
:10247000CB68196A0B6813604B68536070470000A3
:1024800000EB810330B5DD68AA691368D36019B920
:10249000402B84BF402313606B8A1468426D1C4438
:1024A000013CB4FBF3F46343033323F0030302EB77
:1024B000411043EAC44343F0C043C0F8103B2B68CB
:1024C00003F00303012B09B20ED1D2F8083802EB56
:1024D000411013F4807FD0F8003B14BF43F08053C9
:1024E00043F00053C0F8003B02EB4112D2F8003B2E
:1024F00043F00443C2F8003B30BD00002DE9F04139
:10250000244D6E6D06EB40130446D3F8087BC3F8E8
:10251000087B38070AD5D6F81438190706D505EB15
:1025200084032146DB6828465B689847FA071FD575
:10253000D6F81438DB071BD505EB8403D968CCB972
:102540008B69488A5A68B2FBF0F600FB16228AB9FA
:102550001868DA6890420DD2121AC3E900243023B9
:1025600083F311880B482146FFF78AFF84F3118813
:10257000BDE8F081012303FA04F26B8923EA020328
:102580006B81CB68002BF3D021460248BDE8F041B7
:10259000184700BF682D002000EB810370B5DD688F
:1025A000436D6C692668E6604A0156BB1A444FF4D5
:1025B0000020C2F810092A6802F00302012A0AB2B8
:1025C0000ED1D3F8080803EB421410F4807FD4F83E
:1025D000000914BF40F0805040F00050C4F80009DA
:1025E00003EB4212D2F8000940F00440C2F800099F
:1025F000D3F83408012202FA01F10143C3F8341878
:1026000070BD19B9402E84BF4020206020682E8AFA
:102610008419013CB4FBF6F440EAC44040F0005099
:102620001A44C6E72DE9F8433B4D6E6D06EB4013A7
:102630000446D3F80889C3F8088918F0010F4FEA57
:1026400040171AD0D6F81038DB0716D505EB8003F3
:10265000D9684B691868DA68904230D2121A4FF084
:1026600000091A60C3F80490302383F311882146CF
:102670002846FFF791FF89F3118818F0800F1CD0CE
:10268000D6F834380126A640334216D005EB840331
:102690006D6DD3F80CC0DCF814200134E4B2D2F82C
:1026A00000E005EB04342F445168714515D3D5F88B
:1026B000343823EA0606C5F83468BDE8F8830123F8
:1026C00003FA04F22B8923EA02032B818B68002B87
:1026D000D3D0214628469847CFE7BCF81000AEEB90
:1026E0000103834228BF0346D7F8180980B2B3EB31
:1026F000800FE2D89068A0F1040959F8048FC4F85B
:102700000080A0EB09089844B8F1040FF5D81844EC
:102710000B4490605360C7E7682D00202DE9F74F08
:10272000A24C656D6E69AB691E4016F480586E61EF
:1027300007D02046FEF766FD03B0BDE8F04F00F07D
:1027400047BC002E12DAD5F8003E98489B071EBF02
:10275000D5F8003E23F00303C5F8003ED5F8043851
:1027600023F00103C5F80438FEF776FD370505D5DB
:102770008E48FFF7BDFC8D48FEF75CFDB0040CD51C
:10278000D5F8083813F0060FEB6823F470530CBF2C
:1027900043F4105343F4A053EB6031071BD5636837
:1027A000DB681BB9AB6923F00803AB612378052B09
:1027B0000CD1D5F8003E7D489A071EBFD5F8003EE3
:1027C00023F00303C5F8003EFEF746FD6368DB68AF
:1027D0000BB176489847F30274D4B70227D5D4F8E2
:1027E0005490DFF8C8B100274FF0010A09EB4712F7
:1027F000D2F8003B03F44023B3F5802F11D1D2F877
:10280000003B002B0DDA62890AFA07F322EA030380
:10281000638104EB8703DB68DB6813B139465846F4
:102820009847A36D01379B68FFB29F42DED9F0063F
:1028300017D5676D3A6AC2F30A1002F00F0302F46B
:10284000F012B2F5802F00F08580B2F5402F08D14C
:1028500004EB83030022DB681B6A07F58057904274
:102860006AD13003D5F8184813D5E10302D500200A
:10287000FFF744FEA20302D50120FFF73FFE6303EA
:1028800002D50220FFF73AFE270302D50320FFF707
:1028900035FE75037FF550AFE00702D50020FFF746
:1028A000C1FEA10702D50120FFF7BCFE620702D5D9
:1028B0000220FFF7B7FE23077FF53EAF0320FFF7A7
:1028C000B1FE39E7636DDFF8E4A0019300274FF014
:1028D0000109A36D9B685FFA87FB9B453FF67DAFBF
:1028E000019B03EB4B13D3F8001901F44021B1F520
:1028F000802F1FD1D3F8001900291BDAD3F8001953
:1029000041F09041C3F80019D3F800190029FBDB0E
:102910005946606DFFF718FC218909FA0BF321EA8B
:102920000303238104EB8B03DB689B6813B15946D7
:10293000504698470137CCE7910708BFD7F8008089
:10294000072A98BF03F8018B02F1010298BF4FEAF2
:10295000182884E7023304EB830207F58057526896
:10296000D2F818C0DCF80820DCE9001CA1EB0C0C44
:10297000002188420AD104EB830463689B699A684A
:1029800002449A605A6802445A606AE711F0030FE1
:1029900008BFD7F800808C4588BF02F8018B01F191
:1029A000010188BF4FEA1828E3E700BF682D002027
:1029B000436D03EB4111D1F8003B43F40013C1F820
:1029C000003B7047436D03EB4111D1F8003943F4EC
:1029D0000013C1F800397047436D03EB4111D1F882
:1029E000003B23F40013C1F8003B7047436D03EB39
:1029F0004111D1F8003923F40013C1F800397047B0
:102A000000F1604303F561430901C9B283F8001383
:102A1000012200F01F039A4043099B0003F1604329
:102A200003F56143C3F880211A60704730B5039CF9
:102A30000172043304FB0325C0E90653049B0363BE
:102A40000021059BC160C0E90000C0E90422C0E983
:102A50000842C0E90A11436330BD0000416A002208
:102A6000C0E90411C0E90A22C2606FF00101FEF75B
:102A7000FDBE0000D0E90432934201D1C2680AB918
:102A8000181D70470020704703691960C268013241
:102A9000C260C269134482690361934224BF436ADE
:102AA00003610021FEF7D6BE38B504460D46E36843
:102AB0003BB16269131D1268A3621344E3620020F4
:102AC00007E0237A33B929462046FEF7B3FE0028F3
:102AD000EDDA38BD6FF00100FBE70000C368C269A2
:102AE000013BC3604369134482694361934224BF3D
:102AF000436A436100238362036B03B11847704745
:102B000070B53023044683F31188866A3EB9FFF717
:102B1000CBFF054618B186F31188284670BDA36A1D
:102B2000E26A13F8015BA362934202D32046FFF7E7
:102B3000D5FF002383F31188EFE700002DE9F84F5C
:102B400004460E46174698464FF0300989F311881F
:102B50000025AA46D4F828B0BBF1000F09D14146A0
:102B60002046FFF7A1FF20B18BF311882846BDE86E
:102B7000F88FD4E90A12A7EB050B521A934528BF28
:102B80009346BBF1400F1BD9334601F1400251F887
:102B9000040B43F8040B9142F9D1A36A4033403649
:102BA000A3624035D4E90A239A4202D32046FFF7B4
:102BB00095FF8AF31188BD42D8D289F31188C9E7FD
:102BC00030465A46FEF75AF8A36A5B445E44A36255
:102BD0005D44E7E710B5029C0172043303FB042156
:102BE000C0E906130023C0E90A33039B0363049B77
:102BF000C460C0E90000C0E90422C0E908424363A0
:102C000010BD0000026AC260426AC0E904220022CC
:102C1000C0E90A226FF00101FEF728BED0E90423C3
:102C20009A4201D1C26822B9184650F8043B0B60A1
:102C3000704700231846FAE7C368C2690133C360CE
:102C40004369134482694361934224BF436A4361E9
:102C50000021FEF7FFBD000038B504460D46E368CD
:102C60003BB123691A1DA262E2691344E3620020AA
:102C700007E0237A33B929462046FEF7DBFD00281A
:102C8000EDDA38BD6FF00100FBE700000369196061
:102C9000C268013AC260C269134482690361934207
:102CA00024BF436A036100238362036B03B11847A7
:102CB0007047000070B530230D460446114683F37B
:102CC0001188866A2EB9FFF7C7FF10B186F3118805
:102CD00070BDA36A1D70A36AE26A01339342A362C6
:102CE00004D3E16920460439FFF7D0FF002080F3C8
:102CF0001188EDE72DE9F84F04460D4690469946B8
:102D00004FF0300A8AF311880026B346A76A4FB9FC
:102D100049462046FFF7A0FF20B187F311883046CF
:102D2000BDE8F88FD4E90A073A1AA8EB06079742DC
:102D300028BF1746402F1BD905F1400355F8042B37
:102D400040F8042B9D42F9D1A36A4033A362403678
:102D5000D4E90A239A4204D3E16920460439FFF7F3
:102D600095FF8BF311884645D9D28AF31188CDE7B8
:102D700029463A46FDF782FFA36A3B443D44A362DD
:102D80003E44E5E7D0E904239A4217D1C3689BB1DA
:102D9000836A8BB1043B9B1A0ED01360C368013B5E
:102DA000C360C3691A44836902619A4224BF436ABB
:102DB0000361002383620123184670470023FBE769
:102DC00000F030B94FF08043586A70474FF08043AD
:102DD000002258631A610222DA6070474FF0804384
:102DE0000022DA60704700004FF08043586370475C
:102DF000FEE7000070B51B4B01630025044686B05A
:102E0000586085620E4600F0BFF804F11003C4E973
:102E100004334FF0FF33C4E90635C4E90044A5602C
:102E2000E562FFF7CFFF2B460246C4E9082304F111
:102E300034010D4A256580232046FEF7B1FC0123AD
:102E4000E0600A4A0375009272680192B268CDE9A7
:102E50000223074B6846CDE90435FEF7C9FC06B0EE
:102E600070BD00BF002600206C36000871360008D7
:102E7000F12D0008024AD36A1843D062704700BFA0
:102E8000982300204B6843608B688360CB68C360E5
:102E90000B6943614B6903628B6943620B68036092
:102EA0007047000008B5264B26481A6940F2FF110A
:102EB0000A431A611A6922F4FF7222F001021A61B0
:102EC0001A691A6B0A431A631A6D0A431A651E4A75
:102ED0001B6D1146FFF7D6FF02F11C0100F5806063
:102EE000FFF7D0FF02F1380100F58060FFF7CAFF5D
:102EF00002F1540100F58060FFF7C4FF02F1700198
:102F000000F58060FFF7BEFF02F18C0100F58060E4
:102F1000FFF7B8FF02F1A80100F58060FFF7B2FFEC
:102F200002F1C40100F58060FFF7ACFF02F1E0019F
:102F300000F58060FFF7A6FFBDE8084000F0EEB89E
:102F400000380240000002407836000808B500F062
:102F500059FAFEF703FCFFF793F8BDE80840FEF7C7
:102F600071BE000070470000EFF3098305494A6B0A
:102F700022F001024A63683383F30988002383F354
:102F80001188704700EF00E0302080F3118862B6AE
:102F90000C4B0D4AD96821F4E0610904090C0A437D
:102FA000DA60D3F8FC20094942F08072C3F8FC20B3
:102FB0000A6842F001020A602022DA7783F82200D0
:102FC000704700BF00ED00E00003FA05001000E0CC
:102FD00010B5302383F311880E4B5B6813F4006344
:102FE00014D0F1EE103AEFF30984683C4FF080738F
:102FF000E361094BDB6B236684F30988FEF78EFBE4
:1030000010B1064BA36110BD054BFBE783F311889C
:10301000F9E700BF00ED00E000EF00E02F0300083B
:10302000320300080F4B1A6C42F001021A641A6E48
:1030300042F001021A660C4A1B6E936843F00103CA
:1030400093604FF0804353229A624FF0FF32DA626E
:1030500000229A615A63DA605A6001225A611A604A
:10306000704700BF00380240002004E04FF080426B
:1030700008B51169D3680B40D9B2C9439B071161E8
:1030800007D5302383F31188FEF77EFB002383F3FB
:10309000118808BD1F4B1A696FEAC2526FEAD252FB
:1030A0001A611A69C2F308021A614FF0FF301A69F7
:1030B0005A69586100215A6959615A691A6A62F05D
:1030C00080521A621A6A02F080521A621A6A5A6AA6
:1030D00058625A6A59625A6A1A6C42F080521A64EB
:1030E0001A6E42F080521A661A6E0B4A106840F44B
:1030F00080701060186F00F44070B0F5007F1EBF44
:103100004FF4803018671967536823F400735360D5
:1031100000F054B90038024000700040334B4FF0CB
:1031200080521A64324A4FF4404111601A6842F0EA
:1031300001021A601A689107FCD59A6822F003020E
:103140009A602A4B9A6812F00C02FBD1196801F0C0
:10315000F90119609A601A6842F480321A601A689C
:103160009203FCD55A6F42F001025A671F4B5A6F07
:103170009007FCD51F4A5A601A6842F080721A60A4
:103180001B4A53685904FCD5184B1A689201FCD5A8
:10319000194A9A60194B1A68194B9A42194B21D156
:1031A000194A1168194A91421CD140F205121A605D
:1031B000144A136803F00F03052BFAD10B4B9A68DE
:1031C00042F002029A609A6802F00C02082AFAD1D0
:1031D0005A6C42F480425A645A6E42F480425A66F3
:1031E0005B6E704740F20572E1E700BF00380240B5
:1031F000007000400854400700948838002004E024
:1032000011640020003C024000ED00E041C20F418B
:10321000074A08B5536903F00103536123B1054A16
:1032200013680BB150689847BDE80840FFF7D0BE5F
:10323000003C0140E02D0020074A08B5536903F027
:103240000203536123B1054A93680BB1D0689847D4
:10325000BDE80840FFF7BCBE003C0140E02D002067
:10326000074A08B5536903F00403536123B1054AC3
:1032700013690BB150699847BDE80840FFF7A8BE35
:10328000003C0140E02D0020074A08B5536903F0D7
:103290000803536123B1054A93690BB1D06998477C
:1032A000BDE80840FFF794BE003C0140E02D00203F
:1032B000074A08B5536903F01003536123B1054A67
:1032C000136A0BB1506A9847BDE80840FFF780BE0B
:1032D000003C0140E02D0020164B10B55C6904F461
:1032E00078725A61A30604D5134A936A0BB1D06A67
:1032F0009847600604D5104A136B0BB1506B984782
:10330000210604D50C4A936B0BB1D06B9847E205AC
:1033100004D5094A136C0BB1506C9847A30504D52A
:10332000054A936C0BB1D06C9847BDE81040FFF78D
:103330004FBE00BF003C0140E02D0020194B10B5EE
:103340005C6904F47C425A61620504D5164A136D27
:103350000BB1506D9847230504D5134A936D0BB1FB
:10336000D06D9847E00404D50F4A136E0BB1506E30
:103370009847A10404D50C4A936E0BB1D06E9847C0
:10338000620404D5084A136F0BB1506F98472304A9
:1033900004D5054A936F0BB1D06F9847BDE8104034
:1033A000FFF716BE003C0140E02D002008B5FFF7F6
:1033B0005DFEBDE80840FFF70BBE0000062108B522
:1033C0000846FFF71DFB06210720FFF719FB062122
:1033D0000820FFF715FB06210920FFF711FB062146
:1033E0000A20FFF70DFB06211720FFF709FB062136
:1033F0002820FFF705FBBDE8084007211C20FFF748
:10340000FFBA000008B5FFF745FE00F00BF8FDF726
:103410008FFEFDF767FDFFF7A5FDBDE80840FFF74C
:10342000CFBC00000023054A19460133102BC2E926
:10343000001102F10802F8D1704700BFE02D002012
:10344000034611F8012B03F8012B002AF9D170472C
:1034500053544D3332463F3F3F0053544D33324671
:103460003430780053544D3332463432780053545C
:103470004D333246343436585800000001203300B2
:103480000010410001105A000310590007103100CC
:103490000000000050340008130400005A340008F3
:1034A0001904000064340008210400006E34000890
:1034B00000000000610E00084D0E0008890E000893
:1034C000750E0008810E00086D0E0008590E0008E8
:1034D000450E0008950E00080000000001000000E5
:1034E0000000000063300000E4340008F0230020F6
:1034F000002600204172647550696C6F740025428B
:103500004F415244252D424C002553455249414CD0
:103510002500000002000000000000007D100008EF
:10352000E910000840004000A02A0020B02A002036
:103530000200000000000000030000000000000086
:103540002D1100080000000010000000C02A00201B
:10355000000000000100000000000000682D0020B5
:1035600001010200E11B0008F11A00088D1B000890
:10357000711B0008430000007C350008090243006D
:10358000020100C03209040000010202010005240A
:103590000010010524010001042402020524060094
:1035A00001070582030800FF09040100020A000068
:1035B00000070501024000000705810240000000ED
:1035C00012000000C835000812011001020000407E
:1035D000091241570002010203010000040309041B
:1035E00025424F4152442500537065656479426518
:1035F000654634303541494F003031323334353649
:10360000373839414243444546000000004000003D
:1036100000400000004000000040000000000100E9
:103620000000020000000200000002000000020092
:103630000000020000000200000002000000000084
:103640007112000829150008D51500084000400037
:10365000C82D0020C82D002001000000D82D00201A
:103660008000000040010000030000006D61696EF1
:103670000069646C650000000001812A0000000000
:10368000AAAAAAAA00010024FFFE00000000000070
:1036900000A00A000000000100000000AAAAAAAAD7
:1036A00000000001FFFF000000000000000000001B
:1036B0000000000000000000AAAAAAAA0000000062
:1036C000FFFF0000000000000000000000040000F8
:1036D00000000000AAAAAAAA00040000FFFF000040
:1036E00000000000000000000000000000000000DA
:1036F000AAAAAAAA00000000FFFF00000000000024
:10370000000000000000000000000000AAAAAAAA11
:1037100000000000FFFF00000000000000000000AB
:103720000000000000000000AAAAAAAA00000000F1
:10373000FFFF00000000000000000000000000008B
:10374000000000000A00000000000000030000006C
:103750000000000000000000000000000000000069
:103760000000000000000000000000000000000059
:10377000000000000000000097140000000000009E
:1037800000400F0000000000FF009600000000084D
:10379000009600000000080004000000DC3500086E
:1037A0000000000000000000000000000000000019
:1037B0000000000000000000FFFFFFFFFFFFFFFF11
:1037C000FFFFFFFFFFFFFFFFFFFFFFFFFFFFFFFF09
:1037D000FFFFFFFFFFFFFFFFFFFFFFFFFFFFFFFFF9
:1037E000FFFFFFFFFFFFFFFFFFFFFFFFFFFFFFFFE9
:1037F000FFFFFFFFFFFFFFFFFFFFFFFFFFFFFFFFD9
:10C000000006002089D20008B98A0608158A0608A9
:10C01000818A0608158A06084D8A06088BD2000810
:10C020008BD200088BD200088BD20008DD520808A2
:10C030008BD200088BD200088BD200088BD200086C
:10C040008BD200088BD200088BD200088BD200085C
:10C050008BD200088BD20008755E08089D5E080828
:10C06000C55E0808ED5E0808155F08081510080889
:10C070003D1008086910080895100808C110080844
:10C08000E910080815110808990F08088BD2000854
:10C090008BD200088BD200088BD200083D5F0808C5
:10C0A000896008088D600808A1600808A560080874
:10C0B000A96008088BD20008BD600808A11608080E
:10C0C000491808088BD200088BD200088BD20008D0
:10C0D0008BD200081160080825600808396008083C
:10C0E000A15F08088BD200088BD200088BD2000811
:10C0F0008BD200088BD200088BD2000841110808AF
:10C100008BD200088BD20008CD6008088BD20008C3
:10C110004D600808616008088BD200088BD20008C7
:10C120006D11080895110808C1110808ED110808DB
:10C13000191208088BD200088BD200088BD2000895
:10C140008BD200088BD200088BD20008095A08084D
:10C15000411208086D12080899120808756008084D
:10C160008BD200088BD200088BD200088BD200083B
:10C170008BD200088BD200088BD200088BD200082B
:10C180008BD200088BD200088BD200088BD200081B
:10C190008BD200088BD200088BD200088BD200080B
:10C1A0008BD200088BD200088BD200088BD20008FB
:10C1B0008BD200088BD200088BD200088BD20008EB
:10C1C0008BD200088BD200088BD200088BD20008DB
:10C1D0008BD200088BD200088BD200088BD20008CB
:10C1E00079E50008096D01082DC60208194C0408FC
:10C1F0009D6804087DB90408C1C2040809C6040882
:10C20000652E050865330508254B05083DC605085C
:10C210008183060835090708E58E0708ADB50708CC
:10C220008DCB07084DF9070815FF0708FFFFFFFF33
:10C2300081F0004102E000BF83F0004330B54FEAD7
:10C2400041044FEA430594EA050F08BF90EA020F44
:10C250001FBF54EA000C55EA020C7FEA645C7FEAD7
:10C26000655C00F0E2804FEA5454D4EB5555B8BFFA
:10C270006D420CDD2C4480EA020281EA030382EA6B
:10C28000000083EA010180EA020281EA0303362DFD
:10C2900088BF30BD11F0004F4FEA01314FF4801CD0
:10C2A0004CEA113102D0404261EB410113F0004FE2
:10C2B0004FEA03334CEA133302D0524263EB430399
:10C2C00094EA050F00F0A780A4F10104D5F1200E37
:10C2D0000DDB02FA0EFC22FA05F2801841F1000192
:10C2E00003FA0EF2801843FA05F359410EE0A5F166
:10C2F00020050EF1200E012A03FA0EFC28BF4CF097
:10C30000020C43FA05F3C01851EBE37101F000454C
:10C3100007D54FF0000EDCF1000C7EEB00006EEB59
:10C320000101B1F5801F1BD3B1F5001F0CD34908E3
:10C330005FEA30004FEA3C0C04F101044FEA44523A
:10C3400012F5800F80F09A80BCF1004F08BF5FEAC1
:10C35000500C50F1000041EB045141EA050130BDA1
:10C360005FEA4C0C404141EB0101013C28BFB1F5B3
:10C37000801FE9D291F0000F04BF01460020B1FAFE
:10C3800081F308BF2033A3F10B03B3F120020CDAD1
:10C390000C3208DD02F1140CC2F10C0201FA0CF0AF
:10C3A00021FA02F10CE002F11402D8BFC2F1200C14
:10C3B00001FA02F120FA0CFCDCBF41EA0C019040CA
:10C3C000E41AA2BF01EB0451294330BD6FEA040413
:10C3D0001F3C1CDA0C340EDC04F11404C4F12002FE
:10C3E00020FA04F001FA02F340EA030021FA04F310
:10C3F00045EA030130BDC4F10C04C4F1200220FA67
:10C4000002F001FA04F340EA0300294630BD21FAA4
:10C4100004F0294630BD94F0000F83F4801306BF6A
:10C4200081F480110134013D4EE77FEA645C18BF5E
:10C430007FEA655C29D094EA050F08BF90EA020FF5
:10C4400005D054EA000C04BF1946104630BD91EAED
:10C45000030F1EBF0021002030BD5FEA545C05D1F0
:10C460004000494128BF41F0004130BD14F580042F
:10C470003CBF01F5801130BD01F0004545F0FE41A3
:10C4800041F470014FF0000030BD7FEA645C1ABFD8
:10C49000194610467FEA655C1CBF0B46024650EA0F
:10C4A000013406BF52EA033591EA030F41F400213B
:10C4B00030BD00BF90F0000F04BF0021704730B5C1
:10C4C0004FF4806404F132044FF000054FF0000196
:10C4D00050E700BF90F0000F04BF0021704730B557
:10C4E0004FF4806404F1320410F0004548BF40422C
:10C4F0004FF000013EE700BF42004FEAE2014FEA81
:10C5000031014FEA02701FBF12F07F4393F07F4F5B
:10C5100081F06051704732F07F4208BF704793F05E
:10C520007F4F04BF41F40021704730B54FF4607471
:10C5300001F0004521F000411CE700BF50EA010274
:10C5400008BF704730B54FF000050AE050EA01021D
:10C5500008BF704730B511F0004502D5404261EB8D
:10C5600041014FF4806404F132045FEA915C3FF4CE
:10C57000D8AE4FF003025FEADC0C18BF03325FEA6B
:10C58000DC0C18BF033202EBDC02C2F1200300FA1C
:10C5900003FC20FA02F001FA03FE40EA0E0021FA41
:10C5A00002F11444BDE600BF70B54FF0FF0C4CF42F
:10C5B000E06C1CEA11541DBF1CEA135594EA0C0FE1
:10C5C00095EA0C0F00F0DEF82C4481EA030621EA1C
:10C5D0004C5123EA4C5350EA013518BF52EA033557
:10C5E00041F4801143F4801338D0A0FB02CE4FF009
:10C5F0000005E1FB02E506F00042E0FB03E54FF039
:10C600000006E1FB03569CF0000F18BF4EF0010E30
:10C61000A4F1FF04B6F5007F64F5407404D25FEA2C
:10C620004E0E6D4146EB060642EAC62141EA5551DF
:10C630004FEAC52040EA5E504FEACE2EB4F1FD0C21
:10C6400088BFBCF5E06F1ED8BEF1004F08BF5FEA9F
:10C65000500E50F1000041EB045170BD06F0004651
:10C6600046EA010140EA020081EA0301B4EB5C04FE
:10C67000C2BFD4EB0C0541EA045170BD41F48011F6
:10C680004FF0000E013C00F3AB8014F1360FDEBF1B
:10C69000002001F0004170BDC4F10004203C35DAF7
:10C6A0000C341BDC04F11404C4F1200500FA05F37A
:10C6B00020FA04F001FA05F240EA020001F000421B
:10C6C00021F0004110EBD37021FA04F642EB060191
:10C6D0005EEA430E08BF20EAD37070BDC4F10C04BB
:10C6E000C4F1200500FA04F320FA05F001FA04F27F
:10C6F00040EA020001F0004110EBD37041F100016B
:10C700005EEA430E08BF20EAD37070BDC4F1200575
:10C7100000FA05F24EEA020E20FA04F301FA05F2DD
:10C7200043EA020321FA04F001F0004121FA04F285
:10C7300020EA020000EBD3705EEA430E08BF20EA55
:10C74000D37070BD94F0000F0FD101F0004640008F
:10C7500041EB010111F4801F08BF013CF7D041EA11
:10C76000060195F0000F18BF704703F00046520015
:10C7700043EB030313F4801F08BF013DF7D043EAE6
:10C780000603704794EA0C0F0CEA135518BF95EA9C
:10C790000C0F0CD050EA410618BF52EA4306D1D123
:10C7A00081EA030101F000414FF0000070BD50EA42
:10C7B000410606BF1046194652EA430619D094EACC
:10C7C0000C0F02D150EA013613D195EA0C0F05D1B6
:10C7D00052EA03361CBF104619460AD181EA03010A
:10C7E00001F0004141F0FE4141F470014FF00000C2
:10C7F00070BD41F0FE4141F4780170BD70B54FF05D
:10C80000FF0C4CF4E06C1CEA11541DBF1CEA1355DC
:10C8100094EA0C0F95EA0C0F00F0A7F8A4EB0504BE
:10C8200081EA030E52EA03354FEA013100F08880B5
:10C830004FEA03334FF0805545EA131343EA12637E
:10C840004FEA022245EA111545EA10654FEA002633
:10C850000EF000419D4208BF964244F1FD0404F5EC
:10C86000407402D25B084FEA3202B61A65EB030548
:10C870005B084FEA32024FF480104FF4002CB6EB05
:10C88000020E75EB030E22BFB61A754640EA0C0085
:10C890005B084FEA3202B6EB020E75EB030E22BFC5
:10C8A000B61A754640EA5C005B084FEA3202B6EB06
:10C8B000020E75EB030E22BFB61A754640EA9C00C5
:10C8C0005B084FEA3202B6EB020E75EB030E22BF95
:10C8D000B61A754640EADC0055EA060E18D04FEA53
:10C8E000051545EA16754FEA06164FEAC30343EAF3
:10C8F00052734FEAC2025FEA1C1CC0D111F4801FC0
:10C900000BD141EA00014FF000004FF0004CB6E7B8
:10C9100011F4801F04BF01430020B4F1FD0C88BF57
:10C92000BCF5E06F3FF6AFAEB5EB030C04BFB6EB62
:10C93000020C5FEA500C50F1000041EB045170BD55
:10C940000EF0004E4EEA113114EB5C04C2BFD4EB82
:10C950000C0541EA045170BD41F480114FF0000E06
:10C96000013C90E645EA060E8DE60CEA135594EA82
:10C970000C0F08BF95EA0C0F3FF43BAF94EA0C0F85
:10C980000AD150EA01347FF434AF95EA0C0F7FF4FA
:10C9900025AF104619462CE795EA0C0F06D152EA4E
:10C9A00003353FF4FDAE1046194622E750EA410632
:10C9B00018BF52EA43067FF4C5AE50EA41047FF443
:10C9C0000DAF52EA43057FF4EBAE12E74FF0FF3CA8
:10C9D00006E000BF4FF0010C02E000BF4FF0010C79
:10C9E0004DF804CD4FEA410C7FEA6C5C4FEA430CF2
:10C9F00018BF7FEA6C5C1BD001B050EA410C0CBF41
:10CA000052EA430C91EA030F02BF90EA020F0020A2
:10CA1000704710F1000F91EA030F58BF994208BF09
:10CA200090422CBFD8176FEAE37040F001007047C6
:10CA30004FEA410C7FEA6C5C02D150EA013C07D11D
:10CA40004FEA430C7FEA6C5CD6D152EA033CD3D068
:10CA50005DF8040B704700BF8446104662468C4662
:10CA60001946634600E000BF01B5FFF7B7FF002895
:10CA700048BF10F1000F01BD4DF808EDFFF7F4FFBE
:10CA80000CBF012000205DF808FB00BF4DF808ED49
:10CA9000FFF7EAFF34BF012000205DF808FB00BF6C
:10CAA0004DF808EDFFF7E0FF94BF012000205DF88E
:10CAB00008FB00BF4DF808EDFFF7CEFF94BF012043
:10CAC00000205DF808FB00BF4DF808EDFFF7C4FF3C
:10CAD00034BF012000205DF808FB00BF4FEA410C85
:10CAE0007FEA6C5C02D150EA013C0AD14FEA430C68
:10CAF0007FEA6C5C02D152EA033C02D14FF00000A5
:10CB000070474FF0010070474FEA410212F50012E2
:10CB100015D211D56FF47873B3EB625212D94FEA84
:10CB2000C12343F0004343EA505311F0004F23FA6E
:10CB300002F018BF404270474FF00000704750EAC3
:10CB4000013005D111F0004008BF6FF00040704780
:10CB50004FF00000704700BF4A0011D212F50012DA
:10CB600011D20DD56FF47873B3EB62520ED44FEA45
:10CB7000C12343F0004343EA505323FA02F07047C5
:10CB80004FF00000704750EA013002D14FF0FF3003
:10CB900070474FF0000070474FEA4102B2F1E043A6
:10CBA00024BFB3F5001CDCF1FE5C0DD901F0004C94
:10CBB0004FEAC0024CEA5070B2F1004F40EB8300E4
:10CBC00008BF20F00100704711F0804F21D113F110
:10CBD0003872BCBF01F00040704741F480114FEA49
:10CBE0005252C2F11802C2F1200C10FA0CF320FAD2
:10CBF00002F018BF40F001004FEAC1234FEAD323EF
:10CC000003FA0CFC40EA0C0023FA02F34FEA430358
:10CC1000CCE77FEA625307D150EA01331EBF4FF0E1
:10CC2000FE4040F44000704701F0004040F0FE40FC
:10CC300040F40000704700BF80F0004002E000BFF9
:10CC400081F0004142001FBF5FEA410392EA030FF7
:10CC50007FEA226C7FEA236C6AD04FEA1262D2EB41
:10CC60001363C1BFD218414048404140B8BF5B4246
:10CC7000192B88BF704710F0004F40F4000020F0DF
:10CC80007F4018BF404211F0004F41F4000121F0F5
:10CC90007F4118BF494292EA030F3FD0A2F101023F
:10CCA00041FA03FC10EB0C00C3F1200301FA03F17D
:10CCB00000F0004302D5494260EB4000B0F5000FA0
:10CCC00013D3B0F1807F06D340084FEA310102F15F
:10CCD0000102FE2A51D2B1F1004F40EBC25008BF11
:10CCE00020F0010040EA03007047490040EB0000DB
:10CCF000013A28BFB0F5000FEDD2B0FA80FCACF1DC
:10CD0000080CB2EB0C0200FA0CF0AABF00EBC25008
:10CD100052421843BCBFD0401843704792F0000FF6
:10CD200081F4000106BF80F400000132013BB5E749
:10CD30004FEA41037FEA226C18BF7FEA236C21D0BF
:10CD400092EA030F04D092F0000F08BF0846704724
:10CD500090EA010F1CBF0020704712F07F4F04D1F2
:10CD6000400028BF40F00040704712F100723CBF05
:10CD700000F50000704700F0004343F0FE4040F42F
:10CD8000000070477FEA226216BF08467FEA2363ED
:10CD90000146420206BF5FEA412390EA010F40F4D8
:10CDA000800070474FF0000304E000BF10F0004324
:10CDB00048BF40425FEA000C08BF704743F096430B
:10CDC00001464FF000001CE050EA010208BF704726
:10CDD0004FF000030AE000BF50EA010208BF7047AD
:10CDE00011F0004302D5404261EB41015FEA010CC2
:10CDF00002BF84460146002043F0B64308BFA3F1BA
:10CE00008053A3F50003BCFA8CF2083AA3EBC2539B
:10CE100010DB01FA02FC634400FA02FCC2F12002BA
:10CE2000BCF1004F20FA02F243EB020008BF20F0F1
:10CE30000100704702F1200201FA02FCC2F1200257
:10CE400050EA4C0021FA02F243EB020008BF20EA4C
:10CE5000DC7070477BB972B90029BEBF00204FF06B
:10CE6000004106E008BF00281CBF6FF000414FF0F2
:10CE7000FF3000F007BAADF1080C6DE904CE0029CF
:10CE800009DB002B1ADB00F095F8DDF804E0DDE9A2
:10CE9000022304B07047404261EB4101002B1BDBD1
:10CEA00000F088F8DDF804E0DDE9022304B0404238
:10CEB00061EB4101524263EB43037047524263EB23
:10CEC000430300F077F8DDF804E0DDE9022304B065
:10CED000404261EB41017047524263EB430300F073
:10CEE00069F8DDF804E0DDE9022304B0524263EBA7
:10CEF0004303704753B94AB9002908BF00281CBF33
:10CF00004FF0FF314FF0FF3000F0BCB9ADF1080C2D
:10CF10006DE904CE00F04EF8DDF804E0DDE902230F
:10CF200004B07047430803F05533C01A830803F078
:10CF3000333300F03330184400EB101000F00F30A2
:10CF400000EB002000EB0040000E704707EE900A57
:10CF5000F5EEC07AF1EE10FA01D400F00BB8F1EE64
:10CF6000677A08B517EE900A00F004F8404261EBCA
:10CF7000410108BDD0B5FFF7BFFA0C4B00220646B1
:10CF80000F46FFF711FBFFF7E7FD0446FFF792FAA4
:10CF9000074B0022FFF708FB02460B463046394696
:10CFA000FFF74AF9FFF7D8FD2146D0BD0000F03D5C
:10CFB0000000F0412DE9F047089D04468E46002B05
:10CFC0004DD18A42944669D9B2FA82F252B101FA3D
:10CFD00002F3C2F1200120FA01F10CFA02FC41EA4D
:10CFE000030E94404FEA1C48210CBEFBF8F61FFAD2
:10CFF0008CF708FB16E341EA034306FB07F199426D
:10D000000AD91CEB030306F1FF3080F01F8199421F
:10D0100040F21C81023E63445B1AA4B2B3FBF8F0F9
:10D0200008FB103344EA034400FB07F7A7420AD980
:10D030001CEB040400F1FF3380F00A81A74240F2A8
:10D0400007816444023840EA0640E41B00261DB113
:10D05000D4400023C5E900433146BDE8F0878B4248
:10D0600009D9002D00F0EF800026C5E90001304607
:10D070003146BDE8F087B3FA83F6002E4AD18B42E1
:10D0800002D3824200F2F980841A61EB030301208B
:10D090009E46002DE0D0C5E9004EDDE702B9FFDE77
:10D0A000B2FA82F2002A40F09280A1EB0C014FEA22
:10D0B0001C471FFA8CFE0126200CB1FBF7F307FB7F
:10D0C000131140EA01410EFB03F0884208D91CEB22
:10D0D000010103F1FF3802D2884200F2CB804346BF
:10D0E000091AA4B2B1FBF7F007FB101144EA01449E
:10D0F0000EFB00FEA64508D91CEB040400F1FF312D
:10D1000002D2A64500F2BB800846A4EB0E0440EA1A
:10D1100003409CE7C6F12007B34022FA07FC4CEA23
:10D12000030C20FA07F401FA06F31C43F9404FEA16
:10D130001C4900FA06F3B1FBF9F8200C1FFA8CFE2B
:10D1400009FB181140EA014108FB0EF0884202FA7F
:10D1500006F20BD91CEB010108F1FF3A80F0888040
:10D16000884240F28580A8F102086144091AA4B2FD
:10D17000B1FBF9F009FB101144EA014100FB0EFE7E
:10D180008E4508D91CEB010100F1FF346CD28E45AD
:10D190006AD90238614440EA0840A0FB0294A1EB3E
:10D1A0000E01A142C846A64656D353D05DB1B3EB9B
:10D1B000080261EB0E0101FA07F722FA06F3F140CB
:10D1C0001F43C5E9007100263146BDE8F087C2F172
:10D1D0002003D8400CFA02FC21FA03F391400143EA
:10D1E0004FEA1C471FFA8CFEB3FBF7F007FB103623
:10D1F0000B0C43EA064300FB0EF69E4204FA02F4CF
:10D2000008D91CEB030300F1FF382FD29E422DD921
:10D21000023863449B1B89B2B3FBF7F607FB163356
:10D2200041EA034106FB0EF38B4208D91CEB0101D6
:10D2300006F1FF3816D28B4214D9023E6144C91A56
:10D2400046EA004638E72E46284605E70646E3E666
:10D250001846F8E64B45A9D2B9EB020864EB0C0E70
:10D260000138A3E74646EAE7204694E74046D1E77F
:10D27000D0467BE7023B614432E7304609E764442D
:10D28000023842E7704700BF02E000F000F8FEE716
:10D2900072B6374880F30888364880F309883648E4
:10D2A0003649086040F20000CCF200004EF63471BE
:10D2B000CEF200010860BFF34F8FBFF36F8F40F2D3
:10D2C0000000C0F2F0004EF68851CEF20001086076
:10D2D000BFF34F8FBFF36F8F4FF00000E1EE100AE6
:10D2E0004EF63C71CEF200010860062080F31488EF
:10D2F000BFF36F8F78F050F879F0E8F94FF05530C0
:10D300001F491B4A91423CBF41F8040BFAE71D49F3
:10D31000184A91423CBF41F8040BFAE71A491B4AEC
:10D320001B4B9A423EBF51F8040B42F8040BF8E73E
:10D3300000201849184A91423CBF41F8040BFAE713
:10D3400078F02EF879F016FA144C154DAC4203DA49
:10D3500054F8041B8847F9E701F0FEF8114C124D10
:10D36000AC4203DA54F8041B8847F9E778F016B8A2
:10D37000000600200022002000C0000808ED00E0A8
:10D380000000002000060020F8820A080022002089
:10D390009425002098250020A81B0120E0C100084A
:10D3A0002CC200082CC200082CC200082DE9F04F46
:10D3B0002DED108AC1F80CD0C3689D46BDEC108AD3
:10D3C000BDE8F08F002383F311882846A047002092
:10D3D00076F0FEFEFEE776F065FD00DFFEE700007A
:10D3E00001F0FF01102A2BDB10F0070F08D010F816
:10D3F000013B013A8B422DD010F0070F42B3F6D11A
:10D40000F0B441EA012141EA014122F007047FF032
:10D4100000070023F0E80256083C85EA010586EA89
:10D42000010685FA47F5A3FA87F586FA47F6A5FAC5
:10D4300087F68EB9EED1F0BC01F0FF0102F00702D1
:10D4400032B110F8013B013A83EA010313B1F8D17C
:10D450000020704701387047002D06BF354603385D
:10D46000073815F0010F07D1013015F4807F02BF96
:10D47000013015F4C03F0130F0BC0138704700BFE7
:10D4800010F8012B11F8013B012A28BF9A42F7D06E
:10D49000D01A7047034613F8012B002AFBD1181A43
:10D4A0000138704738B50022002304460D46FFF7C7
:10D4B000EDFA28B920462946BDE8384000F00AB800
:10D4C000204605F1004100F005F8404261EB4101C2
:10D4D00038BD00BFD0B50C4B002206460F46FFF703
:10D4E00063F8FFF739FB0446FEF7E4FF074B002221
:10D4F000FFF75AF802460B4630463946FEF79CFEC7
:10D50000FFF72AFB2146D0BD0000F03D0000F041AE
:10D51000036800221B6818470120704737B5019146
:10D520002021044659F038F9D0B10E4B93F9561327
:10D53000A1B1B3F95813D3F8F03A019AB3F90C50EA
:10D5400001F10A039D4203DD40F28D33994205DC6F
:10D550002046054B202159F025F9002003B030BDAD
:10D560000120FBE7A045002050D5080808B505F0CC
:10D570008DFDBDE80840012104F0C6BE2DE9F04351
:10D580008FB00E46054605F081FD002780462E220D
:10D59000394602A801977BF059FE322301AA394689
:10D5A000404605F05BF8044648B9184A01AB3146DD
:10D5B000284659F0E7FA20460FB0BDE8F083DFF8BF
:10D5C0005890D9F8680703689B6898470028F2D0FC
:10D5D000A9F5405003F0C8FC814630B90C4A3146E9
:10D5E000284659F0CFFA4C46E5E76946404604F034
:10D5F0007DFE0028DFD09DF801305B06DBD5054AB3
:10D600003146284659F0BEFA3C46D4E764D50808AE
:10D610006DD5080884D50808A055002008B5064B2C
:10D6200093F8293D9B0704D5044A59F0ABFA002032
:10D6300008BD0120FCE700BFA045002094D50808E4
:10D6400070B50C4C0546D4F868070368DB680E46D5
:10D65000984710B10124204670BDA4F5405003F056
:10D660009FFC04460028F5D1034A3146284659F06C
:10D6700089FAF0E7A0550020A4D508082DE97043E9
:10D68000274BD3F82C3D1D7B814688465DB9254B41
:10D690001B68986A03685B6B984738B9224A414611
:10D6A000484659F06FFA2846BDE8708345F054FEAD
:10D6B000202146F0BDFD38B145F04EFE1F2146F059
:10D6C000B7FD08B1194AEAE7484659F05DF838B99C
:10D6D000D9F80030414648465B6BBDE870431847B7
:10D6E00041464846FFF71AFF41460646484659F06C
:10D6F000ABFE20210640484659F04EF841464846C8
:10D70000FFF78CFFF5B2054041464846FFF798FF0A
:10D710004146054048465AF065F80540C3E700BF5A
:10D72000A0450020105E0020B8D50808CFD5080815
:10D7300008B5FFF7A3FF054A92F8181D60F34101F1
:10D7400082F8181D024A907108BD00BFA045002054
:10D75000BD5E00202DE9F04106460F4659F052F813
:10D76000044668B30221304659F016F840B305F07C
:10D770008DFC4FF48071804604F0C6FD0546F8B973
:10D780004FF40071404604F0BFFDC8B10E485AF096
:10D7900045FA0E4BD3EDA47AF8EEE77A30EE670A3D
:10D7A000DFED0B7AB0EEC00AB4EEE70AF1EE10FA44
:10D7B00006DD084B3A460221304658F0F3FF2C466E
:10D7C0002046BDE8F08100BF28590020A055002068
:10D7D0000000C842ECD50808F8B504460F4659F0D9
:10D7E0005FFA10210546204658F0D6FF58B1204672
:10D7F000FFF7BCFE064630B9044B3A4610212046DE
:10D8000058F0D0FF35462846F8BD00BF00D60808BE
:10D8100070B505460E4658F039FF044678B18021B0
:10D82000284658F0B9FF50B1094B93F88D3243B1F7
:10D83000084B32468021284658F0B4FF0024204689
:10D8400070BD31462846BDE8704059F0EFBB00BFBF
:10D85000A055002014D608082DE9F04180460E4658
:10D86000FFF78CFE1A4F044610B90024FC710AE041
:10D87000184D05F54053D3F8680703689B6898472F
:10D8800020B90123FB712046BDE8F0810821404604
:10D8900058F082FF0028F4D095F8E433B02202FB60
:10D8A000035305F50055B3F8EE21B5F954339A4208
:10D8B00006DD094B32460821404658F073FFD4E795
:10D8C0003146404659F08EF80028DAD1CDE700BF46
:10D8D000BD5E0020A025002028D6080859F0A4BC71
:10D8E00070B505460E46FFF749FE084B0446D87151
:10D8F00031462846FFF7A4FE31460028284608BFD7
:10D90000002459F02BFE204070BD00BFBD5E0020FA
:10D910002DE9F843414F3B788146002B7BD1404CA9
:10D92000D4F82C5D2D7B01263E701DB13B7028463E
:10D93000BDE8F8835AF014F8054630B9394A387012
:10D94000137843F001031370F1E7DFF8F4803AF045
:10D9500035FE314639F058FF88F804600B2633F065
:10D96000A3FC013E33F03EFC16F0FF06F7D12E4932
:10D97000484659F00BFF05F089FBD0F80C22C4F89B
:10D980003C2D90F89432DA0733D404F0D5FE3AF007
:10D9900015FE3C213AF04EFD04F6245300221A6095
:10D9A000224B1B68D86A036801211B689847D4F88A
:10D9B0002C2D137B1BB90123137388F804303AF024
:10D9C000FDFD94F81D2D94F81C1D3AF00DF938F06A
:10D9D000CBF837F0F5FB00233B705BF09FF8144B5E
:10D9E000C3F85C0794F8193D43F0200384F8193D0F
:10D9F0009DE79B07D4D431460E4802F06DF90E48DE
:10DA00005AF00CF9DFED0D7A20EE270A04F62453C4
:10DA100083ED000AC4E7002589E700BF98250020B0
:10DA2000A0450020DC5E002038D60808105E0020EB
:10DA3000A0550020A0250020285900200AD7233C0B
:10DA4000BD5E00202DE9F043364DD5F82C3D1B7B03
:10DA500087B006460C46002B61D000294BD02146EA
:10DA600030465AF035F80446002853D02E49304647
:10DA700059F08CFE05F00AFB074609F009FF8046C5
:10DA8000384604F0A9F8D8B198F92430022B17D100
:10DA900000264FF00009F1B203AA38460191CDF8F3
:10DAA0000C90CDF81090CDF8149004F073FC01990F
:10DAB00018B103AA404609F0F7FB0136032EEAD15C
:10DAC000D5F82C2D137B1BB100231373174A137148
:10DAD0003AF074FD002139F097FE154B1B68D86AA7
:10DAE000036800211B68984795F8193D6FF34513AB
:10DAF00085F8193D0FE005F580530192D3F86807CA
:10DB00000368DB689847019A0028A8D195F8183D6A
:10DB1000DB06A4D40024204607B0BDE8F08301242E
:10DB2000F9E700BFA045002048D60808BD5E0020E8
:10DB3000105E002008B500F5005090F8183DC3F3C2
:10DB400080028A420BD061F3820380F8183D31B124
:10DB50003AF034FDBDE808400F213AF06BBC08BD37
:10DB600010B500F500520C4692F8293D03F0010172
:10DB7000A14209D064F3000382F8293DDB0704D4F5
:10DB800002F0EEFA024B9C7210BD02F097FBF9E72F
:10DB9000BD5E002000F5005090F8293D61F341037F
:10DBA00080F8293D014B1973704700BFBD5E00200E
:10DBB0000020704700207047002070470020704709
:10DBC00000207047002070470020704700207047F9
:10DBD00000207047002070470020704700207047E9
:10DBE000704700007047000000F50D50243070476A
:10DBF000004870472800090800F5005090F81C0DF7
:10DC000070470000034808601C21117008221A6048
:10DC1000704700BF14D9080837F0F2BE16F03ABEBC
:10DC200039F070BF44F0A2BF43F05AB902F0B8BA5D
:10DC300002F0ECB902F018B933F0D4BA49F0B0B937
:10DC400045F052BA11F0F2BC02F034B802F0E4BC74
:10DC500002F0A6B902F036BC02F0B0BF17F036B938
:10DC600003F0B2B902F0D0BA02F082BB70B51F4B1C
:10DC7000036000F500530446D3F8AC0C1C4AC3F80B
:10DC8000542B08B109F052F81A4B236004F5805365
:10DC900093F84C2F42B9D3F8485F2DB1284615F0C0
:10DCA00043FC284609F03EF804F589500C3058F042
:10DCB00087F804F58750103047F08EFB04F6C44512
:10DCC00004F66446B54204D0183D284615F05EF8C7
:10DCD000F8E7094BC4F8983804F694103CF044FC7B
:10DCE00004F510603CF040FC204670BD50DB080895
:10DCF0003CAF0908FC8E09085C63090838B5474B3E
:10DD0000044640F8043B47F0FDFC04F1100008F025
:10DD1000F7FB04F1680037F001FC04F5907010F097
:10DD200021F904F5866007F0EBF904F2545009F08C
:10DD300031F804F6980016F057FC04F5446047F0FB
:10DD400069FC04F5516037F007F904F5815018308B
:10DD500039F0AAFC04F58750103047F025FB04F594
:10DD600089500C3058F018F804F58A50083037F014
:10DD700091FF04F591501C3048F072FE04F5805379
:10DD800004F593520025104683F86052244B10305E
:10DD90001A6033F0ADF8294604F5965003F00EFCF6
:10DDA00004F5CA50183050F079FE04F5EE501C30DE
:10DDB00055F06EF804F5F750143057F047F904F5B4
:10DDC000FA50183057F07CFD04F5FD50103007F084
:10DDD00095F804F50450103051F0EEFA04F50650B1
:10DDE00010304DF07BFE04F50A50203046F06AFFFB
:10DDF00004F5005304F50C5083F80853094D203006
:10DE000058F0A2FB2B6813B107485AF059FE204680
:10DE1000064936F095F92C60204638BDFC8E09087D
:10DE200080690020905F00209CD60808348E090885
:10DE300010B502F09BFF45F08FFA0368BDE8104073
:10DE40005B681847FFF7F4BF38B500F53555044651
:10DE5000284608F02FFA09F01BFD90F92130D3B1C4
:10DE600090F84033BBB12846002107F0E9FFDFED11
:10DE70000A7A04F2AC7393ED287A20EE270ADFEDDC
:10DE8000077AA7EE270A04F2545083ED280ABDE86A
:10DE9000384009F00DBC38BDCDCCCC3D6666663F40
:10DEA000FFF7D2BF10B50121044603F0B1F810B15D
:10DEB000204601F0D9F84FF48051204603F0A8F82D
:10DEC00020B12046BDE8104001F090B810BD000020
:10DED000FFF7E8BF38B50221044603F099F838B1DE
:10DEE0000121204603F094F810B9204601F0BCF857
:10DEF0000221204603F08CF858B3204601F0C2F806
:10DF00004021204603F084F868B104F581551835A6
:10DF1000284638F04FFF04F5805393F9F03013B1E1
:10DF2000284639F091F84FF48061204603F070F8EC
:10DF300020B104F58150183038F0DEFF80212046F2
:10DF400003F066F860B118F003F8BDE8384016F049
:10DF500097B90121204603F05BF80028CDD1CFE727
:10DF60004FF48021204603F053F80028EBD14FF402
:10DF70000021204603F04CF80028E4D138BD000011
:10DF8000FFF7A8BF10B50121044603F041F810B116
:10DF9000204601F077F88021204603F039F828B1B7
:10DFA00017F0D6FFBDE8104016F046B910BD0000CE
:10DFB000FFF7E8BF38B54FF6FF71044603F028F8C5
:10DFC00004F5005528B1D5F8182D0721204601F099
:10DFD00061F846F0A1FD46F0C5FB95F8183D074AEB
:10DFE00083F01003C3F30013537137F0BDFD37F016
:10DFF0000FFABDE83840024850F05CB8BD5E002022
:10E00000145C0020FFF7D6BFF0B52DED028B00F5B4
:10E0100096549FB005460121204604F0BDFF05F54A
:10E020004A513031204604F021FE05F54B510831AC
:10E03000204603F0E5FE05F5B05104F54B701031B4
:10E040001BF0FEFB05F5405405F54B50D4F8B0220B
:10E05000D4F8B43284EDB50A1CA91C301C921D936F
:10E060003BF0A2FF05F54A5105F54C503831203000
:10E07000B0EE608AF0EE408A3BF02EFE05F54B5183
:10E0800005F54D501431C4EDAF8A84EDB08A84EDAE
:10E09000B10A14303BF020FE84EDB60A3AF08EFA55
:10E0A00005465AF043FD2B4B074618680E46FEF70F
:10E0B00023FACDE91801D4F8D002FEF71DFACDE914
:10E0C0001601D4F8CC02FEF717FACDE91401D4F802
:10E0D000C802FEF711FACDE91201D4F8D802FEF712
:10E0E0000BFACDE91001D4F8D402FEF705FACDE918
:10E0F0000E01D4F8C402FEF7FFF9CDE90C01D4F803
:10E10000B802FEF7F9F9CDE90A01D4F8C002FEF72A
:10E11000F3F9CDE90801D4F8B402FEF7EDF9CDE941
:10E120000601D4F8BC02FEF7E7F9CDE90401D4F802
:10E13000B002FEF7E1F9CDE90076CDE90201064B28
:10E14000064A0749284639F0ABFF1FB0BDEC028BE9
:10E15000F0BD00BF783A0020B0D60808BED6080847
:10E16000EBD60808FFF750BF10B5044602F088FE52
:10E170001021204602F04CFF28B117F0E9FEBDE85F
:10E18000104016F04BB910BDFFF7EEBF00F5805000
:10E1900000F5A56300F23450D3ED005AD0ED006ACB
:10E1A000D1ED017A91ED006A26EEE77A67EEA57A65
:10E1B000A6EE257AE6EE267A81ED007AC1ED017AA7
:10E1C0007047000000F5805000F5A56300F2345060
:10E1D000D3ED005AD0ED006AD1ED017A91ED006ADD
:10E1E00027EEA67A67EEA57AA6EE257AE6EE667A9F
:10E1F00081ED007AC1ED017A704700002DE9F04110
:10E200002DED028B054686B0FFF778FDB94B2B60EC
:10E2100005F50E50183005F5005401F01FFC05F50A
:10E220000D531C3305F52C56C4F8F83A062384F830
:10E23000FC3A304658F036FA04AFAF4BC4F8003B16
:10E240003946301D4FF0010805F52D568DF8108028
:10E25000143636F04DFDA94BC4F8543B06F10800C6
:10E2600059F0C4FD0723C4F8B03C0023A4F8B43C23
:10E2700084F8A88C4FF4D27008F052FDC4F8AC0CAE
:10E2800005F53250383059F0B1FD05F533503C30CA
:10E2900059F0ACFD9A4B1A6802B91E6099499FED7E
:10E2A0009A8A304635F04CFF984BC4F8543B05F53C
:10E2B00034500123A4F81C3D1E3059F043FC944B0C
:10E2C0000593944B0495009397E80C004FF400716C
:10E2D00005F5355007F0E2FC05F54A5003A9F7EEC5
:10E2E000008A1430CDED038A3BF0B2FA05F54A50AE
:10E2F000203008F0EBF905F540549FED872A84EDB6
:10E30000AC8A05F59653B0EE083A05F54E50C4F8C0
:10E31000A033F0EE432AF0EE420AB0EE430AF0EEEC
:10E32000481AB0EE481A84EDAD8A84EDAE8A84EDC9
:10E33000AF8A84EDB08A84EDB18A84EDB28A84ED2F
:10E34000B38A84EDB48A84EDC08A84EDC18A84EDF9
:10E35000C28A84EDC38A84EDC48A84EDC58A84EDC3
:10E36000C68A84EDC78A84EDE28A84EDE38A84ED6F
:10E37000E48A84EDE58A84EDE68A84EDE78A243038
:10E3800050F03EF8B0EE083A05F55150F0EE432A51
:10E39000B0EE682AF0EE481AB0EE481AF7EE080A16
:10E3A000B1EE0C0A183050F0D9F9B0EE083A05F584
:10E3B0005350F0EE432AB0EE430A9FED572ADFEDAB
:10E3C000570AF0EE481AB0EE481A103050F0C6F96D
:10E3D000B0EE083A05F55550F0EE432A9FED502A6D
:10E3E000DFED500AF0EE481AB0EE481AB0EE680AB7
:10E3F000083050F005F8B0EE083A05F55750F0EE49
:10E40000432A9FED490AB0EE482AF0EE481AB0EED2
:10E41000481AF0EE480A3C3050F0A0F9F0EE083A05
:10E4200005F559509FED410AB0EE485AF0EE684AA2
:10E43000B0EE484AB0EE633AF0EE632AB0EE002A3E
:10E44000F0EE481AB0EE481AF6EE000A34304FF0FB
:10E45000E1FD374B3748186005F55D522432002343
:10E4600014279EB207FB06010133097C0029F8D16D
:10E47000314B1E80314B196811B131485AF020FBE5
:10E4800005F55D502C30C4F868071A6002F07EF87C
:10E490002C4BC4F86C3705F55E501C3002F076F852
:10E4A000294BC4F89C3705F55F500C3002F06EF82C
:10E4B000264BC4F8CC3705F55F503C3002F066F8C7
:10E4C000234BC4F8FC3705F5605004F62C0383EDAC
:10E4D000008A83ED018A83ED028A3C3002F056F80F
:10E4E0001C4BC4F83C38284606B0BDEC028BBDE896
:10E4F000F08100BF50DB080864D608083CAF09086B
:10E50000B06200203CAB09080000000010DC0808E5
:10E5100069DC000844DB0808CDCC4C3ECDCCCC3EB9
:10E52000CDCCCC3DCDCC4C3D3333333F9A99993F44
:10E53000585F0020B0110908565F0020145F0020CA
:10E54000F0D60808F81A0908381A0908AC1B090897
:10E55000981A0908481B090838B5054B1C68236838
:10E560000A461D68034B01462046A847002038BDD7
:10E57000105E0020A025002010B559F0FDFE064CCD
:10E58000064B18602046FFF739FE2046044A05492D
:10E59000BDE8104078F054B9A0250020105E00209E
:10E5A000CCC200206DDC000810B504460180024991
:10E5B00035F0C6FD204610BDD8DB080810B5002395
:10E5C0004FF07C52274C03654FF07E51C0F88030ED
:10E5D000C0F89030C0F8A030C0F8C0304365C0F833
:10E5E0008430C0F89430C0F8A430C0F8C4308366DA
:10E5F0008367C0F89830C0F8A830C0F8B830C36658
:10E60000C367C0F89C30C0F8AC30C0F8BC304FF0E5
:10E610003F430267C0F8B0204267C0F8B420C0F89A
:10E620008820C0F8C820C0F88C2001664466846544
:10E63000C165C0F8CC304FF47A71212046F01AF849
:10E640004FF47A71222046F015F84FF47A712320A6
:10E6500046F010F8BDE810404FF47A71242046F0DF
:10E6600009B800BF000080BFF8B52DED068B037B15
:10E67000044643B90023C0F8D430C0F8D830C0F8FD
:10E68000E030C0F8DC30D4ED371A94ED381AD4ED10
:10E69000360A94ED350A8548DFED858A00F03AFCAC
:10E6A0005820B7EE001AFFEE000A94ED350A18F074
:10E6B000D5FF592084ED350AB7EE001AFFEE000AA7
:10E6C00094ED360A18F0CAFF5A2084ED360AB7EEE8
:10E6D000001AFFEE000A94ED380A18F0BFFF5B2025
:10E6E00084ED380AB7EE001AFFEE000A94ED370AFF
:10E6F00018F0B4FF84ED370A5AF008FA07EE900AD2
:10E700009FED6C7AF8EE677A04F1100567EE877A70
:10E710002126C4ED027A2F46F7EE009A94ED35AA31
:10E72000D5ED100AB0EE680A6AEE200A78F034FAE5
:10E7300094ED368AD5ED140AB0EE409A68EE200AC0
:10E74000B0EE680A78F028FAD4ED385AD5ED186A98
:10E7500094ED376A95ED1C7A65EEA66A79EE007A3B
:10E76000F0EEE66A26EE077A77EEA67AB0EEC77A82
:10E7700077EE877AB5EEC09AE5EC017A95ED235AEB
:10E78000C5ED079A28EE058A95ED1F5AAAEE058A6F
:10E7900095ED275AA5EE858AD5ED2B5AA6EE258A4A
:10E7A000F1EE10FACCBF01230023B5EEC00A85EDCF
:10E7B000038AF1EE10FA84F8D030C8BF94F8D03054
:10E7C000F5EEC06AC4BF013384F8D030F1EE10FA20
:10E7D000C8BF94F8D030B5EEC07AC4BF013384F816
:10E7E000D030F1EE10FAC2BF94F8D030013384F883
:10E7F000D03094F9D030002BC1BF07EE103AB8EEFC
:10E80000C77AC8EE076AC5ED036A95ED038AB0EED4
:10E81000C87A77EE877AF4EEE97AF1EE10FAC4BF9F
:10E8200079EEC77A45ED017A94F9E83015ED019A51
:10E8300083B1DFED217AB4EEE79AF1EE10FA09D850
:10E84000DFED1E7AB4EEE77AF1EE10FAA4BF4FF0D6
:10E850008043EB6194ED390AD5ED077A20EE270A63
:10E86000D4ED027A20EE270ADFED157A30EE000AA9
:10E8700020EE270A78F00AF9A9EE008A30B20136B4
:10E880009FED100A85ED0B8A28EE000AB6B245F01E
:10E89000CDFE252E7FF442AFBDEC068B04F12002A5
:10E8A00039460248BDE8F84000F066BBA0250020CC
:10E8B00000000000BD3786359A99193FCDCCCC3E7B
:10E8C000DB0F494000007A440022C0F8D420C0F891
:10E8D000D820C0F8E020C0F8DC20FFF7C5BE00005B
:10E8E00000207047002070470120704790F82C30BE
:10E8F0008B4286BF0C3150F8210000207047000089
:10E9000090F82C308B4286BF0C3150F8210000204B
:10E9100070470000FA207047D0E9083242F4E05214
:10E920004262826A43F4F84342F4E0528262036234
:10E9300070470000014802F085BB00BFA025002001
:10E9400013B54FF45870019108F0E4F9044620B172
:10E95000019943F0E1F9024B2360204602B010BD5B
:10E9600058DC08087047000070470000002070471E
:10E97000704700000020704770470000704700009B
:10E980000320704708207047064BD3F82C3D3BB15D
:10E990001B7B002B0CBF5020D02040F001007047A3
:10E9A0005020FAE7A04500207047000070470000A3
:10E9B00010B52DED028B174BD3F82C4D3CB3D4ED95
:10E9C000360A94ED380AF0EEE00AB0EEC00A78F0AC
:10E9D000E3F8D4ED370AB0EE408A94ED350AF0EE54
:10E9E000E00AB0EEC00A78F0D7F8F0EE400AB0EED8
:10E9F000480A78F0D1F8DFED087A20EE270ABDEE5C
:10EA0000C00A10EE103A18B2BDEC028B10BD2046C1
:10EA1000FAE700BFA04500200000C8423EF0E0BA7F
:10EA200010B504463FF0E8FC054802F00BFB054A30
:10EA3000034606212046BDE810403FF0C5BC00BF9C
:10EA4000A025002044DC08083EF090BD08B508462B
:10EA500007F026FF00280CBF0420002008BD00009E
:10EA6000162A01D03EF0F4BA03220A700120704742
:10EA700042F008BC08B53EF091FC40F41C6040F048
:10EA80000D0008BD10B5044608F04CF9204610BD35
:10EA900008B5094B93F8182DD2060BD403F5805313
:10EAA000D3F868070368DB6A984700280CBF022088
:10EAB000042008BD0120FCE7A0450020044B187885
:10EAC00020B9044B93F8190DC0F38010704700BFB4
:10EAD000685E0020A04500201FB50023019302932B
:10EAE000039304F0D3FA01A904F09CF828B101A81B
:10EAF0001BF028FA05B05DF804FB10F0D5FD90F886
:10EB0000C432B02202FB030090ED2F0AF2E70000AE
:10EB10000C4B93F88D228AB9A3F5805393F8292DD5
:10EB200051070BD193F8182DD20609D493F8193D4B
:10EB300013F0020F14BF0420012070470520704716
:10EB400003207047A05500202DE9F04F354F97F86E
:10EB50001C3D012B8DB0044652D9334EDFF8E8A09E
:10EB6000082516F9018BB7F9703308F1FF3B43FA1A
:10EB70000BF3D90740D5207C3CF05AFD8146207C20
:10EB80003DF020FD00F12103994505D2207C0DB018
:10EB9000BDE8F04F3EF07EB9BBF1070F2CD8DFE89F
:10EBA0000BF03E04323436383A3C204B1869596930
:10EBB0005A6AD3F804B0D3F818E0D3F80CC0D3EDF8
:10EBC000007A1B6ACDF82520CDF829306222212356
:10EBD000CDE9003207900891207CCDED037A19230E
:10EBE00003AAC221CDF810B0CDF814E0CDF818C0BA
:10EBF0008DF824803CF086FD013D15F0FF05B0D175
:10EC00000DB0BDE8F08F0A4BD0E70A4BCEE70A4BB8
:10EC1000CCE70A4BCAE75346C8E7094BC6E7094B9E
:10EC2000C4E700BFA04500201CDD0808B059002043
:10EC3000285A0020A05A0020285B0020545B0020A6
:10EC4000A85C002084590020CC5B0020084BD3F83E
:10EC50009C23920701D43EF0EDB903F5805393ED68
:10EC6000A90ADFED047AB8EEC00A20EE270A704741
:10EC7000A04500200AD7233C10B594B0044603A851
:10EC800007F024FD1A4BD3F86807036803A95B6BF0
:10EC9000984750B3247C59F041FF059BDDED047A81
:10ECA0000893069B09930023F8EEE77A9FED117A0B
:10ECB0000B930C930D930E930F9310931193129348
:10ECC0004FF6F853ADF84C300023962267EE877A62
:10ECD0008DF84E303323CDE90032079007AA572133
:10ECE0002046CDED0A7A3CF00DFD14B010BD00BFFA
:10ECF000A05500200AD7233CF0B5254D0E46074607
:10ED00000FCD95B003AC0FC42B682360731EDBB22C
:10ED1000042B29D814AA02EB830353F8445C2B6814
:10ED200028461B6A98472B6804469B6A28469847E2
:10ED3000002305223D7C089009938DF828208DF84A
:10ED400029608DF82A3094B9232221460DF12B0039
:10ED50007AF07CFA86222E23CDE9003240F2B311FC
:10ED600008AA28463CF0CEFC052015B0F0BD204690
:10ED70000DF12B0304F1200250F8041B43F8041B8F
:10ED80009042F9D102881A8082789A70E2E700BF37
:10ED900060D40808014802F053B900BFA025002044
:10EDA000014B93F81C0D7047A0450020024B93F8CF
:10EDB000190DC0F340007047A045002030B52DED7F
:10EDC000028B154B91ED018A0546D3F8680703685D
:10EDD00085B0DB690C46984728B9BDEEC88A18EEA5
:10EDE000103ADB0712D5D4E9040118F0F1FD68B13F
:10EDF000684607F06BFC6A462146284642F068F9EF
:10EE000020B10649684607F057FD00B1022005B061
:10EE1000BDEC028B30BD00BFA05500204058002043
:10EE20008B8B162B05D0C02B01D1FFF7C7BF43F04A
:10EE3000A3BB00207047000030B52DED028B8DB0D4
:10EE40000023054603930493059304F01FF903A9D7
:10EE500003F0E8FE58B304F019F900F5607393E885
:10EE6000070006AC84E80700DDED060A9DED070A01
:10EE70002D7CF1EE600AB1EE400A78F029F82046C8
:10EE8000B0EE408A1BF05EF8DFED0B7A089B0B9327
:10EE9000012228EE278A0C23CDE90032A82109AAF5
:10EEA00028468DED098A8DED0A0A3CF02BFC0DB049
:10EEB000BDEC028B30BD00BFE02E6542242938B581
:10EEC000054605D040290DD0BDE8384042F0A0BC31
:10EED0000C213DF0F1FF044610B12846FFF7ACFFCE
:10EEE000204638BD0124FBE708B591ED007AF6EE27
:10EEF000007AB4EEE77AF1EE10FA06DD044801225A
:10EF00000521FEF79FFD002008BD0420FCE700BF9F
:10EF1000A05000202DE9F04188B080461B2200213E
:10EF200001A810EE107A10EE906A11EE105A11EE50
:10EF3000904A7AF08BF9A3238DF8043095238DF84D
:10EF400005300B238DF8063059F0F0FDCDF80700A1
:10EF500008F58150CDF80B101B2201A91830CDF80F
:10EF60000F70CDF81360CDF81750CDF81B4038F076
:10EF700063FC08B0BDE8F08170B58CB00D46144656
:10EF800006462B22002101A87AF060F9A3238DF810
:10EF9000043095238DF805300C238DF8063059F098
:10EFA000C5FD2B68CDF80F302368CDF813306B68A2
:10EFB000CDF817306368CDF81B30AB68CDF81F3043
:10EFC000A368CDF80700CDF8233006F58150EB6833
:10EFD000CDF80B10CDF827302B22E368CDF82B307D
:10EFE00001A9183038F028FC0CB070BD70B500F5E0
:10EFF0008154183400F54E56054606F16402204649
:10F000000E2138F0D9FA06F1900220460F2138F08F
:10F01000D3FA05F5525220460832102138F0CCFAC6
:10F0200005F5555605F554522046112138F0C4FA1D
:10F0300006F1480220466C2138F0BEFA06F174024F
:10F0400020466D2138F0B8FA05F5585220462C328A
:10F050000D2138F0B1FA05F55C5220460832BDE8C2
:10F060007040692138F0A8BA1FB5002301A900F546
:10F07000965001930293039302F09EF905B05DF858
:10F0800004FB000008B504F001F8BDE8084003F0F7
:10F0900015BD00007FB50E464FF6FF7104461546BC
:10F0A00001F0B6FFE8B11022002168467AF0CEF8F0
:10F0B000A3238DF8003095238DF8013004238DF8BB
:10F0C000023059F033FDCDF8030004F58150CDF83E
:10F0D00007101022694618308DF80B60039538F040
:10F0E0002BFC04B070BD0000A120704738B5044669
:10F0F00000F5815501F0A6FF183502460B49284658
:10F1000038F036FD04F50053284693F81D2D93F88A
:10F110001C1D38F069FD04F5965004F06FF904F5F4
:10F120009070BDE838400FF023BB00BF44DC0808F6
:10F1300037B5069D044600B92C7801B9697802B943
:10F14000AA7803B9EB78002064F3070061F30F207D
:10F1500062F3174063F31F6003B030BD2DE9F04F39
:10F160002DED0C8B9DB0E04C0D93D4ED379ADFED77
:10F17000DF5A90ED006A04F50054F7EE006AD4F807
:10F180002C3DD3ED367A93ED387AF0EEE77AB0EE97
:10F19000C77A77EE877A9246F4EEE67AF1EE10FAC5
:10F1A000C8BF86EEA78A06460F46DFEDD17AD8BFE4
:10F1B000B0EE668A28EE277AA6EE257A80ED007AF0
:10F1C000D4F82C3D93ED357A93ED376AB0EEC77ADB
:10F1D000B0EEC66A37EE067AB4EEE67AF1EE10FAD1
:10F1E000CCBFC6EE878AF7EE008A90ED017A68EE12
:10F1F000A77AE7EE257AC0ED017A39F0DFF9054606
:10F2000059F094FC814618EE900A8846FDF774F98F
:10F21000CDE9080118EE100AFDF76EF9CDE90601F7
:10F220007068FDF769F9CDE904013068FDF764F90C
:10F23000B04BB14ACDE90201CDE900982846AF496B
:10F24000AF4D38F02DFFAF4995ED00AA38461AF0C2
:10F2500065FA8DED160A9AED000ACDED170A30EE2B
:10F260004A0A8DED181A18F0E5F99DED167AD4EDDD
:10F27000E47AB0EEC77AB4EEE77AA5F59B63F1EED7
:10F2800010FA0C9300F10F82D4F82C3D1B7B002B5D
:10F2900000F00982B4F88E93C9F340099DED177A06
:10F2A000B0EEC77AF4EEC77AF1EE10FA00F3FE8101
:10F2B000D4F82C3D1B7B002B00F0F881B4F88E3382
:10F2C00003F001039DED187A0B93B0EEC77AF4EECC
:10F2D000C77AF1EE10FA00F3EB81D4F82C3D1B7BDA
:10F2E000002B00F0E581B4F88E33C3F38008B0EE54
:10F2F000C00AF4EEC07AF1EE10FA00F3DC81D4F823
:10F300002C3D1B7B002B00F0D681B4F88E33C3F369
:10F31000C00B0DAB00930B999FED7B8A5B46424679
:10F320004846FFF705FFC3B20BEE103AC0F30723C0
:10F330000AEE903AC0F307430CEE903A030E0DEE3E
:10F34000103A9DF834300F90002B40F0B7819DF8B3
:10F350003530002B40F0B281F8EE4B7A694ACDEDA2
:10F36000197AF8EE6A7AB0EE690ACDED1A7AF8EEFB
:10F370006C7A19AB394602F52070CDED1B7A4FF04F
:10F38000CBF98DED140ACDED150AB0EE409AF0EEF2
:10F39000608A9DF836305D4C002B40F094811CEE65
:10F3A000901AD4EDB40A97ED020AB0EE691A04F28D
:10F3B000FC504FF0CFFAB0EE40CA9DF83730002B2A
:10F3C00040F084819AED000A30EE4A0A18F032F9D2
:10F3D0001DEE101A4E48F0EE690A4EF0D1FF04F50A
:10F3E000E163DAF800201A6004F20C73F0EE40BA20
:10F3F00083ED00AA474D95EDDD1A4720F1EE410A55
:10F40000B0EE490A18F02AF995EDDD1AB0EE40AADF
:10F41000F1EE410A4820B0EE680A18F01FF995EDA8
:10F42000DE1AB0EE409AF1EE410A4920B0EE4C0AE5
:10F4300018F014F995EDDF1AF0EE408A4A20B0EE8C
:10F440006B0AF1EE410A18F009F996ED007AD6ED53
:10F45000017A9DF834308DED148A6AEE076AF0EE79
:10F4600040BACDED106A69EE276A8DED158ACDEDB3
:10F47000116AD4EDAF6A27EE267AD4EDB06A8DED2D
:10F48000127A67EEA67ACDED137AB3B99DF83530CE
:10F490009BB9B8EE4BBAF8EE6AAAB0EE690A1E48FC
:10F4A0008DED19BA19AB12AA10A9CDED1AAA4FF019
:10F4B0001FF88DED140ACDED150A9DF83630002B9E
:10F4C00040F0078196ED000AD4EDB10A134860EED2
:10F4D000200A1CEE901A28EE800AB0EE691A4FF04E
:10F4E00039FAF0EE40AA1BE0A0250020A4707D3F71
:10F4F00000D7233C89E20808A00E0908B90E0908C4
:10F50000783A00206858002000000000A055002034
:10F51000145C0020A045002044590020F859002028
:10F52000844814A9FEF74EFE9DF83730002B40F0BA
:10F53000D38096ED010AD4EDB60A7F4860EE200A2A
:10F54000B0EE691A1DEE101A20EE2B0A4FF002FAE7
:10F55000F0EE409AD5F82C3D1B7B7BBB19A9774870
:10F560008DED198A8DED1A8A4FF0ECF89FED740A33
:10F5700074484FF00BFA9FED720A73484EF02CFF5F
:10F5800019A972488DED198A8DED1A8A4FF0DAF8B3
:10F590009FED6B0A6E484FF0F9F967489FED680AD6
:10F5A0004FF0F4F904F5327393E807000C9B87E8F9
:10F5B000070003F59B631B68CAF80030B9F1000F20
:10F5C00000F08D80D5F82C3D83ED368A0B9B002B07
:10F5D00000F09080D5F82C3D83ED358AB8F1000F0E
:10F5E00000F09380D5F82C3D83ED388ABBF1000FF5
:10F5F00000F09580D5F82C3D83ED378A9FED558A34
:10F600009FED4F4AD4EDAF2A94EDB21AD7ED000A20
:10F6100062EE882A2AEE082A21EE081A60EE880A8D
:10F62000F0EE443AB0EE443AF0EE441AB0EE440A3A
:10F6300058F044FB9FED424AD4EDB02A94EDB31A42
:10F64000D7ED010A62EE882A29EE082A21EE081A6F
:10F6500060EE880AF0EE443AB0EE443AF0EE441A16
:10F66000B0EE440A58F02EFB9FED354AD4EDB12A96
:10F6700094EDB41AD7ED020A62EEC82A28EEC82A21
:10F6800021EE481A60EEC80AF0EE443AB0EE443A71
:10F69000F0EE441AB0EE440A58F018FB1DB0BDEC71
:10F6A0000C8BBDE8F08F4FF00109F7E5012309E667
:10F6B0004FF001081BE64FF0010B2AE6F0EE488AF6
:10F6C000B0EE489A65E69FED1ECA76E6DFED1CBAFD
:10F6D00090E6DFED1BAA23E7DFED199A3AE79DF8E4
:10F6E0003430002B7FF472AFD5F82C3D149AC3F858
:10F6F000D8206BE79DF83530002B7FF46FAFD5F83D
:10F700002C3D159AC3F8D42068E79DF83630002BBD
:10F710007FF46CAFD5F82C3DC3ED38AA66E79DF8B1
:10F720003730002B7FF46AAFD5F82C3DC3ED379A04
:10F7300064E700BFA0250020705A0020E85A00208E
:10F74000000000009C5B0020145C00204459002055
:10F75000F85900200000C8422DE9F04F2DED068B2E
:10F760008FB0B74C0393D4ED37AA04F5005480460C
:10F77000D4F82C3D1B7B0D461746002B00F02E8144
:10F78000B4F88E63C6F3400B06F0010AC6F3800995
:10F7900016F0080600D0012603AB4A4651460093F6
:10F7A00058463346FFF7C4FC94EDDD1A95ED000A88
:10F7B0000590F1EE410A9A2017F050FF94EDDD1A02
:10F7C000F0EE409AF1EE410A95ED010A9B2017F008
:10F7D00045FF94EDDE1AB0EE409AF1EE410A95ED48
:10F7E000020A984D9C2017F039FF94EDDF1AF0EED5
:10F7F000408A9D2097ED000AF1EE410A17F02EFF96
:10F8000098ED007AD8ED017A9DF80C3069EE876AA0
:10F810000027CDED066A69EE276AB0EE408ACDED8D
:10F82000076AD5EDAF6A0A9727EE267AD5EDB06A5A
:10F830008DED087A67EEA67A0B97CDED097AFBB9C4
:10F840009DF80D30E3B99DF8143007EE103A9DF89D
:10F85000153007EE903AB8EE477AF8EE677AB0EED8
:10F860006A0A0CAB08AA06A905F569708DED0C7A39
:10F87000CDED0D7A4EF03CFE8DED0A0ACDED0B0A72
:10F880009DF80E30002B40F0AE8098ED000AD5EDCB
:10F89000B10A9DF816106C4860EE200AB0EE6A1AA4
:10F8A00028EE800A4FF056F8B0EE40AA64480AA944
:10F8B000FEF788FC9DF80F30002B40F0978098ED04
:10F8C000010AD5EDB60A9DF81710604860EE200ACF
:10F8D000B0EE6A1A20EE080A4FF03CF8B0EE408A0B
:10F8E000D4F82C3D1B7B7BB959480C970CA90D977C
:10F8F0004EF028FF9FED570A53484FF047F89FED11
:10F90000550A52484FF042F8BBF1000F71D0D4F8BD
:10F910002C3DC3F8D870BAF1000F74D0D4F82C3D48
:10F92000C3F8D470B9F1000F77D0D4F82C3DC3F8E8
:10F93000E070002E7AD0D4F82C3DC3F8DC709FED37
:10F94000468A9FED444AD5EDAF2A95EDB21A62EE94
:10F95000882A29EE882A21EE081AF0EE443AB0EE01
:10F96000443AF0EE441AF0EE440AB0EE440A58F07D
:10F97000A5F99FED384AD5EDB02A95EDB31A62EEA0
:10F98000882A29EE082A21EE081AF0EE443AB0EE51
:10F99000443AF0EE441AF0EE440AB0EE440A58F04D
:10F9A00091F99FED2C4AD5EDB12A95EDB41A62EE8E
:10F9B000C82A28EEC82A21EE481AF0EE443AB0EEE2
:10F9C000443AF0EE441AF0EE440AB0EE440A58F01D
:10F9D0007DF90FB0BDEC068BBDE8F08F4FF001094B
:10F9E000CA46CB46D7E69FED1BAA5FE79FED198A73
:10F9F00076E79DF80C30002B8DD1D4F82C3D0A9A77
:10FA0000C3F8D82087E79DF80D30002B8AD1D4F8B1
:10FA10002C3D0B9AC3F8D42084E79DF80E30002BC0
:10FA200087D1D4F82C3D83ED38AA82E79DF80F30BA
:10FA3000002B84D1D4F82C3D83ED378A7FE700BFBB
:10FA4000A0250020A0550020F8590020705A002061
:10FA500044590020000000000000C84270B5044670
:10FA6000103043F097FA0B4E0B4B23613825601989
:10FA700043F0AEFC66513035B5F54E7FF7D104F555
:10FA80004E7044F023FF2046044934F059FB2046D1
:10FA900070BD00BFF41709080818090820110908EB
:10FAA00037B500F50D5101220831044636F0A2FBAE
:10FAB0001C4A1368D90706D41B4904F504531033B4
:10FAC0000B600123136004F50E5017490122183012
:10FAD00033F002FF0125002304F58151CDE90053E5
:10FAE000124A1831FD2033F089FE114B1A68D207F3
:10FAF00005D4104A1D6004F58A54083414600D487A
:10FB0000012133F005FF34F021FD0B4A0B48138827
:10FB100043F0400313800421002203B0BDE83040CD
:10FB200033F068BE145E002000220020A89509086A
:10FB3000185E00200C220020485F002010160908E3
:10FB40000069C0F3401070470F299DBF302303FBAD
:10FB50000100283000207047014B93F96203704781
:10FB6000A0450020024B93F8290D00F001007047DA
:10FB7000A0450020014BD3F8F40A7047A0450020AF
:10FB8000002910B517DB104C94F8FC2ACBB29A422E
:10FB900011D3D4F8F83A0122595CA4F5005000F0D2
:10FBA00063FD94F8193D38B99A0704D5074A1378CC
:10FBB00043F00403137010BD9B07FCD5034A137870
:10FBC00043F00203F6E700BFA0450020DC5E002002
:10FBD000022A10B50F4C12D13522A4F5005000F0C6
:10FBE00043FD94F8193D9B0705D50B4B1A7818B1C6
:10FBF00042F002021A7010BD42F00402FAE794F8D3
:10FC00001C2D8A42F7D143F0A7FBBDE8104043F01A
:10FC1000A7BA00BFA0450020DC5E0020064A92F88B
:10FC2000293D92F8282D03F00103134301D143F03D
:10FC3000A7B90020704700BFA0450020332901D09C
:10FC400044F064B97047000008B50A68332A07D049
:10FC5000382A08D10A790321FFF7BAFF012008BD2D
:10FC60000A790121F8E7BDE8084043F0F5BE00003D
:10FC700030B589B00446684606F028FD04F596556F
:10FC800004A806F023FD6946284602F0B3FF70B1D0
:10FC900004A9284602F0DEFF48B104A9684606F030
:10FCA00043FD236800221B6D69462046984709B032
:10FCB00030BD000000F5805292F85425D2070AD4D6
:10FCC00000F50052D2F82C2D117B09B1FFF7D0BFFF
:10FCD0000368DB6C1847704710B586B0044602A86D
:10FCE000019106F0F3FC02A904F5965002F082FFA0
:10FCF00028B12368019A1B6D02A92046984706B0D7
:10FD000010BD0000F0B5044685B0684604F596576E
:10FD10000E46154606F0DAFC6946384602F09AFFB0
:10FD200010B9002005B0F0BD3146384602F0B2FDF2
:10FD30000028F6D0002DF5D004F58054284694F81C
:10FD4000543543F0020384F85435EBE710B500F561
:10FD50000054D4EDDB7AF5EEC07AF1EE10FA8AB0F9
:10FD60004FF0000343D907930893099306AB01931F
:10FD700007AB03AA04A9009300F5965005AB02F067
:10FD800027FEDDED080A9DED070A76F005FFDDEDA3
:10FD9000090A76F001FFD4EDDB7A9DED047A77EE67
:10FDA000A76AB4EEE70AF1EE10FAF4EEC76AACBF48
:10FDB00001200020F1EE10FA0CD802309DED037AFC
:10FDC000F4EEC77AF1EE10FA0CD8003818BF012013
:10FDD0000AB010BDF4EEC77AF1EE10FA9CBF013004
:10FDE000C0B2EBE7012894BF00200120F0E700201B
:10FDF000EEE7000038B500F50055044695F8293DBA
:10FE00005A071AD443F0040385F8293D38F0D6FB8D
:10FE10000122112138F02EFB084BD3F86807036844
:10FE20009B68984718B995F96933032B05D120468B
:10FE30000621BDE8384000F015BD38BDA0550020B2
:10FE400008B500F5005090F8293D5A070BD56FF31F
:10FE5000820380F8293D38F0B1FBBDE8084000225C
:10FE6000112138F007BB08BD2DE9F043054685B0E8
:10FE7000684605F5965806F029FC6946404602F0AA
:10FE8000E9FEC8B105F50053424CD3F82C2D424F82
:10FE9000127B32B1D3EDDB7AF5EEC07AF1EE10FAD7
:10FEA0000DD8238823F4FF7323F001032380284611
:10FEB0000023FB73FFF7C4FF05B0BDE8F0832846BD
:10FEC00001F066F8064618B9284601F027F80646FC
:10FED0002846FFF73BFF814640B93EB12378002B0F
:10FEE00041D1637803F00103FB73E5E76378DB0737
:10FEF000F7D423780133DBB2082B237006D12846D0
:10FF0000FFF724FF10B1404602F0CEFD2378092B05
:10FF100002D1404602F0C0FD2378092BE1D92388A5
:10FF200023F4FF7323F0010343F48573238038F037
:10FF300045FB0222102138F09DFA58F0EFFD63686E
:10FF4000C01A47F23053984209D905F52D50134A8B
:10FF5000022114303CF094FD58F0E0FD606028462A
:10FF6000FFF748FFBDE7013B23702388C3F3080375
:10FF7000B3F5807FB5D1637860F30003637038F028
:10FF80001DFB4A46102138F075FA2846FFF758FF46
:10FF9000A7E700BF1C5E0020BD5E002024180908F2
:10FFA00037B5044601A900F5965004F5005502F056
:10FFB000BBFBD5F8403B834206D0C5F8400B38F078
:10FFC000FDFA3E2138F036FA04F5805395F9441BCA
:10FFD00093F8E82593F9E835994213D0FF2A11D018
:10FFE00085F8443B38F0EAFA95F8442B182138F0AC
:10FFF00041FA04F52D5095F9443B034A042114308D
:020000040801F1
:100000003CF03EFD03B030BD341809082DE9F04343
:1000100095B0064658F082FD03AB019306F596595C
:1000200002AB0024009305460EAB0BAA08A9484674
:10003000089409940A940B940C940D940E940F94C4
:10004000109402F0B3FCDFED437A9DED0A7AB4EE32
:10005000E77AF1EE10FA074637DB9DED0D7AB4EE44
:10006000E77AF1EE10FAACBF4FF001084FF000084C
:1000700007AB019311AB009304AA06AB05A9484650
:1000800011941294139402F0A3FC06F50054002876
:1000900094F9DC3A08BF002783B17FB1D4F82C3D36
:1000A0001B7B5BB1B8F1000F08D09DED057AF7EE30
:1000B000007AB4EEE77AF1EE10FA09D594F8483BED
:1000C00073B90023C4F84C3B0FE04FF00008CFE7B2
:1000D000D4F84C0B20BBC4F84C5BC4F8500B04E0C4
:1000E000D4F8500B20B9C4F8505B15B0BDE8F083CC
:1000F000281A43F698239842E3D9002584F8485BF0
:10010000C4F8505B38F05AFA2A461D2138F0B2F98B
:1001100006F52D50104A022114303CF0B1FCD0E716
:100120002D1AB5F57A7FE0D994F8483B002BDCD145
:10013000012584F8485B38F041FA2A461D2138F041
:1001400099F906F52D50054A022114303CF098FC2F
:10015000CBE700BF000000344C18090867180908F5
:1001600010B5044638F02AFA0022052138F082F949
:1001700004F52D50034ABDE81040042114303CF032
:100180007FBC00BF8418090800F5005090F8193DA5
:100190009B065ABF90F8180DC0F30010012070475D
:1001A00038B5044602F072FF4FF4804102F0ACF81B
:1001B00004F50052054692F8193DC3F3001181423F
:1001C0001CD060F3041304F52D5482F8193D143447
:1001D00060B138F0F3F902220B2138F04BF9084AEC
:1001E00020460221BDE838403CF04ABC38F0E6F930
:1001F0002A460B2138F03EF9024AF1E738BD00BF2C
:100200009C180908A718090870B500F500550446A0
:1002100095F95233ABB3D5F8A46C96B358F07EFC85
:1002200005F6E42393ED000ADFED167A9FED161A2A
:10023000DFED160A861B20EE270A692017F00EFA5A
:10024000BCEEC00A10EE103A9E4209D295F8293D44
:100250009A0716D520460021BDE87040FDF79ABCEC
:100260000FD995F8293D9B070BD420460121FDF7B6
:1002700091FC04F52C500122BDE870401221FDF7DD
:10028000E1BB70BD00007A440000804F0000000018
:100290000B46012B10B4114604D0052B06D05DF897
:1002A000044B70475DF8044B00F0DCBA5DF8044B7A
:1002B0000122142100F52C50FDF7C4BB2DE9F041BB
:1002C000044604F5005838F079F90122052138F088
:1002D000D1F898F956532046003D18BF0125FFF785
:1002E00053FF04F52D56143690B11D4A04213046B3
:1002F0003CF0C6FB0122102104F52C50FDF7A2FBB7
:100300000025294620460322BDE8F041FFF7C0BF83
:1003100004F54057D7F868070368DB6A984768B167
:1003200097F88D3253B197F98C32012B06DC0D4AC8
:10033000042130463CF0A4FB0125E2E7D7F868072A
:100340000368DB6A984718B1D8F8E03A1B0705D470
:10035000054A042130463CF093FBD2E7034AE7E725
:10036000BC180908D718090805190908141909083B
:1003700070B50446154638F021F90122062138F0FF
:1003800079F82046FFF700FF04F52D56143690B19A
:100390000122072104F52C50FDF754FB144A0421D7
:1003A00030463CF06DFB0025294620460422BDE87E
:1003B0007040FFF76DBF04F54053EDB2D3F8680706
:1003C0000368DB6A984768B104F50053D3F8E03A54
:1003D0001B0707D535B1074A042130463CF050FBD6
:1003E0000125E1E7044A042130463CF049FBDBE704
:1003F00038190908DF18090855190908F8B504461D
:1004000058F084FB284BB4F8BE201988274E91423F
:1004100005460ED01A80264B18603378A3B100240D
:10042000347038F0CBF822461321BDE8F84038F09C
:1004300021B833781F4FC3B93B782BB11C4B1E4AF0
:100440001B68C31A934200D8F8BD0123337004F52A
:100450000053D3F82C0D037B0BB1FEF735FA38F0BF
:10046000ADF80122132138F005F83B78002BEBD0D2
:100470003378002BE8D00E4A10491368EB1A8B42F0
:10048000E2D904F500541560D4F82C2D137B002B11
:10049000DAD0002313730A4AD4F82C0D1371BDE887
:1004A000F840FEF7E1B800BF265E0020245E002081
:1004B000285E0020255E002080841E0040420F0040
:1004C000BD5E00207FB500F5005300F54E550835A0
:1004D00093F8481B0446284657F04EFB04F5965601
:1004E000684606F0F3F86946304602F083FB04F5EF
:1004F0004053029AC3F8A822039AC3F8AC222021E1
:10050000304601F001FFD0B1284657F087FB04F5D3
:100510004A55FDEEC07A203504F5805417EE901A46
:100520000222284617EE906A06F0D4F894F8543563
:10053000DB0706D401223146284606F0CBF804B08A
:1005400070BD0121284606F06DF90028F2D0F6E7CB
:10055000012070470020704700207047002070473E
:10056000002070470020704700207047002070472F
:100570009FED010A704700BF000000009FED010AD7
:10058000704700BF0000000070470000104A026082
:10059000104A426002F15001816002F58251C1604F
:1005A0000D49016102F6E411416102F6E811816131
:1005B00002F5F461C16102F2A471016202F5F56114
:1005C00002F2AC728262054A4162C262704700BFA9
:1005D000E0190908E848002060380020B82600200B
:1005E000042917D8DFE801F003070B0F130000F50B
:1005F0005E501C30704700F55D502C30704700F5A0
:100600005F500C30704700F55F503C30704700F58C
:100610006050FAE70020704700F54050D0F86807B6
:1006200003685B681847000038B500F5405504467C
:10063000D5F8680703685B6998470A4B04F50052D0
:10064000187492F81C2DD5F86807DA7003685B6A95
:100650009847014604F593501030BDE8384030F01B
:100660000BBE00BFBD5E00202DE9F84F00F5005A1B
:1006700006469AF81C3D8B420F46914605D18AF8F2
:100680001D2D01252846BDE8F88FFFF7A9FF044678
:1006900020B9304635F056FF2546F3E7DAF82C3D11
:1006A0001B7B06F52D5883F0010B08F11408EBB9FC
:1006B000236859461B6820469847054680B306F5CF
:1006C000405306F58150C3F868474A4639468AF8D0
:1006D0001C7D8AF81D9D183037F086FA40460021AF
:1006E00041F0FAFE3046FFF79FFFCBE703689B68B7
:1006F0009847E0B11C4800F037FC0546B8B92368BC
:1007000020461B6A9847194A0346042140463CF09C
:10071000B7F937F053FF3A460A2137F0ABFEB1E79D
:10072000236820461B6A9847114A0346EDE70E48A6
:1007300000F036FC0028BBD106F54053D3F868071B
:100740000368DB6898470028B2D023682046DB683E
:10075000984705460028ABD1236820461B6A984776
:10076000044A0346D1E700BFA02500206819090804
:10077000BA190908911909080148FFF775BF00BFA8
:10078000A025002070B5234B93F8293DDB070546D3
:100790000C46164605D5002363602360A3603360D2
:1007A00070BD42F0D9FD037F002BF4D0EB699FEDC3
:1007B0001A7A1B68B3F90A3007EE903AF8EEE77A36
:1007C000C7EE876AC4ED016A2B6A1B68B3F90A3069
:1007D00007EE903AF8EEE77AC7EE876AC4ED006A52
:1007E0006B6A1B68B3F90A305B4207EE903AF8EE89
:1007F000E77AC7EE876AC4ED026AAB6A1B68B3F991
:100800000A3007EE903AF8EEE77AC7EE876AC6ED4F
:10081000006AC5E7A045002000007A440020704728
:100820000120704700207047002070470048704743
:10083000686E090800487047281A090800207047A8
:1008400043691A680023C2F8D43042691268C2F8BA
:10085000D83042691268C2F8DC3042691268C2F8C6
:10086000E03070470A4608B50021FFF7FDFE034A55
:10087000137843F00803137008BD00BFDC5E00204E
:10088000012070470020704701207047002070470A
:1008900000487047801A090800487047881A0908FC
:1008A0000320704730B5084B03F54B52083204461D
:1008B00000F1300507CA85E8070003F5A653183391
:1008C00001201B68E36330BDA025002030B52DED6D
:1008D000028B044687B0574D002301AA03A995ED6A
:1008E000378A039304930593FFF74CFF63689DEDEC
:1008F000037AD3ED0E7A68EE277A27EE277A8DED0C
:10090000037A9DED047A67EE277ACDED047AD3ED74
:100910000F7A28EE277ADDED057A67EE877ACDED3E
:10092000057AD3ED107A93F9443028EE278ADDED6D
:10093000017A27EE888A8DED018A1BB903A9284622
:10094000FDF724FC3C4A94ED0C7AD2EDB27A636850
:1009500094ED0F0AD3ED0E6A77EE677AF0EEE77A40
:10096000F4EEE67AF1EE10FA44BFDDED037A77EEAD
:10097000877A94ED0D7A48BFC4ED0C7AD2EDB37A44
:10098000D3ED0E6A77EE677AF0EEE77AF4EEE67A68
:10099000F1EE10FA44BFDDED047A77EE877A94ED3C
:1009A0000E7A48BFC4ED0D7AD2EDB47AD3ED0F6A5A
:1009B000236977EE677AF0EEE77AF4EEE67AF1EE05
:1009C00010FA42BFDDED057A77EE877AC4ED0E7A34
:1009D000D3ED867A30EE670A16F02CFE6368D3ED0D
:1009E000107AB0EEC00AB4EEE70AF1EE10FA09D5BB
:1009F00094ED0F0ADDED017A30EE270A16F01AFEAB
:100A000084ED0F0A00230D488DF808308DF8093069
:100A10008DF80A308DF80B30029BD0F8300D04F1C0
:100A20003C0204F13001FEF799FB07B0BDEC028BEC
:100A300030BD00BFA0250020A0550020A04500200B
:100A40000020704701207047012070470020704748
:100A500000487047E01A090800487047E81A09087A
:100A6000012070471FB5044600236A4601A901937F
:100A700002930393FFF786FE6369029A1B68C3F82B
:100A8000D4206369019A1B68C3F8D8206369009A6F
:100A90001B68C3F8DC206369039A1B68C3F8E02075
:100AA00004B010BD0120704700207047012070473E
:100AB000002070470048704762E708080048704708
:100AC00062E7080804207047012070477FB50023C3
:100AD0000393049305930193094800238DF808308C
:100AE0008DF809308DF80A308DF80B30029BD0F864
:100AF000300D01AA03A9FEF731FB07B05DF804FB36
:100B0000A045002001207047002070470120704759
:100B10000020704700487047901B09080048704744
:100B20009C1B09080220704710B5044686B00023BC
:100B300001AA03A9039304930593FFF723FE6368B7
:100B40009DED037AD3ED0B6ADDED047A93F9443021
:100B500027EE267A67EEA67A8DED037ACDED047A3C
:100B60001BB9144803A9FDF711FB6368DDED057A95
:100B700093ED0C7A104867EE877A93ED0D7ACDED00
:100B8000057ADDED017AD0F8300D002367EE877A23
:100B90008DF808308DF809308DF80A308DF80B305B
:100BA000029BCDED017A01AA03A9FEF7D5FD06B09F
:100BB00010BD00BFA0250020A045002038B5044688
:100BC00043F0DAFE43F0A8FF04F50054054643F075
:100BD0003DFF43F02FFCD4F82C0DFDF745FD2846D2
:100BE000BDE8384043F03ABF10B500F50054142179
:100BF000D4F8E80A42F000FCD4F8EC0A142142F0E0
:100C0000FBFBD4F8F00A1E2142F0F6FBD4F8F40AFC
:100C10001421BDE8104042F0EFBB000038B5054696
:100C200042F09AFB42F0ECFA05F50054C4F8E80AE9
:100C300042F092FB42F0EEFAC4F8EC0A42F08CFB70
:100C400042F0F2FAC4F8F00A42F086FB42F0F6FAFB
:100C50004FF47A71C4F8F40AD4F8E80A42F0C8FBF9
:100C6000D4F8EC0A4FF47A7142F0C2FBD4F8F40ADB
:100C70004FF47A7142F0BCFBD4F8F00A4FF47A7169
:100C800042F0B6FB2846FFF7AFFF94F8193D43F05A
:100C9000080384F8193D38BD08B543F03DFF43F023
:100CA00061FDBDE8084043F013BD000000F50050B1
:100CB000D0F82C0DFDF708BE38B500F500540546F8
:100CC00094F956332BB900212846BDE83840FCF78B
:100CD00047BFB4F858338B4219D994F8293DDA0745
:100CE0000FD442F039FB037F1BB9D4F82C3D1B7B9A
:100CF0003BB194F8283D01335BB2022B02DC84F84F
:100D0000283D38BD032384F8283D0121DCE794F811
:100D1000283D013B5BB2002BF1DC002384F8283D29
:100D200094F8293DDB07CED4EBE7000038B50D463B
:100D3000044657F0F3FE002D0B4B09DD04F500547B
:100D4000186094F8193D6FF3C30384F8193D38BD5A
:100D50001B68C01AB0F5C87FF9D904F5005494F89F
:100D6000193D43F00803F0E72C5E0020F7B5044678
:100D700057F0D4FE064642F0EFFA42F0C1FA04F50D
:100D80000055B0B395F8183D43F0200385F8183DA1
:100D9000D5F8F03A20461989FFF78EFFD5F8F03ADA
:100DA00004F54057B3F90A102046FFF7BFFFD7F804
:100DB00060379FED307AF31A07EE903AD5F8F03AA3
:100DC000F8EE677AB3F90A3067EE877A04F54A508D
:100DD000CDED007A07EE903AF8EEE77A6A4601A97F
:100DE0001430CDED017A38F041FDC7F8606703B0EB
:100DF000F0BD95F8293DDB07F9D404F54053D3F84D
:100E00006007361A42F05EF980BB42F0A5FA9FED0A
:100E10001A7AD0ED067A67EE877A9FED187AF4EEAB
:100E2000C77AF1EE10FAD8BFF0EE477AFCEEE77A17
:100E300017EE903AB342DAD895F95633002BD6D054
:100E400042F08AFA037F23B9D5F82C3D1B7B002B97
:100E5000CDD037F0B3FB0222114637F00BFB012156
:100E6000204603B0BDE8F040FCF77ABE4FF47A7339
:100E7000E0E700BF6F12833A00007A440000C842E6
:100E800038B5044600F58665284604F07DFB94F8E5
:100E900041049FED087A242202FB0055D5ED0B7A20
:100EA00067EE877A04F54053FDEEE77AC3EDA47A46
:100EB00038BD00BF0000C842FEF718B90148FFF76F
:100EC0009DBA00BFA025002010B5838F044643B90A
:100ED00035F04EFE92224FF4801135F001FE638F03
:100EE000A387A08F10BD000038B500F596550446C5
:100EF000284600F0DBFC04F58053022283F8E0244E
:100F000004F16800FFF7E0FF014604F6980015F0D1
:100F100085F82846BDE8384000F0C2BD38B500F578
:100F200096550446284600F00DFF08B9002038BD4C
:100F300004F50054D4F82C3D1B7B63B910212846DE
:100F400001F0E2F90028F2D14FF400712846BDE823
:100F5000384001F0D9B98021284601F0D5F90028A0
:100F6000E4D11021F2E7000038B500F50053054642
:100F700093F8293D5B0709D4FFF7D0FF044618B961
:100F800005F5965000F0DEFE204638BD0024FBE754
:100F900008B500F5965000F0D5FE002008BD000011
:100FA00010B500F59654204600F0CCFE50B1042157
:100FB000204601F0A9F928B120462021BDE81040C3
:100FC00001F0A2B9002010BD38B500F50055044667
:100FD00095F8183D590719D5D5F82C3D1B7B2BB931
:100FE00020460021BDE83840FCF7A4BD00F5405381
:100FF000D3F868070368DB68984738B195F8193D5E
:101000001A0703D595F8293DDB07E9D538BD00005F
:1010100037B500F581551835044604F500542846C7
:10102000019136F029FD94F8183D019960F3C3034E
:10103000284684F8183D03B0BDE8304037F088BA40
:101040000720704700487047F41B090837B505466C
:101050001048FFF739FF0190EC2005F05BFE0446D5
:1010600010B10199FDF7A0FA05F50050C0F82C4D1C
:1010700024B990F9A413084805F0F2FA074920466C
:1010800033F06CFA012032F0EDFE03B0BDE83040E1
:1010900033F05CBA08260020FC1B0908D8DB0808DE
:1010A00073B5044600F59350103030F099F820469F
:1010B000FFF7BAFA04F5355004F026FE04F5875020
:1010C000103004F5866644F08FF9304604F00EF9CE
:1010D00004F52D5014303EF00BF92046FFF79EFD2D
:1010E0002046FFF7B3FF5F48FFF7EEFE082005F04C
:1010F00011FE18B14FF07E530360436004F50055B4
:10110000C5F8300D42F028F99922292143F0D2F890
:1011100042F022F942F042F82046FFF7BDFD95F873
:10112000193D04F5915043F0400385F8193D1C30FA
:1011300045F066FE4C4B4D491B68986A03684FF4B6
:101140007A72DB6A98470423C4F8743104F590700E
:101150000CF084FF06F09CFB4FF40053036306F091
:1011600097FB07F027F88023C4F844340121304668
:1011700004F01AFB3E4B00933E4B019304F5815063
:1011800002AB13E90600183036F022FB2046FFF7C9
:10119000ABFE4FF40023C4F8A83BD5F82C0DFDF7A7
:1011A0000DFA012104F52C50FCF7B6F910B12046D8
:1011B000FFF77CFD04F168063046FFF785FED5F8A1
:1011C0002C3D07EE900A04F54B50D3ED390AB8EEEA
:1011D000670AF2EE0E1AB6EE001A1C3038F0CCFF99
:1011E0003046FFF771FED5F82C3D07EE900A04F566
:1011F0004C50D3ED390AB8EE670AF2EE0E1AB7EE8C
:10120000001A203038F0E2FD3046FFF75DFED5F8D9
:101210002C3D07EE900A04F54D501430D3ED390AF9
:10122000B8EE670AF2EE0E1AB1EE041A38F0CEFDEF
:1012300095F863131A222046FFF716FA60B92122A7
:1012400001212046FFF710FA95F8193D43F00203FB
:1012500085F8193D02B070BD074A137843F00803C2
:101260001370F1E708260020105E0020BD0E010873
:10127000A0250020B90E0108DC5E0020836833B988
:10128000C36823B94068003818BF012070470120A7
:10129000704700002DE9F0412DED048B92B004461B
:1012A00002AD284605F012FA94F8D433002B70D022
:1012B00004F580630FCB85E80F0094F81034D4ED6B
:1012C000F28A94EDF38A94EDF49A002B61D094F8AD
:1012D000E833002B5DD02846D4F8D883D4F8DC73EB
:1012E000D4F8E063D4F8E443FFF7C8FF002855D1F1
:1012F0002E4B01932D22002106A877F0A7FFA323F0
:101300008DF8183095238DF8193046238DF81A3052
:1013100057F00CFC9FED260ADFED267ACDF81F1062
:1013200068EE808A28EE008A68EEA78A28EE278A6F
:10133000FDEEE88ABDEEC88A18EE903A29EE000A62
:10134000ADF8233018EE103A20EE270ACDF81B0036
:10135000ADF8253016F042F9BCEEC00ACDF8358064
:1013600010EE103AADF82730019BCDF82930049BE0
:10137000CDF82D30059BCDF83130CDF83970CDF852
:101380003D60CDF8414037F019F92D2206A936F01D
:1013900053FA12B0BDEC048BBDE8F08101AA002124
:1013A000284605F04FFA0028A2D0A3E75241C07F9B
:1013B000E02E65420000C84230B52DED028B8BB0A7
:1013C000044624220D4601A8002177F03FFFA32305
:1013D0008DF8043095238DF8053048239FED1F8A42
:1013E0008DF8063057F0A2FBD4ED847A2B68CDF847
:1013F0000F3067EE887A95ED020ACDF80B1017EEE4
:10140000903AD4ED857ACDF8133067EE887A6B6820
:10141000CDF8173017EE903ACDF80700CDF81B3015
:1014200016F0B2F810EE103A94ED860ACDF81F309F
:1014300020EE080A16F0A8F810EE103ACDF8233086
:1014400094F824338DF8273037F0B8F8242201A916
:1014500036F0F2F90BB0BDEC028B30BDE02E6542E8
:1014600030B5104689B00D461446FFF707FF28BB7C
:10147000002301931822002102A877F0E7FEA3239E
:101480008DF8083095238DF8093049238DF80A30FE
:1014900057F04CFBA3680593E3680693019BCDF8D6
:1014A0000F100793CDF80B008DF8135037F086F826
:1014B000182202A936F0C0F909B030BD01AA0021F6
:1014C000204605F053F90028D2D0D3E710B590B0EC
:1014D000044604A805F0FAF804A9204601F08AFBA6
:1014E000002846D001F0D2FD01A901F07DF902A942
:1014F000204600F0C3FC00283DD0DDED027AF1EE7D
:10150000677A03AA002104A8CDED027A05F09AF9C2
:1015100008B91A4B03931F22002108A877F096FE02
:10152000A3238DF8203095238DF821304A238DF8A0
:10153000223057F0FBFA069BDDED017ACDF82B3017
:10154000079BCDF82F30F1EE677A039BCDF833304F
:1015500017EE903ACDF83730029BCDF82710CDF832
:101560002300CDF83B3037F029F81F2208A936F0C8
:1015700063F910B010BDDFED027AC2E75241C07FBF
:101580005241C07F0023036043608360C3600361F6
:1015900043618361C36103627047000090F8C43205
:1015A000B02202FB030390F8082393F8A13012B194
:1015B000012B28BF01231846704700002DE9F04F8A
:1015C00004468BB04FF0000A0D461CF0CFF884F8AB
:1015D00020A204F509704FF07E5756F007FC4FF437
:1015E0007A73A4F87A3284F8805204F52170C4F832
:1015F0006072C4F86472C4F86872002505F066F879
:1016000004F531790323C4F8983204F53A76C4F826
:10161000AC52C4F8B052C4F8B452C4F8B852C4F8CA
:10162000BC52C4F8C0524846FFF7ACFF04F54E7BED
:101630003046FFF7A7FFC4F82C53C4F83053C4F862
:1016400034535846FFF79EFFC4F85C53C4F8605308
:10165000C4F86453C4F86853C4F86C53C4F87053A6
:10166000C4F87453C4F87853C4F87C53C4F8805356
:10167000C4F88453C4F88853C4F8A453C4F8A853D6
:10168000C4F8AC53C4F8C053C4F8BC53C4F8B8533E
:10169000C4F8C853C4F8CC53C4F8D053C4F8E453C6
:1016A000C4F8E053C4F8DC5304F57B70C4F8B47399
:1016B000C4F8D87305F00AF804F5806005F006F860
:1016C00004F2144304F586601D605D6004F58463D4
:1016D00004F27C481D605D609D6004F0F7FF04F239
:1016E000444340461D605D609D606D4BC4F85434BA
:1016F00004F51073C4F8583404F51173C4F85C345D
:1017000004F51273C4F8603404F51373C4F8643438
:1017100004F25123C4F8683404F51473C4F86C342B
:1017200004F58E6304F254421D605D609D60FFF716
:1017300029FF04F59460FFF725FF04F59A6304F28E
:10174000BC501D605D609D6004F2DC431D605D6007
:101750009D6004F59D631D605D609D6004F2F4432F
:101760001D605D609D6004F204531D605D609D60BE
:1017700004F214531D605D609D6004F5A763C2F818
:10178000D470C2F8D8701D605D609D6004F244534F
:101790001D605D609D6004F5AC631F605D6004F2D8
:1017A00084531D605D609D6004F5B2631D605D60E3
:1017B0009D6004F5B5631D605D609D6004F086FF6B
:1017C00004F2CC5324221D605D6004F2D4535146D0
:1017D0001D605D6004F2DC5340461D605D6077F083
:1017E00035FD04F5C060C8F82070C8F81070C8F85E
:1017F0000070FFF7C7FE04F2246304F27C601F60F0
:101800009D605D60DD6004F234631D605D609D601D
:1018100004F5C8631D605D609D6004F24C631D604B
:101820005D609D6004F5CB631D605D609D6004F2AA
:1018300064631D605D609D6004F048FF194B1A49A8
:101840001C60204632F07CFC51462422584677F03A
:10185000FDFCC4F85873C4F84873C4F8387304F531
:101860002B7207CA04F52E7383E80700484694EDEF
:10187000B01AD4EDAF0A94EDAE0A16F0AFFA3546C1
:10188000494668466E4616F0CBF90FCE0FC50FCE0F
:101890000FC533682B6020460BB0BDE8F08F00BF4A
:1018A000DC1E0908305E0020781D090810B50446CA
:1018B00088B001F057FC94F93E32012B02D1274841
:1018C00004F0ECFE022B0AD1032384F83E3204A973
:1018D000012304F111008DF8103033F0F9F994F878
:1018E0003E3284F8A83204F2544001F0F7FB94F938
:1018F0003D32642B30D1652304A904F23D208DF8DC
:10190000103033F023FA04A9204631F0F9FC18B363
:1019100004238DF818300023CDE9013303930F23FE
:101920000593694604A831F06DFE059B28B108AA0D
:1019300002EB8302009942F8581C0133112B0593E6
:10194000EFD954F093FE9DED031ADDED020A9DEDF3
:10195000010A652154F048FE08B010BD0C1C0908AE
:1019600070B500F52B7600F52E758CB00446314627
:10197000284617F073FEE0B996E8070085E80700EF
:1019800004F5317194EDB01AD4EDAF0A94EDAE0ABE
:101990000191084616F022FA02AD019902A816F04C
:1019A0003FF90FCD04F53A740FC40FCD0FC42B6867
:1019B00023600CB070BD000013B540F2751200F545
:1019C0000971044601A811F025FB04F2544001F00E
:1019D0006FFD20461CF0F6F801A811F03DFB02B0A7
:1019E00010BD0000F8B54B68C0F810328B68C0F825
:1019F0001432CB68C0F8183201F1100607460C46C5
:101A000000F54E750FCE0FC50FCE0FC533682B6096
:101A100004F1440207CA07F54B7383E8070004F199
:101A2000500207CA07F5577383E8070004F15C0208
:101A300007CA07F55A7383E80700683494E807007B
:101A400007F55D7383E80700384601F09FFC3846D0
:101A5000BDE8F84001F082BC13B5044600F25440E2
:101A6000019003F03DF904F5BE610198009102F088
:101A700025FD0099204602B0BDE81040FFF7B2BF37
:101A80004A78064BC2F340121A754A78C2F38012A4
:101A90005A750A78C2F300129A757047BD5E00202D
:101AA00013B540F24D32044600F5097101A811F05A
:101AB000B1FA002104F2544001F028FF94F8783282
:101AC00023B120461CF000FE84F8780201A811F032
:101AD000C3FA02B010BD000038B590F824330546B3
:101AE0000C462BB1032B0BD095F88032DB070CD4BE
:101AF00005F27C630FCB84E80F0095F88C0603E0B9
:101B00001CF0E0F80028EFD038BD0020FCE7000012
:101B100000F2544090ED350A7047000000F2544046
:101B200090ED360A7047000010B490F824230C465C
:101B30002AB1032A0AD000205DF8044B704700F553
:101B4000B56007C884E807000120F5E75DF8044B9D
:101B50001CF076B890F89C03431E584258417047D9
:101B600038B590F824330D468BB900F2544001F09B
:101B700007FD044610B90024204638BD01F05EFC84
:101B8000D5ED007A27EE800A85ED000AF4E7D0ED66
:101B9000E67AC1ED007A90F89443002CEBD090EDFA
:101BA000E47ADFED086AB4EEE67AF1EE10FAF7EEC9
:101BB000006AB8BFB0EE667A67EE877AC1ED007A48
:101BC000DAE700BF0000003490F82433032B01D182
:101BD0001BF0B6BF0020704790F82423032A01D1E0
:101BE0001CF028B900F2544002F0EAB830B50546BE
:101BF00085B00C469AB1032A1BD005F52B7017F05F
:101C000067FD01A920468DED010ACDED020A8DED9B
:101C1000031A17F00BFB0123184605B030BD90F8EE
:101C2000F035002BF8D000F224630FCB84E80F00CE
:101C3000E3E790F87832002BEED01CF0D5F8DCE723
:101C400090F82423FFF7D2BF7FB590F8242332B158
:101C5000032A4FF0000309D0039304930CE000F231
:101C6000544007B05DF804EB01F0D4BC03A9039322
:101C7000049305931BF05AFF9DED030ADDED040A62
:101C800007B05DF804FB000037B5044640F2C752C8
:101C90000D4600F5097101A811F0BCF9204629464E
:101CA0001CF03AF894F82433032B08BF044601A82B
:101CB00018BF002411F0D0F9204603B030BD000059
:101CC00010B52DED028BB0F890361B0782B004469C
:101CD00030D5D0F838349FED198A07EE903AB8EE37
:101CE000E77A01A927EE087A00F515708DED017AE3
:101CF00032F0DAFFD4F83C3407EE903AF8EEE77AA7
:101D000001A967EE887A04F51670CDED017A32F0FC
:101D1000CBFFD4F834349FED0A7A07EE903AF8EE10
:101D2000E77A01A967EE877A04F51770CDED017A9D
:101D300032F0BAFF02B0BDEC028B10BD95BFD633B6
:101D40000AD7233C90F82403003818BF01207047BD
:101D500038B590F82423032A0C4604D11BF0E6FE84
:101D60000125284638BD90F87056002DF9D000F2B4
:101D7000646393E8070084E80700F2E710B590F881
:101D8000242303460C461AB1032A0BD0002010BDB1
:101D900090F878060028FAD003F5BE63D3F88430B3
:101DA0000B60F4E71BF0D8FE012084ED000AEEE79B
:101DB00030B590F8243385B005460C4623B1032B8B
:101DC00009D0002005B030BD00F2544005B0BDE898
:101DD000304002F075BA002302A9029303931BF06E
:101DE0008DFE0028EDD001A928461BF093FE0028A7
:101DF000E7D0029B2360039B6360019BA360E1E744
:101E00001FB500230C4601A9019302930393FFF72A
:101E1000CFFF28B1019B2360029B6360039BA360FB
:101E200004B010BD90F824231AB1032A05D0002075
:101E3000704700F2544002F077BA1BF05FBE00001A
:101E400013B500230C46694600930193FFF7EAFFA0
:101E500018B1009B2360019B636002B010BD0000BD
:101E600090F824231AB1032A05D00020704700F20D
:101E7000544002F04BBA1BF04DBE000013B50C46A7
:101E800001A9FFF7EDFF08B1019B236002B010BD6F
:101E900090F93E323BB990F8803213F0010F14BF35
:101EA000032000207047032070470000F7B5044668
:101EB000FFF7EEFF0546002862D0032839D194F8D9
:101EC00078326BB394F88032D8072BD501A920461D
:101ED0001BF0E8FFBDF80430002B18BF002594F874
:101EE000206206F0FD06012E4AD10023032D019346
:101EF00007D101A920461BF0E1FF20461BF0BEFFE1
:101F0000064604F2544002F01FFB08B994F821037E
:101F10009DF80430D90703D55A0701D59F0632D45E
:101F200000252DE020461BF04FFD002808BF0025AE
:101F3000D5E70025D3E713F0020F2EE094F95032D5
:101F400023B99DF80430DB092FD0E9E7002EF8D043
:101F50000DF0AAFBFFF722FB022807D99DF80530F8
:101F60009806DDD59DF80430D906D9D5FB6A93F8DB
:101F70009C30002BE5D118E0DA0601D41B0718D5F8
:101F8000284603B0F0BD0028FAD094F82123B4F914
:101F90009036002ACFD013F0010FF1D1154B1F68F6
:101FA000FB6A93F89C30002BC8D19DF804309C0745
:101FB000E2D405F06DFC05F069FB0028B0D10DF00E
:101FC00073FBFFF7EBFA0228AAD90DF06DFB90F82E
:101FD000C432B02202FB030090ED2F7AF0EE007ABB
:101FE000B4EEE77AF1EE10FA9AD59DF80530DB09E8
:101FF000C6D195E7105E00202DE9F04790F87832C1
:1020000092B00446002B00F0948020461CF0BAF8F1
:102010002046FFF74BFF03287BD104F54E780027BD
:10202000414620460097019702971BF0B3FE694690
:1020300020461BF0A5FE009BC4F81032019BC4F89B
:102040001432029BC4F81832204601F09FF9204652
:1020500001F084F913F07CFF054620461BF040FD9B
:102060000028A8BFC6B203AA4FF0FF312046BCBF6C
:1020700095F80A9395F80B630397A8BFB1460497A8
:1020800005971BF077FD03A817F022FB4FF00C0A11
:102090000AFB095084EDD70AC4EDD80A84EDD91A99
:1020A00004F5577100F5117017F022FB04F55D7708
:1020B0000AFB065584EDCB0AC4EDCC0A84EDCD1A9B
:1020C0003A464FF0FF31204605F5C4751BF066FD1A
:1020D00095E8070006AE86E807003946304617F057
:1020E0006DFB04F53172414609A815F029FD314612
:1020F00009A815F0A7FC09A9204684EDDA0AC4ED69
:10210000DB0A84EDDC1A1BF0D9FE09A92046FFF793
:10211000B7FC94F89236002B3AD109A804F0D6FA0D
:1021200009A920461BF0DAFD90B3012384F892360A
:102130002EE0D0F87C321BB956F0F0FCC4F87C02DB
:10214000154B1B68D86A03685B68984788B156F0DE
:10215000E5FCD4F87C32C01AB4F87A32984204D93B
:1021600020461CF0B1FA84F8780294F878327BB1FA
:102170004BE756F0D3FCD4F87C32C01A41F28733D7
:102180009842E4D836F01AFA36F0FEF90028DED18B
:1021900012B0BDE8F08700BF105E002090F8243335
:1021A00023B1032B4FF0000007D0704790F93E2277
:1021B000032A04D10A70012070470870FBE7184613
:1021C0007047000073B50D460DF107010446FFF797
:1021D000E5FF064628B19DF807302BB1032B09D047
:1021E0000026304602B070BD04F27C630FCB85E858
:1021F0000F00F6E7294620461BF064FD94F878624C
:10220000EFE7000037B50D460DF107010446FFF773
:10221000C5FF28B19DF8072029462046FFF7E6FCB8
:1022200003B030BD37B50D460DF107010446FFF789
:10223000B5FF28B19DF8073023B1032B11D0002042
:1022400003B030BD04F2F4531B682B6004F5BF6388
:102250001B686B6004F2FC531B68AB6094F8F005DC
:10226000EEE7204629461BF08BFD94F87802E7E75D
:1022700010B50446FFF70CFE18B1032807D0002064
:1022800010BD04F25440BDE8104001F04DB994F87F
:102290007832002BF3D020461BF096FB0028EED0BE
:1022A00094F8203203F0FD03012BE9D194F82403C4
:1022B000C31E58425841E3E710B50446FFF7E8FD56
:1022C00080B1032810D194F8780250B156F026FC62
:1022D000D4F87C32C01A44F62063984294BF0020A0
:1022E000012010BD0120FCE70020FAE708B50246F6
:1022F000FFF7CEFD032804D110461BF0DFFD0120BF
:1023000008BD0020FCE7000013B50C4601A9FFF74B
:10231000EDFF20B1019B1C4214BF0120002002B040
:1023200010BD000030B585B00446019102F0FEFDFD
:102330000199054610B9002005B030BD019102F0A9
:10234000C7FD01990028F6D0284602F0C5FD0028F7
:10235000F1D0B4F890365907EED494F82133002B1D
:10236000EAD00B4A1268D26A92F89C506DB103A968
:102370002046FFF7BBFF30B19DF80E309A07DBD542
:10238000C3F38000D8E72846D6E71846D4E700BF55
:10239000105E002010B50446FFF77AFD032804D133
:1023A0002046BDE810401BF063BC002010BD0000BB
:1023B0002DE9F04190F824338CB00027032B06461A
:1023C0000C46154600970197029719D11BF088FB20
:1023D0006A4680464FF0FF3130461BF0DFFBB8F114
:1023E000FF3FA760676027600DD113F0B1FD2B465A
:1023F00090F80B13224612F039FE0CB0BDE8F081C4
:102400004FF0FF38EBE713F0A3FD2B4622465FFAAF
:1024100088F112F02BFE95ED000A684617F094F94A
:1024200003A920468DED051A8DED030ACDED040AB2
:1024300017F0C4F906F5317206F54E7103A815F0D0
:102440007FFB214603A815F0FDFA84ED021A84ED06
:10245000000AC4ED010A95ED007ADFED037AA7EEDC
:10246000271A84ED021AC8E70AE81C411FB5DFED00
:102470000B7A20EE270A0C461946094BCDE900429B
:10248000BDEEC00A18688DED020A064B9DF81820B3
:10249000C06A10F0B9FF04B010BD00BFE02E654265
:1024A000105E0020201C09082DE9F0472DED028B5D
:1024B00092B0002504460F464FF07E5A00F54E714B
:1024C00006A89046CDF818A009950895079516F02E
:1024D0004FFB05F0DDF905F0D9F881462046FFF7FE
:1024E000D7FC032803D094F82433032B4FD19FED5E
:1024F000558ADFED558A00262379F2B2934247D9F7
:102500000AAA71B22046CDF828A00D950C950B951E
:102510001BF04AFC0AA906A816F0FAFEB4EEC80A97
:10252000F1EE10FA0DDD494ACDF800803B464849EE
:102530002046FFF79BFF002012B0BDEC028BBDE8E8
:10254000F0870AA906A803950495059516F0CAFE1A
:1025500003A90EA88DED0E0ACDED0F0A8DED101A10
:10256000CDED111A16F04CFCB9F1000F0DD09DED18
:10257000050AB0EEC00AB4EEE80AF1EE10FA04DD86
:10258000344ACDF800803B46D1E70136B4E700235A
:1025900094F8806216F0010001D0012BCCD104F533
:1025A000C0610AA8CDF828A00D950C950B9516F0E2
:1025B000DFFA0AA906A816F0ABFEDFED227AB4EE28
:1025C000E70AF1EE10FA05DD204ACDF800803B461F
:1025D0002149ADE72046FFF75BFC03282DD12046BB
:1025E0001BF034FC94F88032DB0728D438BB0AA9EE
:1025F00006A803950495059516F074FE03A90EA888
:102600008DED0E0ACDED0F0A8DED101ACDED111ADC
:1026100016F0F6FBB9F1000F11D09DED050ADFEDC4
:102620000A7AB0EEC00AB4EEE70AF1EE10FA06DD5F
:10263000084ACDF800803B46CAE70020D2E70120D7
:102640007AE700BFC2B8323EC2B8B23E4C1C09089D
:10265000571C0908E7D608085C1C09082DE9F74350
:102660001546044688460193FFF702FE019A074685
:1026700038B92848284B00682946C06A10F0C4FEC3
:10268000019A019229462046FFF70EFF064668B3DD
:102690002046FFF7FDFB94F93E12019A43B299429E
:1026A00007D01E4B1B4800682946C06A10F0ACFEDC
:1026B0001CE094F82433834207D0019205F0E8F837
:1026C00004F0E4FF019A0028EBD12046FFF7E0FB7D
:1026D00018B103280FD0124BE4E7134641462A46AF
:1026E00004F2544000F034FF00B107B90026304630
:1026F00003B0BDE8F08394F87892B9F1000F01D1EE
:10270000084BCFE7134641462A4620461BF06CF99A
:10271000EAE700BF105E0020601C09086C1C090875
:102720009C1C09088B1C090890F82433032B01D149
:102730001BF0DABB0020704713B540F6783200F585
:102740000971044601A810F065FC20461BF054FAFC
:1027500001A810F081FC02B010BD000008B50246CF
:10276000FFF796FB10B1032806D008BDBDE808406E
:1027700002F2544000F0ACBEBDE8084010461BF029
:10278000A9BB00000B4610B411462BB1032B09D096
:1027900000205DF8044B70475DF8044B00F2544094
:1027A00000F0A2BE5DF8044B1BF098BA13B50446C6
:1027B000FFF76EFB0A46014620460192FFF7E2FF53
:1027C00070B9084B019A1B68DB6A93F89C0038B11A
:1027D00094F82413204602B0BDE81040FFF7D2BFA2
:1027E00002B010BD105E002070B590F89432DB0787
:1027F00086B004460D460CD403F02CF9437C242209
:1028000002FB0300D0ED0B7AF1EE677AC5ED007A9A
:102810003BE002A803F05AFF01A92046FFF720FB86
:10282000E8B90CF041FF94F95032022B0646E3D18F
:10283000FEF7B4FE0228DFD996F8C4029FED147AA1
:10284000B02303FB0066D4F88832D6F8B0209B1A78
:1028500007EE903AF8EEE77A67EE877AD6E702A9B4
:102860002046FFF7A3FF0028DBD0D4F88822039B83
:10287000DFED076A9DED017A9B1A07EE903AF8EEBC
:10288000E77AA7EEE67A85ED007A06B070BD00BF64
:102890000AD7233CF0B50C4687B000F5097106460F
:1028A00040F6DD3201A810F0B5FBA36853B9E36828
:1028B00043B9636833B9002701A810F0CDFB38464F
:1028C00007B0F0BD204603F0EBFF0028F3D094E8FA
:1028D0000F0002AD85E80F000021284603F0A2FF9B
:1028E00007460028E7D096F89432DB0704D435F089
:1028F00065FE192135F09EFD95E80F0006F5217C57
:102900008CE80F0096F8943243F0010386F8943275
:10291000304600F073FD3FF0E5F946213FF0DCFD65
:102920003FF0E0F945213FF0D7FD084BA2681B6856
:10293000DB6A1A61E2685A6162689A6119F06AFE9C
:102940000028B9D017F08CFDB6E700BF105E00205C
:1029500038B5144B1B68DD6A2B6804465B68284653
:102960009847F0B12B690BB96A69D2B1C4F88C32BF
:102970006B69C4F89032A969002204F5217003F054
:10298000A9FE94F8943223F0030343F0030384F880
:1029900094323FF0A7F9BDE83840034A06213AF0E7
:1029A0006FB838BD105E0020B01C090813B504468E
:1029B0000193FFF76DFA0328019B05D1204602B071
:1029C000BDE810401BF01ABA002002B010BD000094
:1029D00010B588B004460593FFF75AFA0328059B03
:1029E0004FF000000AD10690079006A802900B98BD
:1029F00001900A98009020461BF00EFA08B010BD16
:102A000038B5044602F092FA0546D0B194F8243362
:102A1000032B03D095F84641204638BD20461BF0D5
:102A20001BF9FF280446F5D00146284602F054FA67
:102A30000028EFD02146284602F04AFA0028E9D0C3
:102A4000EAE70446E8E7000008B590F82433032BD2
:102A500005D013F07DFA90F90A03C0B208BD1BF04F
:102A60003FF8431CF9D1F4E708B590F8243383B15B
:102A7000032B03D1BDE808401BF02AB834F078F8E6
:102A800040F64C524FF4801134F02AF84FF0FF30EA
:102A900008BD1846FCE7000090F82433032B01D151
:102AA0001BF0E6BC7047000090F82433032B01D1E3
:102AB0001AF00EBF704700001AF06EBF10B5044642
:102AC0001DF05EFF2046FEF7E5FB2046BDE8104006
:102AD000FEF7FCBC90F824231AB1032A07D001208A
:102AE000704790F95002003818BF012070471BF062
:102AF000B9B9000030B590F840348BB00446002BD3
:102B000064D1B0F89036DB0660D590ED957ADFEDB4
:102B1000307AB0EEC77AB4EEE77AF1EE10FA11D55A
:102B200090ED967AB0EEC77AB4EEE77AF1EE10FA4D
:102B300008D590ED977AB0EEC77AB4EEE77AF1EE69
:102B400010FA43D42046FFF7C5FF00283ED1D4ED4C
:102B5000976ADFED207A9FED206A94ED967A0090D7
:102B600066EEA76AD4ED957A27EE067A67EE867A46
:102B7000FDEEE66ABDEEC77AFDEEE77A16EE903A14
:102B800017EE901A17EE102A06A803F0BDFD06A94D
:102B90002046FFF779F8C8B13FF0A4F80546D4F80D
:102BA0005C02F9F7A9FCCDE90401D4F85802F9F761
:102BB000A3FCCDE90201D4F85402F9F79DFC074AC1
:102BC000CDE900010621284639F05AFF0BB030BD8F
:102BD000000000340000C8428096184BC81C090849
:102BE00090F824330BB1032B01D11BF0ADBC0020B6
:102BF0007047000030B500F57B7304460D460FCBDF
:102C000085E80F0094F8FC0330BD0000D0F898333D
:102C10000B6090F894037047D0F8A0330B6090F8E5
:102C20009D03704710B500F5697203460C4607CA4C
:102C300084E8070093F8B00310BD000030B500F53C
:102C40006D7304460D460FCB85E80F0094F8C4035E
:102C500030BD000030B500F5866304460D460FCB4D
:102C600085E80F0094F8400430BD000010B500F274
:102C7000444203460C4607CA84E8070093F8500410
:102C800010BD00002DE9F0432DED028B8BB0054601
:102C90000E461746FFF7B4FE014680462846FFF76A
:102CA00041FB0446002848D002F040F9414602F0BA
:102CB00015F986ED000A95F93C32002B3ADD0CF04F
:102CC000F3FCFEF76BFC012834D90CF0EDFC90F816
:102CD000C432D5EDE47ADFED5D8A96ED000AB022CC
:102CE00002FB030095F93C32D0ED2F0A07EE103AB3
:102CF000F4EEE87AB8EEC77AF1EE10FAB7EE008A91
:102D0000B8BFF0EE487A37EE201A20EE270A70EEB0
:102D1000C70A40F20E4014F0A1FCD5EDE47AF4EEBF
:102D2000E87AF1EE10FAB8BFF0EE487A80EE277A32
:102D300086ED007A01233B7003E095F8203333B928
:102D4000387020460BB0BDEC028BBDE8F08395F8DF
:102D500024334FF00009CDF80490CDF80890CDF859
:102D60000C9043B1032B10D0CDF81090CDF81490F7
:102D7000CDF818907CB902233B703246414605F2EB
:102D8000544001F027FB0446DBE701A928461AF06E
:102D900057FF0446E8E795F82433002BEBD004A94D
:102DA0002846FFF763FF04460028E4D001A904A8E1
:102DB00016F0B4FC07A8CDED080A8DED091A8DEDCB
:102DC000070A17F0BFF804A8B0EE408A17F0BAF867
:102DD00095F93C32002B30DD07EE903AF8EEE77AB9
:102DE00040F2544070EE670A37EE801AF5EEC00AE2
:102DF000F1EE10FA48BFDFED160AF4EE410AF1EEEB
:102E000010FAB0EE480AC8BFB0EE601A14F026FC03
:102E1000B0EE408AD5EDE47A9FED0C7AF4EEC77AF5
:102E2000F1EE10FAB7EE007AB8BFF0EE477A88EE0E
:102E3000277A032386ED007A7DE7B5EEC08AF1EEAE
:102E400010FA48BF9FED028AE4E700BF000000349B
:102E50000000000038B50446FFF7F6FD94F826336D
:102E60008342054604D013F073F8294611F05EFF43
:102E70002046FFF7E9FD84F8265384F82503204611
:102E8000FFF7E2FD84F827032046FFF7EDFD04F588
:102E9000607184F828032046FEF746FE84F88C0310
:102EA00000F0CCFA04F5677284EDE40A04F566716B
:102EB0002046FFF7E7FE04F5687184F89403204686
:102EC000FEF74EFE04F5697184F89D032046FEF777
:102ED0007BFE04F56D7184F8B0032046FEF7B0FE6A
:102EE00004F5727184F8C4032046FFF79BF904F5DA
:102EF000767184F8D4032046FFF784F904F57B71DA
:102F000084F8E8032046FEF7E7FD04F5806184F8C5
:102F1000FC032046FFF756F984F810042046FEF71C
:102F200093FE04F2144004F5836380ED000AC3EDC0
:102F3000000A16F009FB04F21C4304F584612046E4
:102F400083ED000A04F22C42FFF732FA04F58661A1
:102F50002046FFF72BFC80B194F840349BB9012345
:102F600084F84034204600F049FA3EF0BBFE45218B
:102F70003FF0B2FA2046FEF7A3FE94F8403413B9AE
:102F80002046FFF7B7FD04F244412046FEF7E0FE7D
:102F900084F8500438BD000037B50D46044600F0F3
:102FA000E1F81DB912F0D4FF11F090FF4FF4EA726E
:102FB00004F5097101A810F02DF894F881322BB9AD
:102FC0002046FFF7C5FC012384F88132224B1D689F
:102FD000A86A03689B6998472046FEF7C1FC204613
:102FE000FEF73AFD204600F03BFA2046FFF704F8D2
:102FF000286B30B10368D4EDD80ADB6894EDD70AAA
:103000009847D4F81C0208B156F0E0FC204600F0C6
:1030100065F82046FEF74AFF94F8A83284F82403A6
:1030200083420ED084F8A80298B10C4D0C4B0328B3
:1030300008BF1D463EF056FE0A4A2B46062139F0CF
:103040001FFD2046FFF706FF01A810F005F803B0AA
:1030500030BD054DEEE700BF105E00205EEC0808B5
:10306000571C0908F41C09085C1C0908D0EDE47A17
:103070009FED057AF4EEC77AF1EE10FAB7EE000A8A
:10308000A8BFB0EE670A704700000034014B186813
:10309000704700BF305E002070470000704700009E
:1030A00070470000002070470020704701207047E3
:1030B00003681B6E1847000000207047002070470F
:1030C00000207047002070477047000000207047C4
:1030D00000207047002070477047000070470000D4
:1030E00008B512F035FF90F80A0308BD30B52DED94
:1030F000028B9FED1A1ADFED1A0A91ED000A87B0D4
:1031000005462D200C468DED011ACDED000A14F078
:10311000A5FA9DED011ADDED000AF0EE408A2E20A1
:1031200094ED010A14F09AFA9DED011ADDED000A02
:10313000B0EE408A2F2094ED020A14F08FFA03A912
:1031400005F52B70CDED038A8DED048A8DED050A12
:1031500031F0E0FE07B0BDEC028B30BDC2B8323EAC
:10316000C2B832BE10B5044655F0D8FCD4F80C33C2
:103170001BB1C21AB2F57A7F12D30A4A1268D26A18
:1031800092F89C2002B15BB9C4F80C0394F83D425C
:1031900012F0DEFE80F8054304F07AFB80F825404B
:1031A00010BD00BF105E00202DE9F0432DED028B15
:1031B00091ED007AD1ED037A87B08DED047AB0EE0F
:1031C000C77AB5EEC07AF1EE10FADDE91087DDF8C6
:1031D0004C90CDED057A0C4615461E4606DCF0EE09
:1031E000E77AF5EEC07AF1EE10FA02DD04A816F0E7
:1031F0001FFA6B20B7EE001AFFEE000A9DED050ADC
:1032000014F02CFA6C2089ED000AB7EE001AFFEEDC
:10321000000A9DED040A14F021FA04A888ED000AC2
:1032200016F06CF9B7EE008A002852D00023C9F8D6
:10323000003088ED008AD4ED067A67EEA77AF4EEC6
:10324000C87AF1EE10FA4ADB0023336085ED008A7C
:10325000DFED3F0A96ED000A7C20B7EE001A14F06D
:10326000FDF986ED000A95ED000A7D20B7EE001A03
:10327000FFEE000A14F0F2F985ED000AD4ED067AAB
:10328000129BDFED346AF1EE677AC3ED007A96EDBA
:10329000007AF0EEC77AF4EEE67AF1EE10FA2BD56A
:1032A00003AB02AA01A9204614F0F8FD9DED018AA6
:1032B000B0EE480A73F0EAFB85ED000AB0EE480A6A
:1032C00073F03AFD87ED000A07B0BDEC028BBDE854
:1032D000F08304A816F0FEF80028A7D1ABE738EE7B
:1032E000670A14F019F986ED000A94ED087AC7EE22
:1032F000007AC5ED007AABE794ED076AC6EE077A6F
:10330000C7ED007A96ED007AB0EEC77AB4EEE67AB1
:10331000F1EE10FAC4D495ED007ADFED0F6AB0EE4D
:10332000C76AB4EE666AF1EE10FAB9DCB4EE477A19
:10333000F1EE10FAB4D6B0EEE77AB4EE667AF1EEBA
:1033400010FAADDCF4EE677AF1EE10FABCD7A7E71D
:103350000000000000000034FFFF7F7F1FB500F574
:103360001D73039300F51C73029300F51B73019307
:1033700000F51A73009300F5187200F5197300F543
:103380004E71FFF711FF05B05DF804FB9FED196A60
:10339000D0ED846ADFED187A90ED860A66EE866AD3
:1033A00020EE060A26EEA77A10B5BDEEC77AC0ED6C
:1033B0007E6A80ED817A90ED857A27EE067A044662
:1033C00067EE275A60EE277AFDEEE55AFDEEE77AC2
:1033D000C0ED825A17EE903A002BBCBF03F50C43A8
:1033E000A033C0F80C3280ED7F7A14F0CDF884ED74
:1033F000800A10BDE02E65420000C8421FB50E4B8A
:103400001B680446B3B1684603F060F9694620467C
:10341000FFF720FC20B16A4600212046FEF720F885
:1034200094F89432DB0705D504F52172012120467A
:10343000FEF716F804B010BDD860002008B502F001
:1034400009FBBDE8084001F0E3BD000010B580F8BD
:103450001013044655F062FBC4F8140310BD0000BD
:1034600010B590F81033044653B155F057FBD4F81B
:103470001433C01AB0F57A7F84BF002384F8103368
:1034800094F8183353B155F049FBD4F81C33C01AE3
:10349000B0F57A7F84BF002384F8183310BD000094
:1034A00000F5AA700B4607C883E8070001207047A3
:1034B0000023C0F89C30C0F89830C0F89430C0F8B1
:1034C000A830C0F8A430C0F8A030C0F8AC307047C5
:1034D00070470000024B0B604FF07C531360704745
:1034E000000048427047000010B500F5B4700C466B
:1034F0000FC884E80F00204603F0DCF830B1FFF776
:10350000C5FD00F521700FC884E80F00204603F0C8
:10351000D1F880F00100C0B210BD000010B5044623
:1035200003F000FC204610BD10B5D0F86031044611
:103530005BB155F0F3FAD4F86031C01A41F2883328
:10354000984294BF0020012010BD0120FCE700003C
:1035500013B5009303680192DB6D9847DDE9002104
:10356000044628B90448054B0068C06A0FF04CFFB8
:10357000204602B010BD00BF105E0020601C09088C
:1035800013B50446019101F0D1FC2368019ADB6B6D
:10359000014608B190F84611204602B0BDE810403F
:1035A0001847000090ED007ADFED0F7AB0EEC77A91
:1035B000B4EEE77AF1EE10FA14D590ED017AB0EEA0
:1035C000C77AB4EEE77AF1EE10FA0BD590ED027AF5
:1035D000B0EEC77AB4EEE77AF1EE10FA4CBF0120F4
:1035E00000207047002070470000003410B501F043
:1035F0009DFC044658B190F8461101F069FC30B1C9
:1036000094F846112046BDE8104001F065BC00204A
:1036100010BD00002DE9F0432DED028B8FB0036843
:1036200000259B6B0395049505950695029502A9C7
:1036300004469847064638B1FFF700FFDDED027AF1
:1036400027EE800A8DED020A0CF02EF8FDF7A6FF9A
:103650000746002E50D0DDED027AD4ED646A94ED79
:10366000657A23680B9527EE877A67EEA67A8DED4B
:10367000097ACDED0A7A0C950D955B6B0BA9204666
:1036800009AD98470BA9284615F0A2FE012F8DED34
:10369000030ACDED040A40F2B3800CF005F890F86F
:1036A000C432DFED5B7AB02505FB030090ED308A74
:1036B00028EE278AB0EE480A73F0E8F9F0EE408A67
:1036C000B0EE480A73F038FBCDED0B8A8DED0C0A95
:1036D0000BF0EAFF90F8C43205FB030090ED2F0ACF
:1036E0000BA815F095FE09AD8DED050ACDED060A86
:1036F00005A896BB03C885E00128CED89DED020A37
:10370000B5EEC00AF1EE10FA7FDD07AED4F89421D1
:10371000D4F8903107923046089315F0A3FE236841
:103720000B950C950D955B6B0BA920469847DDED2D
:10373000077A9DED0B7A77EE877A9DED0C7ACDEDC9
:10374000077ADDED087A77EE877A09ABCDED087A56
:1037500096E8030083E8030049E0236993ED000A3B
:10376000B7EE008A38EE408A15F052FE04F5BC79B7
:103770008DED090A4846B0EE480ACDED0A0A15F06B
:1037800047FE0BA92846CDED0C0A8DED0B0A15F06E
:103790001FFE04F5C47603AFC4ED5F0A314684ED25
:1037A0005E0A384615F024FE04F5C0788DED090A4E
:1037B0004046B0EE480ACDED0A0A15F029FE0BA9E5
:1037C00028468DED0B0ACDED0C0A15F001FE97E8A9
:1037D000030084ED600AC4ED610A86E803004946EF
:1037E000404615F0F5FD8DED090ACDED0A0A9DED77
:1037F000090ADDED0A0A0FB0BDEC028BBDE8F083CB
:10380000DDE9030185E80300F1E709950A95EEE794
:1038100035FA8E3C10B590F84213044603F05EFC76
:103820007C23C0B203FB0044D4F8A00010BD00000C
:10383000044B026F1B68DB6A5A60426F9A60826FAA
:10384000DA607047105E0020F0B58FB0044612F0C9
:103850007FFB002302930393049390F80A1301ABB8
:1038600002AA054611F0A8FB04F19407D8B39DED18
:10387000010AB5EEC00AF1EE10FA34DD02A815F027
:1038800073FF04F1B00684ED2C0AC4ED2D0A84ED1B
:103890002E1A3946304615F077FF04F17C01304688
:1038A00015F026FF04F1880105A88DED050ACDED80
:1038B000060A8DED071A15F01BFF08A88DED080A02
:1038C0009DED010ACDED090A8DED0A1A15F03CFFB8
:1038D0000BA904F128008DED0B0ACDED0C0A8DED3E
:1038E0000D1A14F087FB95F80A030C2303FB005014
:1038F000394600F5117015F0FBFE84ED2C0AC4ED7D
:103900002D0A84ED2E1A0FB0F0BD00002DE9F0470E
:103910007E4B00251F682DED028BC0F89C50C0F82F
:103920009850C0F89450C0F88450C0F88050C567D3
:10393000C0F89050C0F88C50C0F88850C0F8B8500B
:10394000C0F8B450C0F8B0500446F86A03688AB0B2
:103950005B680E46984704F12809002854D055F0BA
:10396000DDF842F20F7398424ED8FB6A9FED688AE9
:1039700093ED010A84ED1C0AD3ED020AC4ED1D0A81
:1039800093ED031A484684ED1E1A14F027FA3EF010
:10399000A9F9D4ED1E7A67EE887A054617EE900AEB
:1039A000F8F7AAFDD4ED1D7A67EE887ACDE9040117
:1039B00017EE900AF8F7A0FDD4ED1C7A67EE887A2E
:1039C000CDE9020117EE900AF8F796FD514ACDE9CC
:1039D00000010621284639F053F894ED1E8AB0EE16
:1039E000480A73F053F884ED650AB0EE480A73F0A4
:1039F000A3F984ED640A55F091F8C4F864010AB0A3
:103A0000BDEC028BBDE8F087A6B194ED1C0AB4EEC4
:103A1000400AF1EE10FA0DD6D4ED1D0AF4EE600A5C
:103A2000F1EE10FA06D694ED1E1AB4EE411AF1EE3C
:103A300010FA67D712F08CFA90F80B334FF00C0A9B
:103A40000AFB030303F5C473074693E8070007AEB8
:103A500086E807004FF01508B2EE028AF2EE068AF9
:103A6000304616F06FFAB4EEC80AF1EE10FA11D52E
:103A700008F1FF3818F0FF0815D1304616F062FA49
:103A8000F1EE047AB4EEE70AF1EE10FA1CDC2567D9
:103A9000656731E0304616F055FAB4EEE80AF1EE0B
:103AA00010FAE5DCE9E7384611F044F9384611F040
:103AB0000DFA97F80B330AFB037303F5C47393E80D
:103AC000070086E80700CBE7DDED098A9DED088A4F
:103AD0009DED070A68EEA80AE8EE080AF1EEE00A92
:103AE00073F0F6F9F1EE680A84ED1D0AB1EE480AAA
:103AF00073F0EEF984ED1C0A9FED071AD4ED1D0A50
:103B000094ED1C0A484614F069F966E7105E00203F
:103B1000E02E6542681E0908000000000021FFF742
:103B2000F5BE000037B5044608461546019116F06B
:103B300009FAB7EE007AC7EE007AB4F8D0300198EF
:103B40000133A4F8D03094ED337A37EE277A84ED40
:103B5000337AB0EE007AF4EEC77AF1EE10FA06D5B9
:103B6000B6EE007AF4EEC77AF1EE10FA0DDC9FEDB6
:103B70000E7AF4EEC77AF1EE10FA13D59FED0B7AB8
:103B8000F4EEC77AF1EE10FA0CDDB0EE670A15F02C
:103B9000DBFD012085ED000AC5ED010A85ED021A65
:103BA00003B030BD0020FBE700247449BD378635E3
:103BB00070B52DED028B00F1280600F134058AB0B6
:103BC00029460446304615F03BFEB6EE008A20EE4C
:103BD000088A2846B0EE480A15F0B6FD07A9304617
:103BE000CDED080A8DED091A8DED070A15F096FD49
:103BF00030468DED010AB0EE480ACDED020A8DED9A
:103C0000031A15F0A1FD07A928468DED070ACDED91
:103C1000080A8DED091A15F081FD04A901A88DEDA2
:103C2000040ACDED050A8DED061A15F01DFE32468B
:103C300001A920468DED070ACDED080A8DED091A80
:103C4000FFF770FF58B954F069FF0121C4F8600113
:103C50002046FFF75BFE0AB0BDEC028B70BD2A4622
:103C600004A92046FFF75EFF0028ECD004F14002D3
:103C700007A92046FFF756FF0028E4D0EBE7000035
:103C800030B52DED028B0D4683B091F842130446FA
:103C9000284603F023FAC1B27C2000FB0151903189
:103CA00004F1280013F02AFF68468DED000ACDEDDF
:103CB000010A15F049FCDFED1C7AB4EEE70AF1EEDB
:103CC00010FA05D59FED190A03B0BDEC028B30BD8B
:103CD000684615F0ADFC684615F010FC0028F1D1DF
:103CE000284694ED428A03F061FBF0EE400AB0EE04
:103CF000480A13F0DDFB80B9284603F057FB84ED3A
:103D0000420AB0EE408A72F0C1FE84ED430AB0EE82
:103D1000480A73F011F884ED440A04F58671684688
:103D200015F0CAFBD0E700BF00000034000000001F
:103D30009FED0C7AB4EEC70AF1EE10FA0BD4DFED6A
:103D40000A7AB4EEE70AF1EE10FA07DCC0EE077A61
:103D5000B0EE670A7047F7EE007AF9E7F2EE047A00
:103D6000F6E700BFF3665F3F58A00B4108B51C3073
:103D700015F0EAFBF1EE007AB4EEE70AF1EE10FA84
:103D80009DBFF1EE027A37EEC00ADFED047A9FEDB7
:103D9000040A98BF20EE270A08BD00BFCDCC4C3ED8
:103DA000CDCCCC3D08B5836993F9000038B10BF058
:103DB0007BFCFDF7F3FB012894BF0020012008BD28
:103DC000F8B52DED028B054603F062FD03F05EFCB5
:103DD0000446B8B3FFF75AF990F8213393B3284655
:103DE000FFF7E0FF064668B30BF05EFC90F8C432C4
:103DF000B02707FB030090ED2F7AF0EE087AB4EEBF
:103E0000E77AF1EE10FA1DD495ED1E8A0BF04CFC0A
:103E100090F8C432DFED1E7A07FB030090ED300A04
:103E200098EE270A13F0C6FBDFED1A7AB0EEC00A4F
:103E3000B4EEE70AF1EE10FA08DC54F06FFE3446F7
:103E4000C5F85001BDEC028B2046F8BD05F5AA70FF
:103E500016F078F8B0EE408A0BF026FC90F8C432E9
:103E60009FED0D7A07FB0303D3ED2F7A67EE877A78
:103E7000B4EEE78AF1EE10FADFD554F04FFED5F834
:103E80005041001BB0F5FA6F8CBF00240124D9E724
:103E9000E02E654200003442CDCC4C3F10B50A4BB9
:103EA0001B68DB6A93F89C3004465BB954F036FE1D
:103EB000D4F86431C01A44F61F6398428CBF0020C6
:103EC000012010BD0020FCE7105E0020F8B52DEDAC
:103ED000068B04460BF0E8FB054603F0D9FC0646CA
:103EE00005F09EFD002840F0AA802046FFF768FFFD
:103EF000002800F0A7803046FFF78CFCD4F8DC30B7
:103F0000984200F018813046FFF784FCD4F8DC308A
:103F1000DFED8E7AC31A08EE903AF8EE688A3046E2
:103F200068EEA78AFFF776FC94F8BC30C4F8DC0092
:103F3000F3B9304603F0BCFBD0B104F1280796F882
:103F400042233946304603F035FAD4ED1D0AB0EE6F
:103F5000401A384694ED1C0A13F040FF0023C4F8C1
:103F60009030C4F88C30C4F88830012384F8BC3019
:103F700020463146FFF784FE95F8C40205EB001594
:103F8000B0EE408A2B6FC4F8E03004F1B000D4EDFD
:103F9000129A15F0D7FF6368DFED6D7A93ED007A22
:103FA000B4EEE77AF1EE10FA68EE299AB0EE40AA84
:103FB00001D5C3ED007A2046B0EE4A0AFFF7B8FEFD
:103FC000636820EE299A93ED000A29EE009AFFF724
:103FD000CDFE29EE009A204684ED249AFFF75EFF7D
:103FE00038B1D4ED247AB2EE007A67EE877AC4ED68
:103FF000247AF0EE007AF4EEE78AF1EE10FA10D5AA
:10400000DFED547AB4EEE7AAF1EE10FA09D5DFED50
:10401000527A69EEA79AD4ED2A7AE9EEA87AC4ED2D
:104020002A7A9FED4E0A94ED367ADFED4D7AB0EEA6
:10403000C88A28EE008AA7EE278A84ED368ABDEC6E
:10404000068BF8BDFFF722F890F82133002B72D0D1
:104050002046FFF7A7FE00286DD095F8C42205EB97
:104060000213196FD4F8E0308B4264D0B02606FBFF
:10407000025292ED2F7AF0EE087AB4EEE77AF1EE82
:1040800010FA58DBCB1AC4F8E01008EE903A95F815
:10409000C4329FED341A94ED1E0ADFED337A06FB2D
:1040A0000353D3ED309A69EE819AF8EE688A39EEBF
:1040B000C00A68EEA78A13F0BDFAB0EE409A72F01B
:1040C0003BFE94F8BC30B0EE408AF3B1F3EE047AD4
:1040D000F4EEE78AF1EE10FA17DC95F8C40206FB5D
:1040E000005595ED2F7AF2EE027AB4EEE77AF1EE12
:1040F00010FAFFF64AAFDFED1D7AB0EEC99AB4EEC2
:10410000E79AF1EE10FAFFF640AF9FED198AD4ED71
:104110001D0A94ED1C0AB0EE691A04F1280013F090
:104120005DFE012384ED248A84ED238A84ED228AB6
:1041300084F8BC3029E7BDEC068B04F188009FEDC4
:104140000D0ABDE8F84015F053BB00BFBD378635FA
:10415000CDCC4C3DC2B8B23E0AD7233CCDCC4C3E70
:10416000CDCC4C3F35FA8E3C6F12833A1904863F12
:1041700000000000EC51783F30B50C2303FB010137
:1041800001F1C003144693E807008BB004AD85E845
:10419000070094E8070083E807002846FFF702FAC3
:1041A00007AB58B194E8070083E807009DED070AC4
:1041B000DDED080A9DED091A0BB030BD95E807004A
:1041C000F2E70000F0B52DED028BD0F818318B60CE
:1041D000D0F81C31CB6085B004460D4601F03AFCA6
:1041E00006460BF061FAA36993F90030022B0746EB
:1041F0004BD1FDF7D3F9022847D997F8C432B02242
:1042000002FB0373D3F8B0100022284602F062FAD2
:10421000D4ED4A0A94ED490A284602F06FFD94F85D
:104220002C3163B354F07AFC9FED228A97F8C412C4
:104230008DED018A01AA064638460AF0B3FAD4F891
:1042400020019FED1D0A361A07EE906AF8EE677A94
:1042500040F23C4027EE800AB6EE001AF0EE480A23
:1042600013F0FCF9DDED017A30EE270A04F1F000DD
:104270008DED010A15F0CCF8284602F03FFD94F8C8
:104280002C0105B0BDEC028BF0BD707C242303FB38
:10429000006696ED0B8AFEF7F9FED0EDA27A9FED4F
:1042A000077AF8EEE77AE8EE077AFDEEE77A17EE9E
:1042B000901AA9E7000000006F12833A0000C8427C
:1042C00030B589B0044668460D4602F0FFF96946EC
:1042D0002046FFF709F918B90024204609B030BD7F
:1042E00004A802F0F3F9204604A9FFF76BFF044687
:1042F0000028F1D004A9684602F008FC85ED000A08
:10430000C5ED010A85ED021AE7E700001FB500239D
:104310000C4601A9019302930393FFF7D1FF08B163
:10432000039B236004B010BD30B585B001AD002300
:104330000C462946019302930393FFF7C1FF0346FE
:1043400018B195E8030084E80300184605B030BDB5
:10435000F8B52DED028B06460F46154600F0E6FD3A
:104360000446A0B1394600F0B3FD80B1204639467D
:1043700000F0B2FD044650B100F0D8FD394600F01F
:10438000ADFD85ED000ABDEC028B2046F8BDFEF7C1
:104390007DFE90F82033B7EE008A7BB13046FFF700
:1043A00001FD044650B1D6ED538AFFF747F8C8EE39
:1043B000007A67EEA87AC5ED007AE4E7D6ED538A75
:1043C000FFF73CF8C8EE007A002467EEA87AC5ED46
:1043D000007AD8E770B52DED048B1646FFF7B8FFCD
:1043E000054670B3FEF752FE90F93C424CB30BF019
:1043F0005BF9FDF7D3F8012823D9E4B207EE904A20
:10440000B8EE678A0BF050F990F8C43296ED009A36
:10441000B02202FB0300D0ED2F8AFFF70FF838EE31
:10442000281A78EEC80A40F2654029EE000A13F017
:1044300015F9B0EE408AFFF701F8C8EE007AC6ED34
:10444000007ABDEC048B284670BD000038B50D46DF
:104450000BF02AF90446FDF7A1F8022881BF94F871
:10446000C402B02303FB0040D43089BF07C800203A
:1044700085E80700012038BD30B585B000230D4622
:1044800001A9019302930393FFF7E0FF044620B1D3
:10449000039B2B60204605B030BD01F0DBFA417C68
:1044A00000F092FF04460028F4D001F0D3FA00F0A7
:1044B00051FEB1EE400A85ED000AEBE7F8B5036F57
:1044C0004B60436F8B60836FCB6000F14C070C46F1
:1044D000054601F110060FCF0FC60FCF0FC63B6880
:1044E000336005F1280104F1340014F041FB234648
:1044F000012203F8442B05F1B00207CA83E8070044
:1045000005F1940207CA04F1500383E8070005F19E
:104510001C0207CA04F15C0383E8070004F174017C
:104520002846FFF793FF04F1840184F880002846B1
:10453000FFF7A2FF04F18C0184F888002846FFF7FA
:1045400041FE84F89C00F8BD08B503F0A1F9BDE870
:10455000084003F09BB8000010B5044615F0A0F920
:1045600050B904F10C0015F09BF928B904F11800BA
:10457000BDE8104015F094B9012010BD38B500F128
:10458000280504462846FFF7E7FF28B12046012109
:10459000BDE83840FFF7BAB9D4ED107AB7EE007A2B
:1045A000F4EEC77AF1EE10FA06D5BFEE007AF4EE1B
:1045B000C77AF1EE10FA12DC2046FFF7F9FA284626
:1045C000FFF7CAFF0028E1D1D4ED107AB2EE047AE9
:1045D000F0EEE77AF4EEC77AF1EE10FAD6DC38BDE9
:1045E00010B5044615F0AEFC2046BDE8104015F0AD
:1045F00013B900002DE9F04F2DED048B9FEDCA8A11
:1046000095B00446F0EE408A8DED028A8DED038A66
:104610008DED048AFFF75AFC11F09AFC0023054641
:1046200095F87921012AA8BF012293423FD20021A7
:10463000284610F0E7FA01230028F1D008AB0BAAB6
:10464000002128468DED0B8A8DED0C8A8DED0D8AAB
:1046500010F00CFD9DED080AB5EEC00AF1EE10FA5F
:1046600023DD0BA815F080F811A904F128008DEDC9
:10467000110ACDED120A8DED131A13F0E3F90EA80D
:104680008DED0E0AB0EE680ACDED0F0A8DED101A11
:1046900015F05AF811A904F1E4008DED110ACDEDE1
:1046A000120A8DED131A15F06FF80123B8E795F88B
:1046B0000B130C2303FB015104F1280B01F5C4710A
:1046C000584613F0BFF984ED070A94ED3F0AC4ED94
:1046D000080A70EE288A84ED091AC4ED3F8A0AF0B0
:1046E000E3FF0646FEF7D2FC90F821330193204603
:1046F000FFF758FB80B13046FCF750FF02280BD97A
:1047000096F8C4226169B02303FB026391F900109B
:1047100093F8D200884263DA94ED3F7ADFED837A32
:10472000B4EEE77AF1EE10FA61D4D4ED538AFEF7D5
:104730005DFF58B100F0FAFB90F8461100F0CEFB97
:10474000F0EE408AFEF77AFE60EE288A236C626BF8
:10475000A16A1393B0EE680A11A81292119114F095
:10476000F3FF04F5AA7102A88DED020ACDED030A4C
:104770008DED041A15F008F854F0D0F9002307461F
:1047800084F814312046FFF70DFB002865D096F819
:10479000C422B02302FB033232445268C4F8182109
:1047A00096F8C42202FB033333449B68C4F81C31DF
:1047B00054F0B4F90123C4F8200184ED498A84ED52
:1047C0004A8A84F82C31D4F80031002B58D102AB3E
:1047D00093E80700C4F80071F03484E8070006E0AD
:1047E00006EB0212176FD4F80021BA4204D115B0BB
:1047F000BDEC048BBDE8F08FD43393E8070094F848
:1048000014310DF1080C8CE807001BB904F1F0031A
:1048100083E807000123604684F8143104F5AA7187
:1048200014F07CFF11A904F14C008DED110ACDEDBF
:10483000120A8DED131A13F033F9B5EEC00AF1EE3A
:1048400010FA8DED110AD8BF9FED370ACDED120A8F
:104850008DED131A84ED530A94E794ED3F7AD4ED6D
:10486000497ADDED026AE6EE877ADDED036AC4ED92
:10487000497AD4ED4A7AE7EE267AC4ED4A7AA2E77D
:10488000D4ED3F7A254B8DED058AF5EEC07AF1EE39
:1048900010FA8DED068A0793A9D9214B9FED217A55
:1048A0001B68DB6A67EE877A93F89CA0B7EE007A04
:1048B000C7EE279ABAF1000F4AD094F8143113B911
:1048C000019B002B42D0E36804F1F001D3ED008A94
:1048D00002A814F023FF69EEA88A8DED110A11A831
:1048E000B0EE680ACDED120A8DED131A14F02CFF0C
:1048F0000EA905A88DED0E0ACDED0F0A8DED101A4B
:1049000014F042FF05A8FFF76BFE05A814F0E2FFC4
:10491000F0B154F003F9C4F8600168E7000080BF0B
:10492000105E00200AE81C4100000000CDCC4C3E87
:10493000CDCC4C3FCDCC4C3D920A06BF920A063FEF
:10494000C2B8B23E728A0E3C5B821839DDF804A010
:104950005FED0B8A0023CDE90833CDE90A33CDE9B9
:104960000C334FF0FF32009204F1E40895F87921FE
:10497000012A1046A8BF0120834255D20123002AF4
:10498000FAD095F82D130029F6D0B0EE690A40460A
:1049900014F02EFF0DF12C09BAF1000F3FD0424662
:1049A00000212046FFF7E8FB8DED0B0ACDED0C0A48
:1049B0008DED0D1A4846FEF7F5FD70BB4846FFF732
:1049C0000FFE484614F086FF38BB05A9484614F090
:1049D0004BFF05A94846CDED090A8DED0A1A8DED6C
:1049E000080A14F02DFF08A8B0EE409A15F0AAFAB4
:1049F000009B33B9F4EEC08AF1EE10FAD8BFB0EEE6
:104A0000680AB5EEC09AF1EE10FAF7EE008A4FF0A0
:104A1000000358BFF0EE408A00930123A6E798E810
:104A2000070089E80700C5E7009B002B7FF471AF02
:104A3000002384F804312046FFF7C2F938B120463C
:104A4000FFF7B0F9002840F025818DED0A8A95F82E
:104A50000A3395F878219A4240F233812B4493F837
:104A60002C33002B00F02D8195F80B3395F879212C
:104A70009A4240F226812B4493F82D33002B00F00C
:104A8000208108A9584613F00BF88DED080ACDEDEA
:104A9000090A8DED0A1A08A814F002FF002840F058
:104AA000178108A814F016FF002840F011815FED6F
:104AB000617A94ED357A68EEA78A5FED637AE7EE66
:104AC000278A04F1B000C4ED358A15F03BFAA368DB
:104AD0005FED687A93ED007AB4EEE77AF1EE10FAC2
:104AE000F0EE408A00F1F8802046B0EE680AFFF749
:104AF0001FF908A814F028FEA3688DED110ACDED6A
:104B0000120A8DED131A93ED000A11A814F01CFE81
:104B1000204684ED1F0AC4ED200A84ED211AFFF718
:104B2000BDF928B1B2EE000A04F17C0014F060FE79
:104B3000019BB3B33046FCF731FD012831D996F81B
:104B4000C402B02303FB006696ED2F7AF0EE087ADC
:104B5000B4EEE77AF1EE10FA23D595F80B030C23A7
:104B600003FB005595ED627AF1EE0C7AB4EEE77A2C
:104B7000F1EE10FA15DBD4ED1D7A1FED917AF4EE0B
:104B8000C77AF1EE10FA0CDD1FED947AF4EEC77AD5
:104B9000F1EE10FA05D5B6EE000A04F17C0014F02F
:104BA00027FE5FED997AF4EEE78AF1EE10FA22D54E
:104BB0001FED9C0A08A814F0C7FD0EA88DED0E0A83
:104BC00094ED3F0ACDED0F0A8DED101A14F0BCFDE7
:104BD00011A904F1A0008DED110ACDED120A8DEDA1
:104BE000131A14F0D1FDD4ED2B7A94ED3F7A77EEC1
:104BF000877AC4ED2B7A94ED2B7AF1EE047AB4EE39
:104C0000E77AF1EE10FA3BDB11F0A2F95FEDB27A30
:104C100094ED2B1A94ED280A21EE271A40F2C930A0
:104C2000F1EE410A8DED011ACDED000A12F016FDEC
:104C30009DED011ADDED000A84ED280A40F2CA302C
:104C400094ED290A12F00AFD9DED011ADDED000A2E
:104C500084ED290A40F2CB3094ED2A0A12F0FEFCD2
:104C600004F1A00184ED2A0A04F1940014F08CFDF3
:104C700084ED2A8A84ED298A84ED288A84ED2B8AA2
:104C80000023C4F8E430C4F8E830C4F8EC3084ED14
:104C90003F8A9CE5E368F7EE000A93ED000A12F004
:104CA00007FC00283FF4D1AE94ED1C0AB0EEC00A18
:104CB00072F042F8DDED0A7A27EE800A8DED0A0ADD
:104CC000C5E68DED0A8A8DED098A8DED088AE2E64A
:104CD0002046FFF753FC1CE6C3ED007A04E700BF53
:104CE0002DE9F04D2DED0E8BA0B0044611F030F9FA
:104CF000D0EDC67A90ED618AF4EE487AF1EE10FAC2
:104D000048BFB0EE678ADFED677AB4EEE78AF1EE6E
:104D100010FA0EDD0023C4F8E430C4F8E830C4F81B
:104D2000EC300023C4F8FC3020B0BDEC0E8BBDE8A5
:104D3000F08D2046FEF788FD2046FEF739FFB0EEE5
:104D4000480A2046FFF756FC2046FFF717FCFEF7FF
:104D50009DF916AD00F53A7204F1280116A812F07B
:104D6000EFFE0FCD04F14C060FC60FCD0FC62B681A
:104D7000336004F1740204F1780304F1700104F16A
:104D80004C0013F08BF894ED1E8AB0EE480A71F0D7
:104D90007DFE84ED650AB0EE480A71F0CDFF204635
:104DA00084ED640AFEF744FDFEF770F904F5B47172
:104DB000FDF750FF53F0B2FED4F89831C31A632BBD
:104DC000B2D9C4F8980133F0F9FB9FED378A054654
:104DD00053F0ACFED4ED1C7A67EE887A074617EEE6
:104DE000900A0E46F7F788FBD4ED1D7A67EE887AB5
:104DF00041EC1D0B17EE900AF7F77EFB94ED1E0AAF
:104E000020EE080A41EC1C0B12F0BEFBD4F8D400D3
:104E100010EE108AF7F770FB8246D4F8D8008B4664
:104E2000F7F76AFB41EC180BD4F85401F7F764FB71
:104E300041EC190BD4F85801F7F75EFB41EC1A0B63
:104E4000D4F85C01F7F758FB94ED53EA41EC1B0BE7
:104E5000FEF7F4FACEEE007A17EE900AF7F74CFB65
:104E6000CDE9140140468DED12BB8DED10AB8DEDFB
:104E70000E9B8DED0C8BCDE90AABF7F73DFB0B4B91
:104E800001930B4B0093CDE908018DED06CB8DED21
:104E900004DBCDE90276074B074A0849284633F080
:104EA00015F941E7CDCC4C3EE02E65426DF7080880
:104EB000C3F70808941E09089F1E09085C1C09080E
:104EC00070470000002070477047000000207047C6
:104ED0000020704700207047002070479FED010AB6
:104EE000704700BF000000009FED010A704700BF3F
:104EF00000000000002070477047000010B5044615
:104F0000143000F019F804F12C0000F015F804F149
:104F1000700054F0EBFD04F1F00054F0E7FD4FF0A9
:104F2000FF33C4F84C31204610BD0000014B186817
:104F3000704700BF345E00207047000008B52DEDBB
:104F4000048BB0EE609AF0EE408A00F00FF9B0EEFC
:104F5000408A89EE280A72F025F8DFED0B7A20EE00
:104F6000270A71F0B7FFDFED097A38EE278ADFED07
:104F7000087A28EE278AF7EE007A37EEC00A28EE84
:104F8000000ABDEC048B08BD41D3423E33938843F5
:104F9000A1D81943FFF7D2BF08B52DED048B9FEDC3
:104FA000179AF0EEE07AF4EEC97AF1EE10FAF0EE2C
:104FB000408AB0EE608A04D5B7EE000ABDEC048BDF
:104FC00008BD00F0D3F8DFED0E7A9FED0E7ADFED2D
:104FD0000E6A70EE277A9FED0D0AE8EEC77A27EE8B
:104FE000800A88EE007AC6EE877AF4EEC97AF1EE8E
:104FF00010FAE1DBB1EEE70AE0E700BF00000034A1
:1050000033938843F4FDD43BCDCC9C3F48A18F43E0
:10501000427CD0ED257A242101FB020292ED0B0A9D
:10502000D2ED090A30EE270AFFF7B6BF38B52DEDED
:10503000088BDFED21AA9FED21AA9FED21BA05463D
:10504000B0EE409AF0EE609AB0EE408A1524013C32
:10505000A4B25CB3F0EE490A2846B0EE480AFFF766
:105060006DFFF0EE490A70EE698A284638EE2A0A8A
:10507000FFF764FFB0EEE87A70EE697AB4EECA7AB0
:10508000F1EE10FA77EEE87A10D468EEAA8A40F2D0
:10509000631088EEA70AB0EE4B1A38EE400AF0EE25
:1050A0004A0A12F0DBFAB0EE408AD0E7B0EE480AC6
:1050B000BDEC088B38BD00BFCDCCCC3D0AD7233C1E
:1050C00000247449002343608360C360036143612B
:1050D0008361C361002380F82030704790F820205E
:1050E000531CDBB2062B80F8203000EB820288BF15
:1050F000002382ED010A88BF80F82030704700004D
:105100004FF0FF3310B543610E4BC0F8A8300023B9
:10511000044680F8C830A830FFF7D4FF0A4BC4F823
:10512000A83004F5867052F061FE084B08491C60F7
:1051300020462FF005F8D4F89030C4F8943020467B
:1051400010BD00BFB8200908C8200908385E00203B
:105150006021090808B5A83034F060FADFED027A62
:1051600020EE270A08BD00BF00007A4490ED3C0AFB
:10517000DFED057AB0EEC07AB4EEE77AF1EE10FA20
:1051800048BF90ED3D0A70470000003473B5D0F879
:10519000A43004460E4663B153F0C0FCD4F8A430EA
:1051A000C01A42F20F73984203D894ED280A02B055
:1051B00070BD114B1D687DB195F846112846FFF76B
:1051C0008BFE48B195F8461101AA2846FFF77AFEF2
:1051D00010B19DED010AEAE7242101FB064494ED9C
:1051E0000A0ADFED067AB4EEE70AF1EE10FA58BFCC
:1051F000B0EE670ADBE700BF345E002000000C421F
:1052000008B561B10378022B02D9064853F058FC67
:105210005A1C027000EB83004160012008BD084663
:10522000FCE700BF801F09082DE9F84305460E463C
:105230009146002400F13C082B7CA34211DD0023A1
:105240004A46314601200DF061FD242363430746A1
:10525000002158F803000DF069FD874204D00134A5
:10526000EAE70020BDE8F8830120FBE770B50B46B4
:10527000064614469AB111469847054628B9236850
:1052800020465B68BDE87040184701463046FFF78E
:10529000B7FF20B92B6828465B689847EFE770BDD9
:1052A000F0B50D4685B011461A46CDE90213044605
:1052B000FFF7BAFF034698B90A4800684068042718
:1052C0000668CDE90037DDE902123668064BB047C3
:1052D00002462946204605B0BDE8F040FFF7C6BFAC
:1052E0000022F6E7105E0020801A06007FB5D0EDA0
:1052F000247A9FED2B7AF0EEE77AF4EEC77A012359
:10530000F1EE10FA0446037609D49030002303A985
:10531000019003932FF0B0FC01982FF0E9F80022E0
:1053200076232049E2632266C4F884202046FFF7F2
:10533000B7FF2378032B30D0237C032B2DD0D4F858
:105340000031DA0403D5637E0BB9012363760025AF
:10535000637EEB40DB07EAB20BD40135082DF7D1B1
:1053600023781BB1237C0BB16368B3B90E4801F0FD
:1053700095F93820019201F0CDFC064618B1019A4A
:10538000214654F0A3FC31462046FFF739FF23782D
:10539000032B02D0237C032BDFD104B070BD00BFF0
:1053A00000000034E99F06089C1F0908054B1B6894
:1053B0002BB141694A1C02D0184633F0C9B800200D
:1053C000704700BFD860002002290BD8242303FBBC
:1053D000010191F8390030B191F83A0018B191F813
:1053E0003B007047002070472DE9F047044653F01A
:1053F00095FBD4F8F86042F21073861B9E4288BF7A
:10540000C4F8F80000274FF0240942F2107A237CF8
:10541000FDB2AB421CD929462046FFF7D5FF70B13B
:1054200009FB054898ED0D0AD8ED097AD4ED250A57
:1054300030EE270A2046FFF7F9FD88ED0C0A5645A5
:1054400004D909FB054030302FF052F80137DEE770
:10545000617C2046FFF79AFE84ED3D0ABDE8F087A7
:1054600070B52DED028B044686B053F057FBD4F88F
:105470009830C31AB3F57A7F05463FD33C4B94ED81
:10548000257A1B689FED3B8ADB6AD4ED247A93F87A
:105490009C60F0EEC76AF4EEC86AF1EE10FA22D50D
:1054A000F0EEE76AF4EEC86AF1EE10FA1BD502A836
:1054B00001F00CF916BBFDF7E9FD02A9FDF7CAFBE7
:1054C000E0B1DDED037A9FED2C7AF8EEE77A67EE36
:1054D000877AB0EEE77AB4EEC87AF1EE10FA11D41A
:1054E000C4ED257A11E077EE676AB7EE006AF0EE58
:1054F000E66AF4EEC66AF1EE10FA1EDC06B0BDEC08
:10550000028B70BD1D4BC4F89430C4F89850FDF761
:10551000BDFDFDF711F92046FFF766FF3CF0E2FB09
:105520000546D4F89400F6F7E7FF154ACDE90001E7
:105530000621284637F0A4FAE0E7F0EEE76AF4EE39
:10554000C86AF1EE10FAD9D4002EC9D020469030A6
:1055500080ED007A2EF0CCFF3CF0C4FB094A01211B
:1055600006B0BDEC028BBDE8704037F089BA00BFD1
:10557000105E0020000000340AD7233C6F12833AEB
:10558000E51F0908C01F0908F0B52DED048B85B093
:10559000044640F2723200F5867103A80DF03AFD20
:1055A000D4ED227AD4ED236A9FED796A637C37EEDD
:1055B000E67A2422B0EEC77AB4EEC67AF1EE10FA9B
:1055C000C1BF9FED747A67EE877A9FED737AE6EE3E
:1055D000877A02FB03430025C4ED237A93F83960F0
:1055E0002378E9B28B4206D904EB81030135586870
:1055F00000F09EFAF4E7DFED698A9FED698A9FED7E
:10560000699A0027237CFDB2AB4264D9242303FBB3
:10561000054393F83920002A5BD0D3ED0C7AF4EEE1
:10562000E87AF1EE10FA0BDBF4EE677AF1EE10FA9D
:1056300006D6F0EEE77AF4EE487AF1EE10FA04DDE1
:10564000242303FB05435A6A1A63242303FB0543FF
:10565000D3ED090AD3ED0D7A93F8382070EEA70A3E
:10566000A2B993ED0C0A2046FFF794FCD4ED257AFD
:1056700030EE670AB4EE400AF1EE10FA16D7242392
:1056800003FB0545002385F83A3022E0012A09BFD3
:10569000D3ED0C7A93ED0B0A77EEE00AD4ED3B7A6A
:1056A00004BF80EE897A87EE270AE3E7F0EEC07A3E
:1056B000F4EE487A2423F1EE10FA03FB0545E1DC11
:1056C000012385F83A30D4ED237A37EE800A85ED50
:1056D0000B0A013796E7627C20461146FFF774FEFD
:1056E00048B1242101FB024292ED0B0AD16904F179
:1056F000A80033F073FF94F99C10277C002907DB86
:10570000B94205DACAB211462046FFF75DFE68B914
:1057100000226274D5B2AF4209D929462046FFF76C
:1057200053FE01320028F5D0657400E06274204613
:10573000FFF796FE2046FFF739FE10B1204654F0E1
:1057400051FA637C242505FB034393F83930B342B7
:1057500016D032F033FF4FF6FF7132F0F9FE78B118
:10576000607C05FB004494F83930002B14BF002204
:105770000422019232F022FF019A122132F07AFEC5
:1057800003A80DF069FC05B0BDEC048BF0BD00BFB3
:105790000AD7233C0AD7A33C48E17A3F00000034F3
:1057A000FFFF7F7F002019462DE9F04F0446007C63
:1057B0000F4687B004F13A0300220121D5B2A84276
:1057C00003F1240305D903F8231C03F8241C013238
:1057D000F4E76F4B1E68F06A03685B68984740B156
:1057E0003CF080FA6B4A062107B0BDE8F04F37F075
:1057F00047B93CF077FA684A062137F041F90023AF
:1058000003A904F1880003932FF036FA0A2553F018
:1058100085F980462046FFF7B7FE53F07FF9A0EBED
:105820000800B0F5FA7F02D95C4800F037FFB06A93
:1058300003680A215B689847617C2046FFF7C4FD36
:105840000028E7D0B06A036864215B68013D98478F
:1058500015F0FF05DBD1524B05951B888DF80650DE
:10586000CDE90355ADF80430052553F057F98046CE
:105870002046FFF789FE53F051F9A0EB0800B0F580
:10588000FA7FD1D8617C2046FFF79EFD0028EFD03B
:1058900094F810B00DF10C08A14601AA4FF0000ACF
:1058A0005FFA8AF18B4516D92046FFF78DFD50B17E
:1058B000D8ED007A99ED097A137877EE877A01337B
:1058C000C8ED007A13700AF1010A08F1040809F121
:1058D00024090132E4E7B06A036864215B68013D92
:1058E000984715F0FF05C0D1A9464FF02408237C46
:1058F0005FFA89F6B34226D906AB334413F8143C59
:1059000033B908FB064686F83B3009F10109EEE79A
:10591000002FFAD007EE903A06AA02EB8602F8EEC4
:10592000E77A12ED030AD4ED250A204680EE270A15
:10593000FFF77CFB08FB064002A930308DED020A20
:105940002FF09AF9E1E7617CDFF85C902046FFF7E1
:105950001DFC002684ED3D0A4FF02408237CF7B29D
:10596000BB420FD908FB074393F83B3043B13CF0EF
:10597000B9F97B1C4A46062137F082F80135EDB2B1
:105980000136EBE70DB907484FE707B0BDE8F08FE8
:10599000105E0020002009082B200908412009087A
:1059A00074D408087D2009085B20090808B5037C29
:1059B000022B02D9034853F083F85A1C027418468C
:1059C00008BD00BF9C20090838B5057C02460024AC
:1059D000E1B28D4206D91046FFF7F6FC01340028EB
:1059E000F6D138BD281E18BF0120FAE770B50D4664
:1059F00009780729044606D8027E437E22B901228F
:105A00008A401343437670BD002BFCD000262278D9
:105A1000F3B29A42F7D904EB830329465868036826
:105A2000DB6898470136F2E737B50D460192FFF77C
:105A3000CBFF0199044630B90448054B00682A465B
:105A4000C06A0DF0E1FC204603B030BD105E0020BE
:105A5000DF4B0A08014B1868704700BF385E002012
:105A60007047000073B543681B7C8B4205460C46AB
:105A700042D900F10801212201A80DF0CBFA53F020
:105A80004DF86A68242303FB0423D969411AB1F550
:105A9000FA7F33D2196A401AB0F5FA6F2ED2D3EDDD
:105AA000097A9FED177AF0EEE77AF4EEC77AF1EE15
:105AB00010FA54BF01200020242606FB04F31A44E8
:105AC0009FED107A82F8390069680B44D3ED0A7AA9
:105AD000F4EEC77AF1EE10FA06D49FED0B7AF4EEED
:105AE000C77AF1EE10FA04DD06FB0411002381F8F9
:105AF000393001A80DF0B0FA02B070BD0020DBE72C
:105B000000000034000048C30000484310B5044BB7
:105B10000446C0E90031083052F068F9204610BD53
:105B2000582209084368242000FB0131CA637047EA
:105B300013B50368019104469B689847236801994F
:105B40001B69204602B0BDE810401847F8B52DED9E
:105B5000028B43681B7C8B4205460C46F0EE408A64
:105B6000B0EE608A1FD952F0D9FF24276B686743D3
:105B70003B4493ED090AF0EE680A064611F098FCE2
:105B8000A0B96B68242202FB04331E626B682421D7
:105B90004C432344C3ED098A6B68234483ED0A8A8E
:105BA00069680C44E661BDEC028BF8BD6B683B4450
:105BB00093ED0A0AF0EE480A11F07AFC0028E0D0D2
:105BC000E4E70000DFED2A7AB0EEC07AB4EE677A3F
:105BD000F1EE10FA49DCB4EE400AF1EE10FA44D6C8
:105BE000436893F9FC3063B190ED087ADFED217AD8
:105BF000F0EEC76AF4EEE76AF1EE10FA03D580ED35
:105C0000080A01232BE077EE407A37EE006AF0EEC7
:105C1000E77AC7EE866ADBB29FED176A07EE903A25
:105C200026EE866AF8EE677AB4EEE76AF1EE10FACD
:105C30009FED126A15DDF2EE047A66EEA76A436AFA
:105C4000C6EE267A013343620023F7EE006A76EE51
:105C5000E76A27EE800AA7EE260A80ED080A1846B2
:105C60007047F0EE467A0123EFE70023F7E700BF25
:105C7000FFFF7F7F0000003400004843CDCCCC3DC7
:105C800090F83C35934207D900EB8200D0F8140518
:105C900010B103689B6A1847002070472DE9F34153
:105CA00005466E4686E80C00134B45F8043B044657
:105CB0000F4600F5C87828462C3500F017FCA8459B
:105CC000F9D196E8030004F5A863C4F8387583E8B1
:105CD0000300089BC4F84835084920462EF030FAE6
:105CE000074B1A6812B1074852F0EAFE20461C60C2
:105CF00002B0BDE8F08100BF40240908082309086C
:105D00003C5E00206C2209082DE9F04F90F83C65BC
:105D100085B00446002E55D17F2380F84C350DF117
:105D20000F01042328308DF80F302EF0E1FF04F529
:105D3000C87504F21458271D5FFA86F91822FF214E
:105D4000284673F083FA85F8589097F924A0BAF1A1
:105D50000A0F4DD039DCBAF1040F0FDCBAF1020F93
:105D60000FDD442000F0D6FF834620B13B462A4693
:105D7000214654F0F9FAC8F800B002E0BAF1090F70
:105D80002AD0D8F8000050B1296EC5F85CA031B116
:105D9000244B43F826102EF0E1FB2EF0D7FB58F8E9
:105DA000040B09F101095FFA89F920B103689B68C6
:105DB000984784F83C950136092E05F1640507F1F2
:105DC0002C07B9D105B0BDE8F08FBAF1190F1DD07D
:105DD000BAF11F0FC5D0D4E7382000F09BFF8346EF
:105DE0000028C8D03B462A46214654F035FFC2E77A
:105DF000302000F08FFF83460028BCD0CDF8009003
:105E00003B462A46214655F0C1F8B4E7482000F049
:105E100081FF83460028AED03B462A46214655F0F6
:105E200027F9A8E7405E002090F83C358B4283BFFD
:105E3000642303FB010090F8D501002070470000A7
:105E400090F83C358B4283BF642303FB010090ED47
:105E50006A0A9FED010A70470000000090F83C3587
:105E60008B4206D900EB8100D0F8140508B154F03C
:105E70002DBC9FED010A70470000000010B490F89F
:105E80003C458C420A4614D900EB8104D4F81445F1
:105E90007CB1E468246A640603D55DF8044BFFF71F
:105EA000DDBF642101FB020393ED6A0A5DF8044B38
:105EB00070479FED010AF9E70000000090F83C35BB
:105EC0008B420BD900EB8100D0F8140538B1C368C0
:105ED0001B6A1A4214BF012000207047002070473F
:105EE00070B590F83C35934204460E46154601D8ED
:105EF000002070BD00EB8203D3F814050028F7D012
:105F000003689B6998470028F2D0642202FB05448D
:105F1000D4F8AC313360ECE770B590F83C3593427F
:105F200004460E46154601D8002070BD00EB8203E2
:105F3000D3F814050028F7D003689B699847002818
:105F4000F2D0642202FB0544D4ED6C7AF4EE677A59
:105F5000F1EE10FAE8D6C6ED007AE6E770B590F8F3
:105F60003C35934204460E46154601D8002070BDCC
:105F700000EB8203D3F814050028F7D003685B69AF
:105F800098470028F2D0642202FB0544D4F8B431CB
:105F90003360ECE790F83C3593420ED900EB820376
:105FA000D3F814355BB1642303FB020292F8E401D9
:105FB00030B1D2F8E0310B607047002070471846CE
:105FC0007047000008299DBF2C2303FB0100406897
:105FD000002070472DE9F04F4B4B2DED028B1B68D5
:105FE000DB6A93F89C3089B00446002B00F0868071
:105FF000DFF82CB19FED458A4FF0000994F83C354D
:106000005FFA89F5AB4279D904EB8503D3F814051F
:1060100000285DD003685B6B9847642303FB05434E
:10602000074693F8D431834252D2032861D8DFE87F
:1060300000F04F025259364E4FF000083BF052FE2E
:1060400094F83C25AA4284BF642202FB05424FF02B
:10605000640105F1010301FB05458CBFD2F8A821BD
:1060600018EE102A8246D5F8B001CDE90632F6F7CF
:1060700043FA079ACDE904011046F6F73DFA069B6C
:106080000096CDE902015A460421504636F0F8FC4C
:106090000123204A84F84D3585F8D471D372D4F8A1
:1060A00048354BB3002255B25957481C03D04145DF
:1060B00002F10102F7D194F94C35AB4208DBD4F878
:1060C0004435D4F8400542463146984784F84C554B
:1060D00009F1010992E72C2303FB05430E4E93F9C6
:1060E0002B80ABE72C2303FB05430C4E93F92C804C
:1060F000A4E70026B046A1E71D46DCE709B0BDECE9
:10610000028BBDE8F08F00BF105E00200000000091
:1061100099220908BD5E0020C6570A089022090886
:10612000A822090890F83C358B4207D900EB810082
:10613000D0F8140510B10368DB69184700207047D8
:1061400008299CBF642303FB010000F5C870704759
:1061500090F83C35934207D900EB8200D0F8140543
:1061600010B103685B6A1847002070472DE9F04FB3
:10617000002493B005460E46174621462F2206A856
:10618000059405F2145973F061F805F1280A4FF0EF
:106190002C0B05F5F6730BFB04F259F8040B1AF9F6
:1061A0000210E5B230B951B90134092CF3D14FF0E6
:1061B000010813E0642262439A58914212D01548B4
:1061C000154B006801930135EDB20095134BC06A81
:1061D000324639460DF018F94FF00008404613B02A
:1061E000BDE8F08F05A93322039354F051FB039BC4
:1061F000804605A90028D7D1064801910135EDB2A6
:1062000000680095054BC06A324639460DF0FCF82F
:10621000E4E700BF105E0020152E0908D02209080F
:106220002DE9F04FDFF88090DFF880A0DFF880B034
:106230008DB00646002796F83C35FCB2A3422ED915
:10624000642505FB046595F8DC3133B395F8DD1161
:1062500019BB4FF001082022444404A889F8198092
:1062600072F0F4FF07EE904A4AF21043F8EEE77A34
:1062700003AA4C21ADF8283050462423CDED037AF3
:1062800036F010FA3BF02EFD9BF80030054A0094E2
:10629000042136F0F5FB85F8DD810137CBE70DB041
:1062A000BDE8F08FE0220908BD5E002059610020A2
:1062B000CD2200202DE9F04F2F4B1E6885B00446FB
:1062C00046B1D0F83815304632F042F910B13046B8
:1062D00030F0EAFF52F022FC4FF0000801904FF03E
:1062E0002C0A4FF0640B94F83C355FFA88F5AB420A
:1062F00039D904EB8507D7F8140588B30AFB0543A1
:106300000BFB054993F92820D9F8EC118A4227D1D3
:1063100032B30268D2689047D7F814050268126B4E
:10632000904799F8D52112B1019BC9F8D831BEB177
:10633000D4F83815304632F00BF988B152F0F6FB3C
:10634000CDE9021002460B46D7F81405294654F051
:1063500097FCDDE90232D7F81405294654F006FD12
:1063600008F10108BFE72046FFF734FE204605B0DC
:10637000BDE8F04FFFF754BFD86000202DE9F0478B
:106380004FF000082DED028B04468946B0EE408A9E
:10639000474601264FF0640A94F83C355FFA88F5C9
:1063A000AB421AD929FA05F3DB070AD504EB8503BA
:1063B000D3F8140578B10368B0EE480A9B6B984790
:1063C00006400AFB054508F1010895F8D4319F42C3
:1063D00038BF1F46E0E70646F3E727B97F23A4F856
:1063E0004C35034BDF72BDEC028B3046BDE8F087C5
:1063F000BD5E002090F83C358B4207D900EB810050
:10640000D0F8140510B10368DB6B18470020704703
:106410000B46114690F83C259A4207D900EB8300C1
:10642000D0F8140510B103681B6C184770470000C2
:1064300070B504460E46002594F83C35E9B28B420F
:1064400005D932462046FFF7E3FF0135F4E770BD7A
:106450002DE9F84390F83C550246002400F1280647
:106460002C2700F5F6784FF06409E1B28D420FD980
:1064700007FB04F309FB04F0F35658F800008342CD
:1064800009D11BB11046FFF7CFFC10B10134ECE786
:106490000120BDE8F8830020FBE7000010B590F86C
:1064A0003C258A42044617D9642202FB010393F873
:1064B000D431022B03D004D9032B18BF0023184674
:1064C00010BDFFF797FF48B92046FFF7C1FF00282E
:1064D0000CBF06230123F2E70023F0E70623EEE7D3
:1064E000014B1868704700BF3C5E002010B503499F
:1064F00004462DF025FE204610BD00BFC02409082B
:1065000010B50446203045F0A5F9044B04491C6041
:1065100020462DF015FE204610BD00BF645E002011
:1065200030260908F7B5B7EE000A0022022104461A
:106530002DF008FA204654F0EBFD45F079FA144BA3
:106540001D680646E86A03685B6A98470B460221A5
:1065500002460091304645F093F9B4F94A60002EA6
:1065600014DDEF6A3B6838465B68B4B2984728B1DF
:1065700097F84D3013B1C92EA8BFC824A86A036884
:106580005B68214603B0BDE8F040184703B0F0BD9A
:10659000105E002010B5044654F088FD2046BDE88A
:1065A000104054F0B3BD00002DE98048284BDFF8BF
:1065B000A490DFF8A4A0DFF8A4B01446012293B0A1
:1065C00005460E461A704FF0000852F0A7FAD9F8A7
:1065D00000300393A0EB080241F287339A4207464A
:1065E0001FD9CDE9005603985346342205A9C06A45
:1065F0000CF00AFF214605A8049451F075FCCDE982
:10660000005603985B46342205A9C06A0CF0FCFED4
:1066100004943BF067FB049B05AA022136F018FAAC
:10662000B8463BF05FFB3AF05BFC3BF05BFB3CF0B9
:106630009DFA0A2105A80CF0D3FC039B986A036815
:1066400005215B68984705A80CF0D6FCBDE700BFA4
:10665000685E0020105E0020B0250908256B0A083E
:106660000FB400B595B016AA002152F8043B03926E
:1066700005A83C220193049172F0E8FD054A019BB4
:10668000402104A851F0D8FB039A034804A9FFF75E
:106690008BFF00BFB8250908CE2509080FB407B540
:1066A00004AA034852F8041B0192FFF77DFF00BFC4
:1066B000E025090808B50449102272F06DFDB0FA12
:1066C00080F0400908BD00BF6C5E00201022002150
:1066D00072F0BCBD0378416023F00D03022A037001
:1066E00008D0032A0AD0012A03D1DBB243F0010308
:1066F00003707047037843F00803F9E7037823F049
:10670000050343F00503F3E773B504460E4615464B
:106710000193FFF7DBFF2046C4E90265069A019961
:10672000FFF7D8FF02B070BD4B6843600A7803786A
:1067300062F3000303700B780278C3F3800363F302
:10674000820202700B78D2B2C3F3C00363F3C302B8
:10675000027070470078420704D4030704D400F0A5
:10676000010070470320704702207047F0B585B0E4
:1067700005461646FFF7EEFF88420F4605D16B68C7
:1067800033600124204605B0F0BD032801D1002468
:10679000F8E70329FBD001280BD0022816D018BB3C
:1067A0006D68012F22D0022F2ED0002FEFD135603F
:1067B000E7E7FCF76BFC90F89432DB07E7D56D68F0
:1067C000FCF764FCD0F888321D44EAE76846FFF71E
:1067D0007DFFFCF75BFC6946FCF73CFA04460028A9
:1067E000D0D06D68019BEFE70025DAE7FCF74EFC9F
:1067F00090F8944214F00104C9D0FCF747FCD0F89B
:106800008832ED1A3560BDE76846FFF75FFFFCF799
:106810003DFC6946FCF71EFA04460028B2D0019BF5
:10682000EFE7000073B501AA05460E46FFF79EFF8D
:10683000044620B1019932462846FFF74BFF204617
:1068400002B070BD13B5144601AAFFF78FFF48B11F
:10685000DDED017A9FED047AF8EEE77A67EE877A4C
:10686000C4ED007A02B010BD0AD7233C07EE900AAF
:106870009FED090AF8EEE77A08B527EE800A70F076
:1068800005F9DFED067AB4EEE70AF1EE10FAD8BFAB
:10689000B0EE670A08BD00BF50E0EF300AD7233CD6
:1068A00010B50446806811F06BF820B1E068BDE8CF
:1068B000104011F079B810BD73B5856804460E46D6
:1068C0001DBBC36823B98B688360CB68C360012597
:1068D000636873B92378DB070BD52046FFF73AFFCF
:1068E00001AA01463046FFF741FF10B1019B6360EA
:1068F00005462046FFF7D4FF20B9B368A360F368CC
:10690000E3600125284602B070BD0025E0E70000E5
:106910000D4B83424FF000038B4106DA00F1255006
:1069200000F5311000F5E0507047084B98424FF0E9
:10693000FF3371EB0303BEBF00F1564000F51300B7
:1069400000F52440704700BF00D2496B002EB6947A
:1069500090EA010F01D4401A7047C317401A63EB45
:10696000E1710D4B83424FF000038B4106DA00F1D9
:10697000255000F5311000F5E0507047074B984264
:106980004FF0FF3371EB0303BEBF00F1564000F53B
:10699000130000F52440704700D2496B002EB694D6
:1069A00070B52DED028B84B0044668460D46FFF7A6
:1069B0008DFEFCF76BFB6946FCF74CF9064608B305
:1069C000A368029ADFED128A03999B1A07EE903AA8
:1069D000F8EEE77A67EEA87AC5ED007AE068FFF78F
:1069E000B7FF08EE100AA068024402EBD272B8EEBC
:1069F000C88A5010FFF73AFF28EE288A28EE000ACE
:106A000085ED010A304604B0BDEC028B70BD00BFBD
:106A1000F67C8E3F37B500230C4601AA02210546BD
:106A20000193FFF7A3FE10B9002003B030BD21464B
:106A30002846FFF7B5FF0028F6D0DDED017AF8EE25
:106A4000E77AC4ED027AF0E710B52DED028B846889
:106A50008A680B46111B08EE901AC168D868FFF7C8
:106A600077FF224402EBD27208EE100A5010FFF7B3
:106A7000FDFEB8EEC88AF8EEE88A28EE000A20EE9D
:106A8000000AA8EEA80ABDEC028BB1EEC07A9FED19
:106A9000020A27EE000A10BD8262363CF0B52DEDE9
:106AA000028B0D4689B08C680646D0E90271E86811
:106AB000FFF74EFF08EE100AE01900EBD07040100F
:106AC000FFF7D4FE73686A689FED0E1A9B1A07EEF3
:106AD000903AE41BB8EEE77AF0EE400A07EE904AEF
:106AE0009FED090AB8EEC88AF8EEE77A28EE008A28
:106AF00027EE011A27EE800A68EE200A09B0BDECE5
:106B0000028BF0BD0AD7233C8262363C84B004B0CD
:106B1000FFF7C4BF38B52DED028B0C460246C168A5
:106B2000E068FFF715FF9568A46808EE100A601981
:106B300000EBD0704010641BFFF798FE07EE904A00
:106B4000F8EEE77AF8EEC80A87EE807ABDEEC70A5B
:106B500010EE103A5B4200EE103AB8EEC00A70F048
:106B6000B7F9DFED087A30EE270ABDEC028BB5EEFF
:106B7000C00AF1EE10FA44BFDFED037A30EE270AC7
:106B800038BD00BFDB0FC93FDB0FC94030B52DED6D
:106B9000028B0B4685B08C68D0E90251D868FFF7AC
:106BA000D7FE08EE100A601900EBD0704010FFF716
:106BB0005DFE641B07EE904AF0EE400AB8EEC88A0C
:106BC0009FED060AF8EEE77A28EE008A27EE800AA3
:106BD00068EE200A05B0BDEC028B30BD8262363C07
:106BE00082B002B0FFF7D2BFF0B52DED028B0B469D
:106BF0008F68D0E9025185B0D868FFF7A9FE7B19EC
:106C000003EBD37304465810FFF730FE781B10EEE9
:106C1000106AF5F75FFC14A3D3E90023F5F7C4FC71
:106C2000F5F7BAFF08EE100A2046F5F753FC0EA35D
:106C3000D3E90023F5F7B8FC044630460D46F5F7D6
:106C40005BFC02460B4620462946F5F7ADFCF5F7FE
:106C5000A3FF00EE900AB0EE480A05B0BDEC028B2F
:106C6000F0BD00BFAFF300800000004050CC863F75
:106C7000094B984206DDC0F1D64000F5930000F5BF
:106C8000A4407047054B9842BEBFC0F1144000F5C8
:106C9000360000F53850704700E9A43500175BCA8C
:106CA000F8B52DED028BDFED148A076820EE280A77
:106CB0000646FDEEC07A0D4617EE904A04EBD470FE
:106CC00007EB6000B0EE608AFFF7D0FD28EE288A5F
:106CD0003819C8EE007AFFF7CBFF306017EE900A44
:106CE000F6F734F92B68C01841EBE371FFF710FE9B
:106CF000BDEC028B2860F8BD02AAB34200F10C0182
:106D00000830FFF7CDBF00000148FFF7DFBC00BF30
:106D10006C5E00200121884238BF08466DF08ABFB2
:106D2000FFF7F8BF08B16DF089BF7047FFF7FABFF2
:106D3000F8B506460F46144622B96DF07FFF25468A
:106D40002846F8BD10461EB9BDE8F8406DF042BFB8
:106D50006DF040FF05460028F2D0BC422246314685
:106D600028BF3A4672F028FA30466DF067FFE7E731
:106D700037B504460846089D11461A460368019532
:106D80009DF81C5000951D68069BA8472060204672
:106D900003B030BD00214FF0FF3310B50022036374
:106DA000044601600171C0F80510417280F8251099
:106DB00000F13C0300F50B70D9709A60DA601A613B
:106DC0005A619A61DA611A625A629A62DA631A64E3
:106DD0005A649A64DA641A655A659A65DA65DA66FD
:106DE0001A675A677C339842E6D1214604F516703B
:106DF00006F0FCFD044B1A6822B904491C602046C9
:106E00002DF09EF9204610BD7C5E002088280908E0
:106E100073B5D0F83C3201919942044613D0D0F8B2
:106E20004032994218D0D0F844328B4216D1022019
:106E30000AE0D4F8343253B3D4F838324BB34FF0BD
:106E4000030002B070BD002094F822308342F8D8CD
:106E5000431C84F82230F4E70120F5E7D0F83062D3
:106E6000002EE6D194F841233546B6009AB1A31915
:106E7000C3F83012A319019AC3F83C2294F82230C7
:106E8000AB429CBF6B1C84F822302846D9E7012610
:106E9000E8E70226E6E704F50C7001A930442DF07E
:106EA000F9FFE7E738B504460D462DF069FF291DC7
:106EB000201D2DF065FF05F1080104F108002EF0FA
:106EC00039F805F1140104F114002EF033F805F13E
:106ED000200104F120002EF02DF805F12C0104F121
:106EE0002C002DF0E1FE05F1300104F130002DF011
:106EF000E9FF05F13C0104F13C002EF01BF8AB6BFF
:106F0000A3636B6B636338BD2DE9F043A1B000232D
:106F1000002500F13C0706468DF8075003930493C3
:106F2000059306930793089309930A930B93109381
:106F30001193129313931493159316931793189315
:106F40001C931D931E9300F50F78B94658F8043B27
:106F5000F3B1F26E934223D0D6F8E820934221D0C9
:106F6000D6F86421934213D10221EBB299420FD09B
:106F7000C1EB411109EB8104214601A8FFF792FF03
:106F800039462046FFF78EFF01A93846FFF78AFFF2
:106F90000135032D07F17C07D8D121B0BDE8F0837E
:106FA0000021E2E70121E0E72DE9F04704460E4623
:106FB0001546804607464FF0000A31462046FFF747
:106FC00027FF7A6FB2425FFA8AF90ED1C3B2022B61
:106FD0000BD87C2202FB0A44012084F83E0084F88E
:106FE0003F3085F80090BDE8F0870AF1010ABAF158
:106FF000030F07F17C07E0D1002731462046FFF759
:1070000007FFD8F86C205FFA87F912B9C3B2022BD8
:1070100019D90137032F08F17C08EED131462046FB
:10702000FFF7F6FEC2B2C2EB421304EB830393F800
:107030003E7067B9022A0BD8012083F83E0083F81E
:107040003F202A70CFE77C2000FB0744C4E70027DD
:107050004FF07C0904F13E0A31462046FFF7D8FE86
:10706000034609FB07F05FFA87F81AF8002012B907
:10707000DBB2022B09D90137032FEDD194F823009D
:1070800004280BD9144851F01BFD0444012084F856
:107090003E0084F83F3085F80080A4E704F543778C
:1070A000002157F8043BB342CAB208D1904202D83B
:1070B000531C84F8233003322A70002093E73BB935
:1070C000411C04EB800084F82310C0F80C63F2E745
:1070D00001310529E5D1F0E7C0260908C9B200EB66
:1070E0008101D1F83C3253B1026F93420AD0D0F8FB
:1070F000EC20934208D0D0F86821934206D04FF09C
:10710000030070470020704701207047022070473D
:107110002DE9F8430F469146044600F5BA7894F8F5
:107120003E5035B97C344445F9D100252846BDE8A8
:10713000F88300234A46394601200BF0E7FD002181
:107140000646E06E0BF0F2FD8642EBD1EEE7000062
:10715000012303FA01F1D0F8083319420AD14AB1E8
:1071600090F82030032B1FBF591C80F8201000EB33
:1071700083004261704700002DE9F043DFF87C8016
:1071800085B0044600F50F7600257C27B14656F8F9
:107190000C3CD9F800209342E9B206F1040619D15B
:1071A000C3B12046FFF79AFFC0B207FB004090F83A
:1071B0003E307BB903A9A9F10C0003932DF06AFEC0
:1071C0003AF090FD56F8043C009342462B460121CC
:1071D00035F056FC0135032DD8D104F16C0504F5CA
:1071E000F074296821B9AB6813B128462CF0A4F8D3
:1071F0007C35A542F5D105B0BDE8F083DC26090851
:1072000038B504461546FFF769FFC0B2022808D812
:107210007C2303FB004029465030BDE838402DF068
:1072200079BE38BD38B504461546FFF757FFC0B2E2
:10723000022808D87C2303FB004029465C30BDE8C7
:1072400038402DF067BE38BD37B50D4604468DED8C
:10725000010AFFF743FF022D07D8C0B27C2303FBCE
:10726000004001A968302DF007FD03B030BD0000DB
:1072700038B50546FFF732FFC4B2022C13D8C4EB71
:107280004414A4003C3504F10800284400212CF0EB
:1072900053F804F1340104F1300029442844BDE8D6
:1072A00038402DF0F7BD38BD70B505460E46144682
:1072B000FFF714FFC3B2022B0DD87C2000FB035351
:1072C00094E80700443383E8070031462846BDE8C8
:1072D0007040FFF7CDBF70BD37B504461546FFF7C8
:1072E000FDFEC0B2022809D87C2303FB00400DF14B
:1072F000070140308DF807502DF042FD03B030BD3E
:107300001FB590F92C30044623B390F921300BB30C
:107310006846FFF7DBF9FBF7B9FE6946FBF76AFC45
:10732000C0B1DDED037A9FED0C0AF8EEE70ADDED62
:10733000027AF8EEE77A0123C0EE800A84F83D3342
:1073400087EE800A06F0A4FDDFED047A20EE270A1E
:1073500084ED0A0A04B010BD8096184B35FA8E3CB5
:10736000024690F9210058B192F8400340B111440F
:1073700091F92C0220B192F92400033818BF0120A2
:107380007047000038B590F8223005465BB1002404
:107390002346E1B22846FFF7E3FF08B10133DBB231
:1073A0000134032CF5D1184638BD000090ED0A0ACF
:1073B0007047000038B50C46D1ED066A1146054607
:1073C000FFF78CFEC3B27C2000FB0353D4ED087A98
:1073D000D3ED260A94ED076AD3ED255A93ED245A8E
:1073E00026EE600A67EEA00AA5EEA70AF0EE607A24
:1073F000E5EE867AB7EE007AA6EEE67A67EEE60A62
:10740000B1EE400AE5EE070A6FF062FD9FED071A44
:10741000DFED070A40F6580010F020F9D5ED0A7AA2
:10742000BDE8384030EE270A10F004B9DB0F4940C0
:10743000DB0F49C02DE9F04190F822308B42044621
:107440000D4602D20020BDE8F081FFF747FEC0B232
:1074500004F13C06C0EB401006EB8000083012F04F
:1074600071FDDFED157AB0EEC00AB4EEE70AF1EE79
:1074700010FAE7D429462046FFF730FEC5B27C203B
:1074800000FB05473B6F002BDCD0032DDAD000FB5F
:1074900005603030D7F86C802CF028FFD7E91B321C
:1074A000934201D1984505D07C2000FB0544C4F8E7
:1074B0006C80C7E70120C6E7000000342DE9F74FD4
:1074C00004460E46174600F50F7A4FF0000B5AF8A7
:1074D000049B5FFA8BF8B9F1000F26D04146204695
:1074E000FFF73EFF08B341462046FFF7F7FD7C2338
:1074F000C0B203FB004090F83E505DB908F10103B3
:107500001B4ADBB23946304650F096FC284603B0A1
:10751000BDE8F08F5AF8102C914506D0154A39462F
:10752000304650F089FC0025F0E70BF1010BBBF170
:10753000030FCCD14FF0000894F822305FFA88F1A5
:107540008B420DD920460191FFF774FF054620B903
:1075500001992046FFF704FF20B908F10108EBE785
:107560000125D3E7044A3946304650F065FCCDE7A3
:1075700004270908192709083E2709082DE9F041C1
:107580002DED048B90F842139FED348ADFED348AA1
:107590009FED349A82B00646FFF7A0FD06F13C0746
:1075A000C5B27C2000FB057554354FF0000896F8F5
:1075B00022205FFA88F39A424ED919463046FFF7E7
:1075C000CFFE10B908F10108F1E719463046FFF780
:1075D00085FDC4B27C2000FB0474D4ED157AF0EE76
:1075E000E77AF4EEC87AF1EE10FA04F154040ED5FD
:1075F000D4ED017AF0EEE77AF4EEC87AF1EE10FA03
:1076000005D5002002B0BDEC048BBDE8F081294611
:10761000204612F0A7FCB4EEE80AF1EE10FAF0DC16
:107620002946204611F09CFFB4EEC90AF1EE10FA8B
:10763000E7DC2146284611F0DBFE68468DED000AA6
:10764000CDED010A11F080FFDFED077AB4EEE70A15
:10765000F1EE10FAB6DDD4E70120D3E700000034E4
:10766000DB0FC93F920A863F00004843022910B54C
:10767000044608D8FFF732FD7C23C0B203FB004468
:1076800094F83D0010BD0020FCE7000013B590F811
:10769000421301910446FFF7E9FF30B101992046FA
:1076A00002B0BDE81040FFF75BBE02B010BD0000A5
:1076B000F7B590F921500446002D73D090F840534F
:1076C000002D6FD090F84213FFF7D0FF94F83D33B0
:1076D000064613B92046FFF713FE002594F8202034
:1076E000EBB29A4207D904EB83030135586903686A
:1076F0009B689847F2E751F011FA0027224604F5FB
:10770000BA7140F2F315D2F89C30C31AAB428CBF69
:107710000023012382F83D307C32914247EA03077F
:10772000F1D194F92430032B07D194F83C33002B8A
:107730003BD0D4F83803002849D167B1236B01331B
:1077400009D030F03BFF216B30F002FF18B130F070
:1077500035FF2FF0BDFE94F92C32002B3AD194F96D
:107760002D32CBBB94F92E3213B1022384F842336D
:1077700094F842132046FFF779FF8642054611D060
:1077800030F01CFF4FF6FF7130F0E2FE50B1002DDB
:1077900014BF00220422019230F010FF019A03214D
:1077A00030F068FE284603B0F0BD012384F83C3376
:1077B0000420FFF7AFFA054610B1214606F0B6F9EE
:1077C00094F92430C4F83853032BB2D0B5E706F04F
:1077D000C7F9B2E70023C9E70123C7E738B590F935
:1077E00021300446D3B190F84053BDB1FFF776FC89
:1077F000C0B2022812D87C2303FB0044D4ED1A7ACD
:107800009FED087AF4EEC77AF1EE10FA06D4B7EEDF
:10781000087AF4EEC77AF1EE10FA00DD002528466A
:1078200038BD00BFABAA2A3F70B5D0F8085315F495
:10783000003504460E460DD190F840335BB90A7806
:10784000072A07D8012303FA02F290F83F331343C3
:1078500080F83F3370BD94F82020EBB29A42F9D9FA
:1078600004EB8303314658690368DB6898470135A8
:10787000F1E7000038B505466C242B591BB10021F7
:1078800028192BF059FD7C34B4F5F07FF5D138BDC3
:10789000014B1868704700BF7C5E002010B504469D
:1078A000006810B103685B689847204610BD00006F
:1078B00010B50446006810B103685B68984720461D
:1078C00010BD00002DE9F04FD0F808538DB015F42D
:1078D000807B9DF858909DF85CA004460F461646A4
:1078E000984660D1FFF714FC054600283FD0CDE94B
:1078F00006BB069B04934FF0000B424639462046D8
:10790000CDE905BBFFF704FC064600283DD0CDE9D4
:107910000ABB0A9A089200234A4608A9CDE909330E
:1079200004A8534600F042FF074608A8FFF7C0FF2F
:1079300009A8FFF7BDFF0AA8FFF7B0FF16B10BA813
:10794000FFF7ACFF04A8FFF7B3FF05A8FFF7B0FFF0
:1079500006A8FFF7A3FF15B107A8FFF79FFF3A4658
:10796000082120460DB0BDE8F04FFFF7F1BB04231E
:107970000E49CDE9010309680D4B00934968334670
:107980003A4606A8FFF7F4F9B3E704230749CDE91F
:1079900001030968064B0093496843463A460AA822
:1079A000FFF7E6F9B5E70DB0BDE8F08F105E0020F7
:1079B000801A06002DE9F04F91460124D0F80823E3
:1079C0008BB08C40144098469DF854A09DF85030E0
:1079D0009DF858B006460F4635D11A4641460593E4
:1079E000FFF796FB059B054600B3CDE90844089ACE
:1079F000069200235A46514606A8CDE90733C847E8
:107A0000044606A8FFF754FF07A8FFF751FF08A890
:107A1000FFF744FF15B109A8FFF740FF224639469A
:107A200030460BB0BDE8F04FFFF792BB0422074988
:107A3000CDE901020968064A00924968424608A851
:107A4000FFF796F9D3E70BB0BDE8F08F105E00208A
:107A5000801A06002DE9F04FB04BDFF8CC921D687C
:107A600004466868036889B09B6898470026074603
:107A70004FF001084FF0080A08FA06F33B4240F0C5
:107A80002D820136202EF7D16868DFF89CA20368AA
:107A9000DB689847002607464FF001094FF00608BB
:107AA00009FA06F33B4240F02B820136202EF7D133
:107AB0006868DFF8789203689B6898470026074655
:107AC0004FF001084FF0080A08FA06F33B4240F075
:107AD00028820136202EF7D1686803689B68984792
:107AE0000026804601274FF01A0907FA06F313EA29
:107AF000080F40F026820136202EF6D16868036810
:107B0000DB689847002607464FF0010A4FF01A0934
:107B1000B0460AFA06F33B4240F02E820136202E90
:107B2000F7D16868DFF808920368DB689847002699
:107B300007464FF0010AB0460AFA06F33B4240F00E
:107B400036820136202EF7D16868DFF8E4910368A9
:107B5000DB689847002607464FF0010AB0460AFA4C
:107B600006F33B4240F033820136202EF7D168689D
:107B7000DFF8BC9103689B689847002607464FF0E2
:107B800001084FF0020A08FA06F33B4240F02F8248
:107B90000136202EF7D16868DFF8949103689B685E
:107BA0009847002607464FF001084FF0020A08FAEE
:107BB00006F33B4240F02B820136202EF7D1686855
:107BC000DFF8709103689B689847002607464FF0DE
:107BD00001084FF0060A08FA06F33B4240F02E82F5
:107BE0000136202EF7D16868DFF848910368DB681A
:107BF0009847002607464FF0010AB0460AFA06F3F6
:107C00003B4240F02B820136202EF7D1444BDFF867
:107C10002891079307AF04264FF00C0A68680368A1
:107C20009B6898474FF0000805904FF0010B059AAC
:107C30000BFA08F3134240F0218208F10108B8F171
:107C4000200FF4D168680368DB6898474FF000089C
:107C500005904FF0010B059A0BFA08F3134240F020
:107C60001E8208F10108B8F1200FF4D1013E16F090
:107C7000FF0607F10107D1D16868DFF8C0A00368EB
:107C80009B6898474FF001080746B14608FA06F38B
:107C90003B4240F017820136202EF7D16868DFF8AA
:107CA0009CA00368DB689847002607464FF001094F
:107CB000B04609FA06F33B4240F014820136202E0A
:107CC000F7D16868DFF878A003689B6898470026BA
:107CD00007464FF00108B14608FA06F33B4240F070
:107CE00011820136202EF7D16868DFF854A00368AE
:107CF000DB689847002607464FF00109B04609FAAD
:107D000006F33B4240F00E820136202EF7D1686820
:107D1000044B079303689B68984713E0105E0020AC
:107D20000C0D0E0F202122239DAA0108BDBA0108C7
:107D30001DB2010839870108E9AF010801AD01084A
:107D400091B70108BA4A804600264FF0010909FAA6
:107D500006F313EA080F1AD00DF11C0A0427F3B238
:107D60004FF0000B1AF8011B0091CDE9019B102187
:107D700020460593FFF71EFE94F82310052900F016
:107D8000BC80013F17F0FF07A94A059BEAD10136E5
:107D9000202EDCD168680368DB689847A44A8046D7
:107DA00000264FF0010B0BFA06F313EA080F1AD066
:107DB0000DF11C090427F3B24FF0000A19F8011B5A
:107DC0000091CDE901AA102120460593FFF7F2FDAD
:107DD00094F82310052900F09080013F17F0FF0769
:107DE000934A059BEAD10136202EDCD16868DFF882
:107DF00048A203689B689847002780464FF0010916
:107E000009FA07F313EA080F15D01026FBB24FF05A
:107E1000000B5246CDE9019B0096032120460593B5
:107E2000FFF7C8FD94F82320052A66D00136F6B284
:107E3000142E059BEDD10137202FE1D16868DFF8C2
:107E4000F4A103689B689847002780464FF001091A
:107E500009FA07F313EA080F15D01426FBB24FF006
:107E6000000B5246CDE9019B009615212046059353
:107E7000FFF7A0FD94F82320052A3ED00136F6B284
:107E8000182E059BEDD10137202FE1D16868694E8E
:107E90000368DB689847002780464FF0010A0AFA1A
:107EA00007F313EA080F15D014255FFA87FB4FF08C
:107EB00000095B46CDE9019900953246152120461F
:107EC000FFF778FD94F82330052B16D00135EDB27D
:107ED000182DEED10137202FE1D10EE01E230093A3
:107EE000CDE9018AF3B24A4600212046FFF762FD40
:107EF00094F82330052B7FF4C4AD09B0BDE8F08FB2
:107F00001E230021CDE90031CDF80880F3B252469E
:107F10002046FFF74FFD94F82330052B7FF4C5ADC5
:107F2000EBE70D230093CDE9018AF3B24A460C2119
:107F30002046FFF73FFD94F82330052B7FF4C9ADB1
:107F4000DBE7F1B26923CDE900790C2220460591E7
:107F5000FFF7B8FC94F82330052BCED06823CDE989
:107F6000007905990C222046FFF7ACFC94F82330E9
:107F7000052B7FF4C0ADC0E7F1B26923CDE90089DC
:107F80000C2220460591FFF79DFC94F82330052B29
:107F9000B3D06823CDE9008905990C222046FFF76C
:107FA00091FC94F82330052B7FF4B8ADA5E71C2392
:107FB0000093CDE90188F3B24A4605212046FFF738
:107FC000F9FC94F82330052B7FF4BBAD95E71E2315
:107FD0000093CDE90188F3B24A4605212046FFF718
:107FE000E9FC94F82330052B7FF4BEAD85E71C2314
:107FF0000093CDE9018AF3B24A4605212046FFF7F6
:10800000D9FC94F82330052B7FF4C2AD75E71E230D
:108010000093CDE9018AF3B24A4605212046FFF7D5
:10802000C9FC94F82330052B7FF4C6AD65E700BF8B
:1080300011BE0108599401087D8C01080C2300939E
:10804000CDE9018AF3B24A4606212046FFF7B2FC89
:1080500094F82330052B7FF4C3AD4EE70C23009337
:10806000CDE90188F3B24A4606212046FFF7A2FC7B
:1080700094F82330052B7FF4C6AD3EE7CDE901BA75
:108080003B7800934A465FFA88F307212046FFF7C2
:1080900091FC94F82330052B7FF4CFAD2DE700231E
:1080A000CDF808A001933B7800934A465FFA88F325
:1080B00007212046FFF77EFC94F82330052B7FF440
:1080C000D0AD1AE70C230093CDE90189F3B25246F3
:1080D0000F212046FFF76EFC94F82330052B7FF428
:1080E000DAAD0AE70C230093CDE90188F3B25246DA
:1080F0000F212046FFF75EFC94F82330052B7FF418
:10810000DDADFAE630230093CDE90189F3B25246A2
:1081100009212046FFF74EFC94F82330052B7FF40D
:10812000E0ADEAE630230093CDE90188F3B2524690
:1081300009212046FFF73EFC94F82330052B7FF4FD
:10814000E3ADDAE670B50446FFF784FC94F823301B
:10815000052B29D0002594F83F33EB40DB07E8B22C
:1081600015D40135082DF6D194F82330052B1BD0FA
:1081700094F8203013B194F82230ABB90B4B0C4972
:108180001B6898690368BDE870401B68184703F0D6
:1081900087FB02460028E4D011212046FEF7D8FFD5
:1081A00094F82330052BDCD170BD00BF105E002099
:1081B000582709082DE9F04F90F9213089B004467D
:1081C000002B00F00481012300F50C7580F8413389
:1081D000024600F50F712B462E46D06E002859D06E
:1081E000002384F8413394F94030642B5BD094F938
:1081F000BC30642B00F08D8094F93831642B00F092
:108200008A80D4F830722FBB01A920462BF078F871
:1082100000B30C230593012306978DF81830714B9A
:1082200007936946BDF80430049704A8ADF81030F0
:108230008DF800702BF0E6F99DF9001051B102297C
:1082400008DC38B1C9B27C2303FB01416C312846FC
:108250002CF038FE94F841B3BBF1000F5DD0E36E13
:108260006367D4F8E830C4F8F030D4F86431C4F867
:108270006C3194F8233003F1C30204EB8202002135
:10828000042B7CD852F8040B1061013342F8041C13
:10829000DBB2F5E753F8040B0028A1D18B4202F1C1
:1082A0007C029AD19FE7002066238DF810307C2352
:1082B00003FB004004A940302CF048FD04A92046EF
:1082C0002BF01EF800289CD004238DF818300023D2
:1082D000CDE90133039331230593694604A82BF0BC
:1082E00091F9059B28B108AA02EB8302009942F894
:1082F000E01C0133332B0593EFD94EF0B7F99DED18
:10830000031ADDED020A9DED010A66214EF06CF9BB
:1083100077E70120C8E70220C6E70127A94655F8FC
:10832000043B23B1AB600137042FF7D197E7AA468E
:10833000B8465FFA88F3022BF5D8DAF8002055F832
:10834000043C9A4205D104A95046CDF810B02CF057
:10835000B9FD5AF8043B08F101020BB99046E8E771
:1083600004A906EB88000193CDF810B02CF0AAFD0B
:10837000019BAB6001A948462CF0A4FDD3E794F81B
:10838000413313B92046FEF7BFFD94F822300BB3FA
:10839000154B1B68986A036864215B689847204600
:1083A000FFF786F994F83E3003B9E36694F8BA30E3
:1083B0000BB9C4F8E83094F836310BB9C4F864311D
:1083C000FAF764FEFAF7CEFE0123A4F8403309B0B1
:1083D000BDE8F08F2046FFF7B5FE94F82230002B61
:1083E000E0D0D5E700C40908105E00207047000007
:1083F000012070470120704743689868704700006B
:1084000010B5054B03600446C06A10B103685B6891
:108410009847204610BD00BF1C2C0908406803681F
:108420009B6A184733B46C46406884E80C000368C4
:10843000DD6A94E80C00AC4602B030BC6047000036
:1084400010B50446FFF7DCFF2046FEF76BFC204624
:1084500010BD000040680AF08BBB0000406801239B
:108460000AF086BB40680AF05FBB000040680A2241
:108470000AF004BB40680AF019BB000090F83130E4
:1084800013B1002101F028B97047000040680AF0DC
:1084900093BB000073B5044605250026E06A8DF8FD
:1084A000076003680DF10702DB680121984778B186
:1084B0009DF807300C2B09D0102B05D0092B07D1C4
:1084C00084F8333002B070BD1523F9E71423F7E7C1
:1084D000013DE3D12846F5E710B4C06A03681C6982
:1084E0000822A44601235DF8044B312160470000B7
:1084F00010B4C06A03681C690122A44600235DF819
:10850000044B322160470000F7B50446C06A036897
:108510005B6998470546002871D0E06A03685B698B
:10852000984703689B689847E06A03689B69984787
:1085300060B9344B34491B68986903681B689847D5
:108540002B682846DB689847002655E02046FFF751
:10855000CFFF0028F4D02046FFF79CFF0028EFD083
:10856000E06A03680121DB6A98472046FFF7B4FF01
:1085700030B9244B25491B68986903681B68DEE7FE
:10858000E06A0368DB69984730B91E4B20491B68D5
:10859000986903681B68D2E7E06A94F833100127F2
:1085A00084F8317003685B6A9847E06A03689B6AE5
:1085B00098470146204601F0F1F806460028BFD052
:1085C00094F830301BB13946204601F0F7F894F8A2
:1085D0003210204601F018F92B682846DB689847CE
:1085E000E06A009403681D6A0A4B019302AB13E929
:1085F0000C0042F21071A847304603B0F0BD0646A9
:10860000FAE700BF105E0020882B0908AE2B09088E
:10861000CD2B09080987010870B5002586B0CDE982
:10862000005500230446C06A8DF808500593039353
:10863000049303686A469E6810210923B047A0B1DD
:108640009DF8003013F0010615D194F83430013351
:10865000DBB2052B84F8343007D12046FFF748FF02
:108660002046FFF739FF84F83460E06A03681B6B2B
:10867000984706B070BD9DF8083084F834501B0749
:10868000F3D4BDF901309FED1E6A06EE903ABDF9B4
:10869000033007EE103ABDF90530F8EEE66A07EE52
:1086A000903ACDED036AF0EEE66AB8EEC77AF8EEDE
:1086B000E77AF4EEC66AF1EE10FA8DED047ACDEDAC
:1086C000057A0DD5B0EEC77AB4EEC67AF1EE10FA9F
:1086D00006D5F0EEE77AF4EEC67AF1EE10FAC4D4DD
:1086E0009FED080A03A811F083F8B2EE040A03A86C
:1086F00011F07EF80A2203A9204601F0EBF8B4E756
:10870000000000349A99193EFFF786BF10B5044B5C
:10871000044640F8043BFFF7CBF8204610BD00BFED
:10872000342C090810B50446FFF7F0FF2046FEF789
:10873000F9FA204610BD0000F7B503680F4616464B
:108740001BB90024204603B0F0BD002404600820BB
:108750000193FEF7DFFA054620B1124B0360019B3F
:108760004360019401A8FFF7A3F8002DE9D0382059
:10877000FEF7D0FA04460028E3D000F0ADFE0A4B25
:10878000E562236084F8307084F832602046FFF799
:10879000BBFE05460028D5D1236820465B68984774
:1087A0002C46CFE7342C09081C2C09082DE9F74F7B
:1087B000046806460D4690469946002C6CD00B681E
:1087C000002B49D0236820469B6A984703689B6822
:1087D0009847012328680DEB030200210AF0C8F92D
:1087E00098B39DF80130EA2B2FD1DFF8F0B04FF0AD
:1087F000060A28680023802206210AF095F920B392
:10880000DBF80070B86A03680A215B6898470023A8
:1088100028681A4606210AF087F9B0B1B86A0368D9
:108820000A215B689847012328680DEB03020621A3
:108830000AF09EF948B19DF8014014F040042FD091
:108840000AF1FF3A1AF0FF0AD3D1306803689B6A35
:1088500098470368DB68984700241DE002222346FE
:108860000F2128680AF060F9B86A036801215B6883
:108870009847306803689B6A98470368DB689847A5
:10888000336834604A46414601A80193FFF754FF1C
:10889000044601A8FFF70CF8204603B0BDE8F08FAE
:1088A000224623460F2128680AF03EF9B86A036879
:1088B00001215B6898470223214630680DEB0302D3
:1088C0000AF056F904460028C8D0B869024903687E
:1088D0001B689847B9E700BFF42B0908105E002019
:1088E000002100F0F9BE000070B504468CB00426EB
:1088F000013E76B2731C4AD0E06A15236A465D21B8
:108900000AF036F90028F3D0E06A152306AA5D21A3
:108910000AF02EF905460028EAD0152206A9684675
:1089200070F03AFC0028E3D19DF8003084F8303034
:108930009DF8073084F832309DF8143084F83C30CC
:108940009DF813309DF8102084F83D309DF80F30CD
:1089500043EA0223E3879DF8013084F831309DF823
:10896000083084F83330039B9DF80C20C3F30F23A9
:10897000A3869DF80B3043EA0223E386049BC3F3EE
:108980000F232387019BC3F30F23638707E0054B66
:1089900005491B68986903681B68984700252846A5
:1089A0000CB070BD105E0020682C09082DE9FF4155
:1089B00004460023C06A8DF807300368DFF8508151
:1089C0009B6A984703689B689847E06A03680A2196
:1089D000DB6C9847E06A0A2204210AF04FF804256C
:1089E000013D6DB26B1C32D000234B21E06A822224
:1089F0000AF09AF8D8F800600746B06A03680221C6
:108A00005B689847002FEBD001231A464B21E06AA0
:108A10000AF08AF80746B06A036802215B68984743
:108A2000002FDDD0E06A01230DF1070240210AF09A
:108A30009FF80028D4D09DF80720322A10D0002DAE
:108A4000CED1B069304903681D683223A847E06A77
:108A500003689B6A98470368DB68984700254EE0E7
:108A60002046FFF741FF0028F1D0E06A01231722DA
:108A700051210AF059F80028E9D05222E06A012376
:108A800011460AF051F80028E1D0E06A01233822AB
:108A90004C210AF049F80028D9D0E06A03689B6AA3
:108AA00098470368DB689847E06A052109F0FEFFF4
:108AB000E36A2046996800F071FE0546F8B194F823
:108AC0004410204600F0A0FE94F845301BB101216F
:108AD000204600F073FEE06A03680221DB6C9847D1
:108AE000E06A02940368DE6A084B039304AB13E95F
:108AF0000C0044F21B11B04750F010F820642846D7
:108B000004B0BDE8F08100BF902C0908798C010801
:108B1000105E002070B5C58F90F93D60AD03B5FBC8
:108B2000F2F2A2F5804404FB04F2D51190F83C2047
:108B30000498D201624306FB05225212A03002F5CE
:108B40008012424312134A43DB0003EB623000B24F
:108B500070BD000010B5848E53005C43B0F93A300C
:108B6000C91AC38FD31AB0F93820B0F9360053436D
:108B700004F500449B10C3EBC13300EB24400449CF
:108B800093FBF0F04FF400420EF096FD00B210BDE2
:108B90000080FFFF10B52DED028B8AB0044608233C
:108BA000C06A05AA422109F0E3FF18B1BDF81A20F6
:108BB000D30719D4E06A09F0FFFF4FF0AFFF236C31
:108BC000C31AFA2B0CD92064002382224B21E06ABD
:108BD00009F0AAFF0123E06A1A464B2109F0A4FF1D
:108BE0000AB0BDEC028B10BDBDF9141094F93230FF
:108BF0000093920894F930300392C9102046FFF791
:108C000089FFBDF9161094F93330039A009308EEEA
:108C1000900A94F93130C9102046FFF77BFFBDF967
:108C20001810039A491008EE100A2046FFF792FF29
:108C300007EE900AF8EEE88AF8EEE77AB8EEC88A0E
:108C4000B3EE000A07A8CDED097ACDED078A8DEDC8
:108C5000088A10F0E1FDB2EE040A07A810F0C8FD82
:108C60004FF05CFF0A22206407A9204600F032FE84
:108C7000E06A09F0A1FFB3E7FFF78CBFF7B503681F
:108C80000D4616461BB90024204603B0F0BD002750
:108C9000076048200193FEF73DF8044650B100F00C
:108CA0001BFC0D4B2360019BE362019784F8446039
:108CB00084F8455001A8FEF7FBFD002CE3D02046C8
:108CC000FFF774FE05460028DED1236820465B6866
:108CD00098472C46D8E700BFC82C090810B5044BAC
:108CE000044640F82C3BFEF7E3FD204610BD00BFD4
:108CF000C82C090810B50446FFF7F0FF2046FEF720
:108D000011F8204610BD0000002100F0E5BC000075
:108D1000F8B504460D4617461E4600F0DDFB094B2C
:108D200023602B68E362002200232A6084F83070FD
:108D300084F831606365A365E36523666366A366B3
:108D40002046F8BDE02C0908F8B51C460933164644
:108D5000DB086A46A2EBC30300AF9D46C06AA31CB2
:108D60006A4609F005FF054628B122460DF10201C9
:108D7000304670F021FA2846BD46F8BD2DE9F34192
:108D800006460F4614464FF0C9FE114BD3F800803B
:108D90000546D8F82800036801215B68984701233D
:108DA0000DF1070207213046FFF7CEFF60B19DF8B5
:108DB0000730DA0702D4B7EB531F05D04FF0AEFEF1
:108DC000431BA342E5D3002002B0BDE8F08100BF01
:108DD000105E00202DE9F041DFF8608292B0044679
:108DE00002AF002646F02002E06A0023D2B25021F2
:108DF00009F09AFE002800F00C810325013D6DB2B8
:108E00006A1C00F00681D8F80030986A03684FF4B5
:108E100096719B68984701230DF106025521204663
:108E2000FFF792FF002800F0F4809DF8063013F061
:108E3000E00F40F0EE80DB07E0D502230DF10602E3
:108E400052212046FFF780FF002800F0E280BDF8A5
:108E5000063001365BBA202E27F8023BC2D1BDF89E
:108E600024309DF826109FED6D7ADFED6D6A9FED41
:108E70006D6A43F30B0207EE902A1B0903F470633B
:108E8000BDF82620F8EEE77A0B4343F30B03C4ED5D
:108E90000D7A07EE903A02F470639DF82820F8EE00
:108EA000E77A134343F30B03C4ED0E7A07EE903ACF
:108EB0009DF92230F8EEE77AC4ED0F7A07EE903A8A
:108EC0009DF92930F8EEE77A67EE877A07EE103AD7
:108ED000B8EEC77A9DF92A30C4ED107A27EE267ACB
:108EE000DFED517A84ED117A07EE103AB8EEC77AC9
:108EF0009DF92B30E7EE267AC4ED127A07EE903A10
:108F0000F8EEE77A9DF9233067EEA67ADFED476A3F
:108F1000C4ED137A07EE903A9DF92C3007EE103A23
:108F2000B8EEC77A9DF92E3027EE267AF8EEE77A6A
:108F300084ED157A67EE867A07EE103A9DF93030A7
:108F4000C4ED147A07EE903AF8EEE77A9DF92D30E9
:108F500067EEA67AB8EEC77AC4ED177A27EE267ABE
:108F600007EE903A84ED167AF8EEE77A9FED307AC4
:108F70009DF92F3067EE877AC4ED187A07EE903AA4
:108F80009DF93130F8EEE77A06EE903A67EE877A8F
:108F9000F8EEE66AC4ED197ADFED267ABDF93830CD
:108FA000E6EE877A07EE103A9DF93230C4ED1A7A70
:108FB000B8EEC77AF3EE077AE7EE067A07EE103AD4
:108FC000DFED1D6AC4ED1B7AB8EEC77A27EE267A6C
:108FD00084ED1C7A9DF9333007EE103AB8EEC77A6B
:108FE0009DF9343027EE267A84ED1D7A07EE103A8B
:108FF0009DF9353007EE903AB8EEC77AF8EEE77A89
:1090000027EE267A67EEA67A84ED1E7AC4ED1F7AE3
:1090100000E0002012B0BDE8F08100BFCDCC4C3E96
:109020000000803B0000003B0AD7233C0000003DCD
:109030000000803817B7D1B80AD7A33A105E0020D5
:1090400073B501230E460DF1070206210446FFF712
:109050007BFE18B90025284602B070BD9DF8073088
:10906000013B012B0CD80023E06A1A46062109F0C7
:109070005BFD0028EED0062200212046FFF77EFE91
:10908000E06A00233246062109F04EFD054600281D
:10909000E0D0262231462046FFF770FEDBE70000D5
:1090A00013B501230DF1070207210446FFF74CFE1B
:1090B00010B9002002B010BD9DF807301B070CD579
:1090C0000023E06A1A46062109F02EFD0028F0D0A0
:1090D000062200212046FFF751FEE06A0023072206
:1090E000062109F021FD0028E3D0132207212046A4
:1090F000FFF744FE0028DCD0E06A002305220621A9
:1091000009F012FD0028D4D0172205212046FFF7D0
:1091100035FE0028CDD001212046FFF791FFC9E799
:10912000F7B50446C06A544F03689B6A98470368C2
:109130009B689847E06A03680A21DB6C9847E06AFD
:109140000A22042109F09AFC0525013D6DB26B1C31
:1091500000F08980E06A0023B6227E2109F0E4FC59
:109160000028F2D03B68986A036818215B686E4655
:1091700098470123324600212046FFF7E5FD0028ED
:10918000E3D09DF80030332BDFD12046FFF722FEDD
:10919000002868D0E06A00238022502109F0C4FC36
:1091A000002860D02046FFF77BFF00285BD0E06AF4
:1091B000002386222E2109F0B7FC002853D0E06A54
:1091C00000232422042109F0AFFC00284BD0E06AE0
:1091D00000230222062109F0A7FC002843D0142214
:1091E00002212046FFF7CAFDE06A0023072205217D
:1091F00009F09AFC002836D001212046FFF720FF15
:10920000002830D0E06A03680321DB6C9847E06AED
:1092100003689B6A98470368DB689847E06A1721F0
:1092200009F044FCE36A2046996800F0B7FA054665
:10923000B0B194F83110204600F0E6FA94F83030DE
:109240001BB10121204600F0B9FAE06A0368DF6A29
:109250000A4B0094019396E80C0042F21071B84753
:10926000284603B0F0BDE06A03689B6A984703682C
:10927000DB6898470025F3E7105E0020559401084D
:1092800010B586B00C236A4631210446FFF75CFD19
:10929000002800F0D5809DF80A309DF809209FED48
:1092A000697A9FED696ADFED694A94ED115A94ED90
:1092B0001D4A94ED1E3A1B0403EB02239DF80B207C
:1092C00003EB02631B1207EE903AF8EEE77AF7EE33
:1092D000006AA7EE876A9DF801309DF80020D4ED62
:1092E000147A94ED107A77EEA67A1B04A7EE867AAC
:1092F00003EB02239DF8022094ED0D6AD4ED157A5C
:1093000003EB02631B12F0EE475A07EE103AB8EE79
:10931000C77A35EE265A27EE247A9DF804309DF858
:109320000320A5EE076A1B0403EB022394ED1B7ACE
:109330009DF8052094ED135A35EEC77AD4ED185AEE
:10934000A7EE876A03EB02631B12F0EE667AE7EE84
:10935000257A9DF80620D4ED125AC6EE273A03A9C5
:10936000204607EE903AF8EEE77A75EEA65A67EED9
:10937000A47A94ED0E6A9DF80730D4ED1C4AA5EE50
:10938000A76A1B0403EB0223D4ED165A9DF80820AC
:10939000F0EE467A94ED196AE7EE257A03EB026364
:1093A0001B12F0EE665AE7EE065A0A2235EE265AEE
:1093B00087EEA56A07EE903ADFED255AF8EEE77AD8
:1093C00067EEA57AD4ED0F5AE5EE275AD4ED177A59
:1093D00094ED1A5AE7EE275AF0EE667AE7EE057A30
:1093E000E4EEC46AC5EEA72AF0EE637AE4EEC67A2C
:1093F00094ED1F7A87EEA65AF0EE467AE4EE637A91
:10940000C7EEA65AF0EE437AD4EE077AA4EEC37AFA
:1094100026EE476AB2EE047AA7EEA36A25EE075A53
:10942000C6EE267A65EE875A77EEA27A8DED035A5C
:1094300067EE877ACDED045ACDED057A00F04AFA51
:1094400006B010BD5B9E803A85EBCBC147ABE73BD6
:10945000F61BEB3BFFF714BF30B51346026885B02F
:109460000D461AB90024204605B030BD0021016028
:10947000802001930392FDF74DFC044620B1019B2F
:109480002A4603A9FFF744FC03A8FEF711FA002CB3
:10949000E8D02046FFF744FE05460028E3D12368C4
:1094A00020465B6898472C46DDE7000010B5044B6A
:1094B000044640F82C3BFEF7FBF9204610BD00BFE8
:1094C000E02C090810B50446FFF7F0FF2046FDF731
:1094D00029FC204610BD0000064B10B50360044671
:1094E000FEF7D6F9A06004F10C004EF07FFC204698
:1094F00010BD00BFF82C090873B505467C23AC6885
:109500002E7903FB0643C6EB461604EB8604084699
:1095100093F8A410019010F001FA94F93C300198EE
:109520003BB9AB6893F8251002B0BDE8704010F06D
:10953000F5B994F84010F7E737B5846805790191DB
:109540007C2303FB054595F83F3004EB8304D4F8F6
:109550004C325BB14FF0E2FAC5F89C000199D4F8A7
:109560004C0203B0BDE8304003F0F8BD03B030BD9D
:109570002DE9F04F90F804A08768CAEB4A144FEA2F
:10958000840806460D4607F13C0B08F108018BB034
:109590005944284610F0F8F83179B0680BEB840490
:1095A000FEF71CF938B17C2303FB0A7393ED1A0A0A
:1095B000284610F01DF97C2303FB0A7393ED146A0F
:1095C000DFED3A7AD3ED156AB0EEC67AB4EEE77AFB
:1095D000F1EE10FA0FD5B0EEE67AB4EEE77AF1EEDE
:1095E00010FA08D594ED077AB0EEC77AB4EEE77AB0
:1095F000F1EE10FA1BD47C2303FB0A73D86D196EAD
:109600005A6E9B6D029003910490079101A8294620
:109610008DED016ACDED056A0692089209930EF070
:1096200011FA85ED000AC5ED010A85ED021A7C23C9
:1096300003FB0A770023C7F88C30C7F88830C7F8D7
:109640008430B06890F95C3208F13C0908F14808B0
:10965000D944D8446BB133795BB9414600F51670F3
:1096600004F034FA414628460BB0BDE8F04F10F044
:109670008BB890F93430012B0BD190ED0E0A48468F
:1096800010F062F884ED120AC4ED130A84ED141A86
:10969000E8E7022BE6D1FCF723FF002201A9FCF743
:1096A0001FFC0028DED09DED010AE8E70000003431
:1096B00010B5037984687C2202FB034407C904F1D6
:1096C000900383E807004FF029FAC4F89C004FF09C
:1096D0001DFAC4F8A00010BDF0B5054685B0A6225D
:1096E0000E4600F10C0103A809F094FCAC682F7938
:1096F0007C2303FB0743D3F8B42022B903A809F065
:10970000ABFC05B0F0BDBEB196ED007AD3ED2A7A80
:1097100067EE877AC3ED2A7A96ED017AD3ED2B7A3C
:1097200067EE877AC3ED2B7A96ED027AD3ED2C7A29
:1097300067EE877AC3ED2C7A7C2607EE902A06FB2B
:109740000741A831B8EE670A0846019110F064F8A5
:1097500001992846FFF7ACFF06FB07430022C3F838
:10976000B020C3F8AC20C3F8A8200022C3F8B4206E
:10977000C4E7000073B504468068237901917C2614
:1097800006FB03000D466C3001A92BF07BFBA368A0
:10979000227906FB02331D6702B070BD70B5021D51
:1097A000044680680E46FDF7FFFB054618B13146BA
:1097B0002046FFF7DFFF284670BD000007B582682E
:1097C00003797C2000FB032090F93C0002280BD099
:1097D00002F13C00C3EB43138DF8071000EB83004C
:1097E0000DF107012BF0A8FA03B05DF804FB0000AF
:1097F000836802797C2101FB023393F93C00003835
:1098000018BF012070470000836802797C2000FBAC
:10981000023383F8A4107047F8B5054608460F4692
:1098200010F058F810B100242046F8BD384610F06A
:1098300037F804460028F6D1AB6893F934637EB15B
:10984000384610F07FFB95ED097ADFED1F7AF0EED8
:10985000C76AF4EEE76AF1EE10FA03D585ED090A5E
:109860000124E1E777EE407A30EE076AF0EEE77A1E
:10987000C7EE866AF6B207EE906A9FED146AF8EEBC
:10988000677A26EE866AF4EEC67AF1EE10FA48BFE1
:10989000B2EE046ADFED0E7A45BFAB6A66EE866A09
:1098A000B0EE676A87EEA66A46BF0133AB62012459
:1098B000F7EE007A77EEC67A20EE060AA7EE270AC0
:1098C00085ED090AB0E700BF0000003400004843FE
:1098D000CDCCCC3D2DE9F74304460E461746FFF7A5
:1098E0000BFE31462046FFF727FE31462046FFF7A4
:1098F0003FFE31462046FFF78FFF30B304F10C01E5
:10990000992201A809F086FBA56894F804804FF01D
:109910007C0909FB0854A834314620460FF034FF77
:1099200009FB0851D1F8B4300133C1F8B4304FB15C
:10993000BB4207D35B08C1F8B430B0EE000A204642
:109940000FF06AFF01A809F087FB03B0BDE8F083C0
:1099500010B50446FDF7C2FBC0B23C34C0EB40106A
:1099600004EB800010BD0000F8B50A4E044600F577
:10997000167704F5137555F8040B08B103F022FFB0
:10998000BD42F8D13368986A036801215B68984743
:10999000EFE700BF105E002008B5FFF7E5FF00000D
:1099A000F0B5144E00EB810773780446D7F84C02EB
:1099B0006FF3410387B00D467370C8B102F0F0FA3F
:1099C00068B1737843F0100373702C440023A372C2
:1099D000D7F84C0207B0BDE8F04002F065BAD7F8FE
:1099E0004C12684602F00CFB009B012BEDD1E8E71E
:1099F00007B0F0BDDC5E002070B506460D460024C1
:109A000045FA04F3DB07E1B202D53046FFF7C8FFA1
:109A10000134032CF4D170BDFF21FFF7EDBF00002E
:109A200030B500F5137587B000F5167455F8041BB2
:109A300021B9A542FAD1002007B030BD684602F036
:109A4000DFFA009B013B022BF3D80120F4E7000072
:109A50002DE9F0472DED028B88B004460D46904667
:109A6000B0EE408AFDF702FE30B90026304608B05D
:109A7000BDEC028BBDE8F08729462046FDF770FC5F
:109A800006460028F1D004EB8507D7F83C22D7F82A
:109A900030329A4206D038F025F95C4A032132F080
:109AA000EFFFE2E7D7F84C3283B94FF49870FDF737
:109AB00031F9814608B102F089FFC7F84C92B9F13B
:109AC000000F03D138F00EF9514AE7E7B4F84A32F3
:109AD000D90711D505F0E8FD90F8082390F8C432B5
:109AE00032B9B02202FB030090F8A130012B03D859
:109AF00038F0F8F8474AD1E72046FFF791FF20B940
:109B0000454A537843F00203537094F9353053B308
:109B100029462046FFF71CFF90F90030002B53D058
:109B200029462046FFF714FF90F80490B9F12B0F57
:109B300019D829462046D7F84CA2FFF709FF94F917
:109B4000353090F90020022BD4BF00210121012BD8
:109B5000D4BF00230123003A009118BF01224946D7
:109B6000504602F0B5F9631900229A7275B3D4ED2C
:109B7000C10AB4F84822D7F84C0270EEA00A2B466E
:109B8000B0EE480A414602F0C3F994F83E33002B88
:109B900031D1224A069412680127E773906A02685D
:109BA000156D1F4A0792029309224FF40063CDE915
:109BB000003208AA12E906001A4BA847C8B938F0C3
:109BC00091F8194A02216AE79946B2E729462046E8
:109BD000FFF7BEFE90F90030002BC8D0D4EDC10ACB
:109BE000B4F84822D4F84C022B46B0EE480A41465D
:109BF000C9E784F83E7300230DF1170104F1240036
:109C00008DF817302BF0A2F830E700BF082D0908B7
:109C10003A2D09085D2D0908DC5E0020105E002049
:109C2000999901087B2D0908862D09082DE9F04135
:109C30002DED028B002443739DF82030837305467D
:109C40000F469046B0EE408A264647FA04F3DB07FB
:109C5000E1B210D5B0EE480A42462846FFF7F8FEBA
:109C6000064640B939462846FFF7C6FEBDEC028BD2
:109C70003046BDE8F0810134032CE6D1F6E7000060
:109C8000F8B500242DED028B05460F46B0EE408A54
:109C9000427383732646E1B2B0EE480A3A4628463C
:109CA000FFF7D6FE0134002818BF0646032CF2D178
:109CB000BDEC028B3046F8BDF0B500EB81030D46DC
:109CC000D3F84C129BB0044611B900201BB0F0BD74
:109CD0000BA802F079F96319987A0028F6D10B9A4B
:109CE000002A48D0042AF0D101229A720DAA07CA8C
:109CF00002AB83E8070010AA07CA05AF87E8070090
:109D000013AA07CA9DED180A08AE86E807001A468E
:109D1000294620468DED010AFDF7C6FA3A46294646
:109D20002046FDF76DFA324629462046FDF77AFABD
:109D30009DED010A29462046FDF786FA9DF864301C
:109D400083B129462046FFF703FE90F900304BB15E
:109D500094F93530012B05DD9DF85D20294620461C
:109D6000FDF7BAFA2046FFF75BFE20B9034A5378A5
:109D700043F0040353700120A8E700BFDC5E00201D
:109D80002DE9F0410546884600F5137700240126A9
:109D900057F8043BE1B26BB148FA04F3DB0709D58D
:109DA0002846FFF789FF002857F8040C08BF002653
:109DB00002F07AF80134032CEAD13046BDE8F08194
:109DC0002E4B2DE9F04F1F68FB6A93F89C8087B0FB
:109DD0000446B8F1000F38D1DFF8A8A000F51376DB
:109DE00000F1030B054656F8040BA5EB04095FFAD6
:109DF00089F9E8B102F0C0F828B19AF8013043F0CF
:109E000008038AF8013056F8040C02F0C9F8F8B9D2
:109E1000637B6BB1AB7A5BB956F8041C684602F001
:109E2000EFF8009B042B03D149462046FFF744FF7F
:109E300001355D45D7D1124B204683F81280FFF7DC
:109E4000EFFD054630B10123237407B0BDE8F08F64
:109E50008046EDE7237C002BF7D0A37B002BF4D0CA
:109E6000B86A03684FF47A715B689847B86A036808
:109E70009B6B294607B0BDE8F04F1847105E0020E5
:109E8000BD5E0020DC5E0020F0B5002587B000F547
:109E900013762C46012756F8041B41B1684602F0A0
:109EA000AFF8009B1BB107FA05F31C43E4B2013580
:109EB000032DF0D1204607B0F0BD00002DE9F04F92
:109EC0002DED028B03270E7C9FED348A91B0054661
:109ED0008846B946AC5D0134E4B2B4FBF9F303EB58
:109EE0004303E41AE4B205EB8403D3F84C1209B936
:109EF000AC554CE003A802F083F8DDF80CB00BF190
:109F0000FF33022BF4D8304631F092FB82463046C4
:109F100032F058FB00F11B039A4508D2304632F06C
:109F2000B9FF002011B0BDEC028BBDE8F08FAC553D
:109F3000284698F810A0FFF7A7FFDDED057A8DF809
:109F40003100FCEEE77A9DF810208DF8332017EEF3
:109F5000903A8DF8343006AB03CB1B88ADF83D301A
:109F60005C221B23CDE90032CDF83500CDF8391045
:109F700009AABF2150468DED098A8DED0A8A8DED23
:109F80000B8A8DF830408DF832B031F0BBFB013FC9
:109F900017F0FF079ED10120C4E700BF00000000BA
:109FA0002DE9F04F0F7CA1B006468846032500EB53
:109FB000070999F805400134E4B20323B4FBF3F335
:109FC00003EB4303E41AE4B206EB8403D3F84C1228
:109FD00011B989F805400AE011A801F0F5FFDDF894
:109FE00044A0BAF1030F08DCBAF1000FF1DA013D29
:109FF00015F0FF05DDD1012012E0AAF10402032AC9
:10A00000F5D8384631F014FB8346384632F0DAFA98
:10A0100000F13602934506D2384632F03BFF00206D
:10A0200021B0BDE8F08F89F80540304698F810B0AF
:10A03000FFF72AFFDDF848E0CDF80CE0DDF84CE052
:10A04000CDF810E0DDF850E0CDF814E0DDF854E094
:10A05000CDF818E0DDF858E0CDF81CE0DDF85CE064
:10A06000CDF820E0DDF860E0CDF824E03219DDF82D
:10A0700064E01C9BCDF828E0DDF868E092F80AC0A7
:10A080009DF874109DF87520CDF82CE00E93DDF846
:10A090006CE01E9B8DF835008DF83C108DF83D204E
:10A0A000CDF830E08DF834408DF836A08DF837C00B
:10A0B0002422CDF83E303623CDE90032C0212C23B6
:10A0C00003AA584631F01EFB91E700007FB58A8B4A
:10A0D0000B464AF2B9518A4205465FD04AF2BA515C
:10A0E0008A4274D04AF2B8518A420BD1474A126868
:10A0F000D26A92F89C203AB137F0F4FD444A052127
:10A1000032F0BEFC042479E0D3ED007AF5EEC07A9B
:10A11000F1EE10FAF6D49FED3F7AF4EEC77AF1EE45
:10A1200010FAEFDC93ED017ADFED3B6A1C6993EDE9
:10A13000030AB0EEC77AB4EEE67A93ED027AFCEE4B
:10A14000E77AB0EEC77AF1EE10FAB4EEE67A17EEDF
:10A15000903A54BF01260026F1EE10FA54BF0122B6
:10A160000022003C18BF012413F0FF0110D18DED37
:10A17000030A0292FDF700F89DED030A029A2346B6
:10A1800031462846FFF77CFD0028BBD0002435E08F
:10A19000134600943246FFF749FDF5E7D3ED007A08
:10A1A000F5EEC07AF1EE10FAACD49FED1A7AF4EE27
:10A1B000C77AF1EE10FAA5DCFCEEE77A17EE903ADA
:10A1C00013F0FF0108BFFF21FFF7DAFDDCE7D3ED55
:10A1D000007AF5EEC07AF1EE10FA93D49FED0D7A85
:10A1E000F4EEC77AF1EE10FA8CDCFCEEE77A17EEAB
:10A1F000904A14F0FF0404D1FFF70EFC204604B08F
:10A2000070BD2146FFF7F8FBC0E700BF105E0020DD
:10A21000B82D090800007F4300000034F0B58BB072
:10A220000E4614460746FFF793FB543007C884E8F0
:10A23000070031463846FFF78BFB90ED057ADFEDDE
:10A24000267AB0EEC77AB4EEE77AF1EE10FA054658
:10A2500011D590ED067AB0EEC77AB4EEE77AF1EE5A
:10A2600010FA08D590ED077AB0EEC77AB4EEE77A27
:10A27000F1EE10FA24D431463846FFF769FB016A43
:10A28000426A836AE869D5F814E0D5F818C00990E5
:10A2900001A8CDF804E0029103920491CDF814C016
:10A2A0000693079208930DF079FD98B1214601A815
:10A2B0000DF0C8FB84ED000AC4ED010A84ED021A1A
:10A2C00031463846FFF744FB00F1080120460FF005
:10A2D00075FA01200BB0F0BD000000342DE9F04705
:10A2E0002DED048BACB0B0EE608A0546B0EE409A1E
:10A2F0000F46F0EE418A9046FCF73EFFDFED8B7A89
:10A30000B0EEC87AB4EEE77AF1EE10FA4BD5B0EEC3
:10A31000E87AB4EEE77AF1EE10FA44D523AC2046A1
:10A32000FCF7D4F9F8F7B2FE2146F8F763FC0646CD
:10A3300058BB05F0B9F990F8083390F8C42233B14E
:10A34000B02303FB020393F8A130012B07D84FF091
:10A35000B00909FB020090F8A130022B0BD837F0AE
:10A36000C1FC734A032132F08BFB30462CB0BDECAC
:10A37000048BBDE8F08705F097F990F8C43209FB2B
:10A380000300AC300FC884E80F00DDED257A9FEDA7
:10A39000691AB8EEE78ADDED267AF8EEE78A28EE4C
:10A3A000018A68EE818A04AA03A902A8F0EE680A6D
:10A3B000B0EE480A03F056FC064618B937F092FC96
:10A3C0005D4ACFE79FED5D7ADDED027A9FED5C8A15
:10A3D000DFED5C8A8DED068A67EE877A2422002104
:10A3E00011A8CDED057A8DED078A6EF02FFF9DED5A
:10A3F000031ADDED040ADFF858A121EE281A68EEF1
